:020000040000FA
:1000000000F80202D16F0000F534000071420000D8
:1000100000000000000000000000000000000000E0
:1000200000000000804E0100C84E0100F5340000C1
:100030000000000000000000F534000055760000CC
:10004000ED320000F5340000F5340000F16F0000DF
:10005000794A00007D6B000085340000793500008E
:100060005918000095170000F5340000F93400001D
:100070004D4A0000958C0000716F00009D6F0000DC
:10008000F5340000F5340000F5340000B1790000CB
:10009000D1790000F5340000F5340000F53400009B
:1000A000657E00006F7E0000EF320000856E00006C
:1000B000F5340000E56B00000000000000000000C7
:1000C0000348854600F016FF0048004715CA0000A7
:1000D00000F8020230B50B46014600202022012420
:1000E00009E00D46D5409D4205D31D469540491B6C
:1000F0002546954040191546521E002DF1DC30BDB5
:1001000070B500242546002801DA01244042002968
:1001100001DA01254942FFF7DDFFAC4200D0404241
:10012000002C00D0494270BDF8B5002425460029B6
:1001300004DA0E46012400214042B141002B04DACA
:100140001E46002352420125B34100F0D1FC8C46EB
:1001500017461E46AC4203D0002540428D41AC46B6
:10016000002C02D0002657429E4161463A46334653
:1001700001B0F0BD03460B439B0703D009E008C95B
:10018000121F08C0042AFAD203E00B780370401C47
:10019000491C521EF9D27047D2B201E00270401CD5
:1001A000491EFBD270470022F6E710B513460A46F7
:1001B00004461946FFF7F0FF204610BDCAB2401EA4
:1001C0004178401C8A4202D00029F9D100207047B2
:1001D000421C0178401C0029FBD1801A704730B5C1
:1001E00004460020034600E05B1C934203D2E05C1F
:1001F000CD5C401BF8D030BD30B50546002003462D
:1002000000E05B1C934205D2EC5CC85C201A01D173
:10021000002CF6D130BD00000FB400B58DB00990B0
:100220000B9010A900200091C0430A9000200C9070
:1002300006480690064807906A4609A80F9900F0FC
:10024000C1FC0DB008BC04B018470000E50B00006D
:10025000050C0000FFB5002083B0009050680190AD
:1002600091691446002697680498884705460C99BA
:100270000698084305D009E0A169761C04988847D0
:100280000546216A284688470028F5D1681C03D016
:100290000198C00704D017E00020C04307B0F0BDAC
:1002A0002068011D2160006800900DE00198C007E2
:1002B00004D1009805700098401C0090A169761C3C
:1002C0007F1E049888470546002F1CDD681C1AD045
:1002D000069800280FD0E817C00E401941118A0077
:1002E00006994009511840012A1A096801209040D6
:1002F0000142DBD107E00C980028D7D1216A2846BB
:1003000088470028D2D0E169049888470C980028D3
:1003100007D1002E05DD0198C00702D10098002109
:100320000170A068B84204DD0C98002804D0002FAA
:1003300002D00120C043B1E73046AFE770B50646B2
:1003400011F006F9046805460A220021304600F043
:10035000C5FC2C6070BDF8B502464A40D40F42007F
:100360004B0052085B089A4202D2024608461146E8
:100370004A0023D0C30D4A00DDB2120EAD1A202D63
:1003800035DA49020126490AF6058A19002C00D0FF
:10039000524220214F1B1146B9402A411018C20D6C
:1003A0009A4221D0002C17D0012D08DCDA05801AE2
:1003B000D20F8019D207DBB200F0D0FCF8BDDA050D
:1003C000801A012340001B06C01880185A4280186A
:1003D000CA0F1043490007E04908C2071143DA0574
:1003E000801A80194008801800F0B0FCF8BD610048
:1003F0000122511A001BF7E70122D2075140AAE758
:100400000122D2075040A6E7024670B54A40D30FFA
:10041000DB0740002DD04A002AD0010E140E000246
:1004200012020919400A520A8418E501044654438D
:10043000000A120A2E045043A4194219200CC54385
:10044000AA18120C0125AD03521C521912047F394F
:10045000240400D0521C104301D44000491EC2B2F3
:100460000C06C0092018401C4008802A02D003E076
:10047000002070BD40084000002900DA0020184329
:1004800070BD70B502464A40D50F40004A00ED07E6
:1004900040085208002814D0002A12D0C40DD30DF1
:1004A00041020120C0055202490A520AE41A091801
:1004B00012187D34914201D3641C00E04900002CE5
:1004C00001DA002070BD0023914201D3891A034351
:1004D000400849000028F7D100290AD0914202D1F2
:1004E0000121C90705E0914201D2012101E001216A
:1004F000C943E005C018401900F028FC70BD000099
:10050000F0B507460846584087B0C00F0490480031
:100510000E46590040084908BC1A884105D23846A1
:1005200031461E4617460B46024658004008104307
:100530004CD0300D039040055900400D490D0590F9
:10054000401A0290402872DA18030121000B0905B5
:100550000843019004980092002805D00199524266
:100560000020884100920190029840210A1A0199C6
:10057000009800F0EDFA05460C466B4607CB00F0FC
:1005800008FBC0197141039A0E0D0023D71756407E
:100590001A467A40164344D0049A002A2DD0029A73
:1005A000012A039A15DC1205C01A9141012636056D
:1005B000001C7141D20F059ED20700930192029652
:1005C0002A46234600F010FC07B0F0BD38463146FD
:1005D000FAE71605224A0F46B218C01AB7410121A0
:1005E0000905001C4F4100187F4111461818794138
:1005F000E20F10436D19644113E0E2076D081543E3
:100600006408C2071443039A01261205C01A9141D7
:100610003605001C7141CE07400830434908C01818
:1006200051412A46234600F0D2FBCDE7FFE704986C
:1006300001224000C117121A00238B410498314651
:10064000C417381AA141EEE730B40124E40763402F
:1006500030BC55E730B40124E407614030BC4FE7BB
:100660000000E0FFF0B51FB488B00B990998002492
:1006700048400999C00F490049080991C0070B99E2
:100680000090490049080B9109990898A64608432B
:100690001CD00B990A98084318D0099801244000EF
:1006A000420D4800410D099824050003000B20432A
:1006B00009900B980003000B20430B9050181C4925
:1006C0004018002201901446104605E00020014623
:1006D0000DB0F0BD032801DA034600E003239C4679
:1006E000C11A0AAE0AE05F0008ADED5B4F00F75B90
:1006F0007D430027AA187C41491C5B1E6145F2DD41
:10070000410004AB5A522104120C0A43240C401C31
:100710000828DFDB01980290009970460191009053
:10072000059B049A0799069800F05EFBD0E700004D
:100730000DFCFFFFF0B50C465C4085B0E40FE4070C
:1007400003944C0000266408590094464908024668
:100750000296224321D062460A431ED06200570D02
:100760004A000E032303550D012402462C4924059B
:10077000781B1B0B360B4018234326436146009021
:100780001C46501AB44103D30098401C009002E06C
:10079000921800985B41002803DA0020014605B05A
:1007A000F0BD0020012109050746864611E0644698
:1007B0001D46141BB54106D36546521BB341744612
:1007C00007430C43A646CD07400849082843921822
:1007D0005B4105460D43EAD11046184313D06046ED
:1007E000194650407140084306D06046101AB34184
:1007F00006D20122002306E000220123DB0702E0EB
:100800000122D2435310009874460105381C6141FF
:10081000029C039D0019694100F0D9FABFE700006E
:10082000FD0300000122D207002800DB101A002976
:1008300000DB511A814201D8012070470020704727
:100840000122D207002800DB101A002900DB511A10
:10085000814201D201207047002070470122D20757
:10086000002800DB101A002900DB511A814201D355
:1008700001207047002070470122D207002800DBCA
:10088000101A002900DB511A814201D9012070475A
:10089000002070470122D207002800DB101A00292F
:1008A00000DB511A814201D10120704700207047BE
:1008B00010B5002904DB0C460121C9074042A141C3
:1008C000002B04DB1C460123DB075242A341801AA4
:1008D000994101D3012010BD002010BD10B50029A1
:1008E00004DB0C460121C9074042A141002B04DB77
:1008F0001C460123DB075242A341101A8B4101D34E
:10090000012010BD002010BDC217C10F504010B50E
:100910004018CA079623002100F020FA10BD10B538
:1009200000229623114600F019FA10BD0EB5C21729
:10093000C10F5040CA0740180021054B0293019295
:1009400000910A460B4600F04FFA03B000BD0000CC
:10095000330400000EB505490291002100910A46BA
:100960000B46019100F040FA03B000BD33040000D3
:100970003EB5CA17CB0F002450405140C01861410A
:10098000DA07054B0293019200942246234600F0B9
:100990002BFA03B030BD000033040000C20F410049
:1009A00040020123400ADB05D207090EC0187F2947
:1009B00001DA00207047962903DC9623591AC840B3
:1009C00001E096398840002AF4D040427047410047
:1009D00040020122400AD205090E80187F2901DA5F
:1009E00000207047962903DC9622511AC8407047B0
:1009F000963988407047000070B5CD0F4A00090352
:100A00000123090B1B0519430B4BED070024520D65
:100A10009A4201DA002070BD074B34339A4203DC5E
:100A20009A1A00F0A5F802E00449511888402C43B6
:100A3000F1D0404270BD0000FF030000CDFBFFFF7E
:100A400070B5CD0F4A0009030123090B1B0519439B
:100A50000D4BED070024520D9A4202DA00200146A8
:100A600070BD094B34339A4203DC9A1A00F080F8C7
:100A700003E0064BD21800F06BF82C43F0D00022B4
:100A800040428A41114670BDFF030000CDFBFFFFCD
:100A9000C20FD207400040080BD0C10D0723DB0175
:100AA000C91840020905400A1143C2084007114312
:100AB0007047002001467047CB0FDB07490010B597
:100AC000490802460A4307D00A0D07240903E40136
:100AD000090B121B002A01DC002010BDC900440FC5
:100AE0000C43C100E018D205801800F02FF910BDAA
:100AF000F0B51FB40646002082B00546402401919F
:100B000000901BE0019922460F46304600F030F875
:100B1000049A059B801A994110D310461946224623
:100B200000F016F8361A8F41019722460120002165
:100B3000009F00F00DF838184D4100902046641ECB
:100B40000028DFDC019B00982946324607B0F0BD43
:100B500010B5202A04DB0146203A9140002010BD48
:100B6000914020239C1A0346E3401943904010BD56
:100B700010B5202A04DB0846203AD040002110BDE1
:100B80000B46D340D0402024A21A91400843194676
:100B900010BD10B5202A06DBCB170846203A1041BD
:100BA000C1170B4306E00B461341D0402024A21A84
:100BB00091400843194610BD02681378511801602E
:100BC0001846704710B5D16004495161044911625B
:100BD00000211161114600F0ADF910BDB90B000004
:100BE000210F00004268002A08D001680B78491CD8
:100BF000002B03D0521E06C0184670470121C16069
:100C0000881E70474268002A0BD0C3680168002B19
:100C100007D183688B4204D0491E521C06C00020B5
:100C200070470020C04370470FB400B589B00A4632
:100C30000DA9009100230C99002ACB60234B069349
:100C4000234B079301D0042300E00023214A0292A2
:100C5000214A0892019302466B46002000F095FB62
:100C600009B008BC04B01847F0B585B007460020AD
:100C7000C04301901E46002015460C46009102918B
:100C800004903B466A46314604A8FFF7CDFF04991D
:100C900002466018002D05D0002901D0034600E06F
:100CA00023462B6000290ED0002A02DD00998142E4
:100CB00009D0001B019000943B466A4631460294DD
:100CC00004A8FFF7B1FF05B0F0BD0000E50B000080
:100CD000050C0000FFFFFF7F210F0000F7B5009C0F
:100CE0000F4600262578641C002D05D000F014F96D
:100CF0000068405DC007F5D12B2D02D02D2D18D0F6
:100D0000641E39462046029A00F06AFC002F04D087
:100D10003968A14201D10099396071050224002986
:100D20000BDA4042002803DD10F012FC0460A0073B
:100D3000FEBD012080020643E3E70028F8DA10F048
:100D400007FC04600048FEBDFFFFFF7F002904DAB6
:100D5000401C490001D140084000704770B4002495
:100D6000050C05D11024000402D1002921D0112442
:100D7000050E01D100020834050F01D10001241D28
:100D8000850F01D18000A41C002801DB4000641CF9
:100D9000002908D020252E1B0D46F540A14000D08B
:100DA00001212943084301061B1B000ADB1D02D554
:100DB000002070BC7047DB05181880180029F8DA8D
:100DC000401C4900F5D170BC40084000704710B588
:100DD000002B08DA0024401C614192185B411A4341
:100DE00001D14008400010BDF0B51FB482B00546E7
:100DF0000C0003D0084610F093FB02E010F090FBCB
:100E000020300246009021462846FFF7A1FE049BB1
:100E1000059A04460F4618431143084314D0184658
:100E200010431BD0009840210A1A18460599FFF775
:100E30009FFE05460E46009A05990498FFF788FE26
:100E4000084305D0012004E02046394607B0F0BD34
:100E50000020C11705430E432C43374300990E98D9
:100E60006305401A7905E40A00220C43FD0A0A30A2
:100E700002D500200146E9E70105101969410C9CE3
:100E80000D9D00196941FFF7A2FFDFE74A00090342
:100E90000123090B1B0519430A4B10B5520D9A4249
:100EA00002DA0020014610BD064B34339A4203DCBF
:100EB0009A1AFFF75DFE10BD034BD218FFF748FEEC
:100EC00010BD0000FF030000CDFBFFFF10B500299F
:100ED00004DB0124E40740428C412146002B04DB63
:100EE0001C460123DB075242A341994200D19042A4
:100EF00010BD0000064C0125064E05E0E36807CC56
:100F00002B430C3C98471034B442F7D3FFF7DCF87E
:100F1000C8480100E848010000487047EC1E010085
:100F200010B50446FFF7F8FF0068005DC007C00F6A
:100F300010BD0000F3B58DB000200A9001200B9089
:100F4000002608460C300C46099062690121099878
:100F50009047051E2ED0252D2DD0216A88470028C8
:100F600018D06269012109989047216A88470028B2
:100F7000F7D1411E62690998904700E0761CA1698B
:100F80000D988847216A88470028F7D1E1690D98B4
:100F90008847DAE7A1690D9888470746A84201D13A
:100FA000761CD2E7E1690D9888477F1C02D10A9828
:100FB000002877D049E1002762693D463946099803
:100FC00090472A280CD16269012109989047012590
:100FD00006E00A214F433F18303FEBD41020054371
:100FE0006269012109989047014630390A2903D2E4
:100FF0009B498F42DEDCECE7E90600D4994F6C2870
:101000000AD04C2810D0682824D06A282ED0742802
:101010000CD07A280AD00DE0626901210998904726
:101020006C2823D004211CE02020054362690121A3
:1010300009989047A760656065284FD026DC58283E
:1010400039D01ADC452849D012DC252834D0412873
:10105000B0D143E06269012109989047682802D025
:1010600008210D43E6E70120C002DEE70220DCE7AD
:10107000462833D047282CD130E05B2870D0612837
:101080002CD063286CD0642823D161E06F284FD026
:1010900009DC662822D0672820D0692826D06E284F
:1010A00017D12EE0CDE070284DD073286FD0752871
:1010B0004ED078280DD154E0A1690D988847054697
:1010C000252800D16CE7E1690D9888476D1C00D197
:1010D0006DE7BAE00A224CE00A2252E001202346E2
:1010E0006A46C0430D9900F050F9A3E0284640211C
:1010F00008436060A807234601D5002239E000229A
:101100003FE0E80700D020E72068011D216000686B
:10111000290501D5067018E7290701D5068014E7CF
:10112000A90703D5F117066041600EE706600CE7DA
:101130002846402108436060A807234601D50822BD
:1011400017E008221DE0484928460840606016E084
:101150002846402108436060A8072346BCD5B9E76C
:1011600015E02846402108436060A80707D52346BC
:1011700010220120C0430D99C046C0465AE02346C4
:1011800010220120C0430D99C046C04652E0002104
:101190000C910B460091632802D05B2807D043E0F6
:1011A000E80601D40120A060012000903CE06269C3
:1011B0000121099890475E2805D101200C90014635
:1011C0006269099890472169002906D10B4601AA56
:1011D0008F00491CD3510829FADB002835D021693A
:1011E00000290ED1C117C90E09184A11930001AA8E
:1011F0009A1849094901411A01201368884003439C
:10120000136062690121099890475D28E5D10C9827
:10121000002808D0002001AB81005A58401CD2435E
:101220005A500828F8DB01AB01202246C0430D9933
:10123000FFF710F800280ADA401C06D10B980028A6
:1012400003D00020C0430FB0F0BD0A98FBE7E907C8
:1012500002D10A99491C0A91361800200B9074E6B5
:10126000CCCCCC0CFFFFFF7FF1F7FFFFFFB5087878
:1012700089B01546FF2805D0491C2D2804D000222E
:10128000002407E000240BE00122F9E70A235C4375
:101290000419491C0878FF28F8D1002A00D06442BC
:1012A000002004902A7801462D2A01D02B2A0FD144
:1012B0006D1C2D2A02D00022049209E00122FBE7D6
:1012C00000260A2233466D1C00F0DDF93818714102
:1012D0002F78FF2FF4D10C9AA218069202460A43E7
:1012E00004D0FF23069A9133DA4205DA00210998E7
:1012F0000A4606C00DB0F0BD0024B74AB54D2646DB
:10130000079200F00DFA029006980391002801DA86
:10131000474200E0074639050020AF4A001C514112
:101320000191009012E0F80707D022462B46304684
:101330000799FFF797F90646079122462B46104674
:101340001946FFF78FF904460D467F10002FEAD1AA
:101350000698019B0028009A0399029806DAFFF785
:10136000E9F93246079BFFF7E5F905E0FFF77AF95F
:101370003246079BFFF776F9049A002A02D0012231
:10138000D2075140099A03C2B4E7FFB591B00020DB
:1013900009900025ED432E209E685C681F46019051
:1013A000B9696D1C129888470090396A88470028EF
:1013B000F6D10098401C0AD00D20C0018443002EB5
:1013C00012DD00982B2809D02D280DD103E0002034
:1013D000C04315B0F0BD012080020443B9696D1C03
:1013E00012988847761E009003A9600501D52D202C
:1013F00000E02B206A461073491C0CA80F91029044
:101400000AE0B9696D1C12988847009001204002DB
:1014100004431398761E0560002E02DD00983028E4
:10142000EFD001990098884245D18020044308E01C
:101430000998401E09900120400204431399681C3A
:101440000860B9696D1C761E129888470090302894
:10145000EED030E00199884205D1200603D48020E7
:101460000443761E1DE0009810F040F9002825D0B6
:10147000012149020C43009807AA0F990332303822
:10148000761E914208D208700F98401C0F902006DB
:1014900007D50998401E03E0200602D40998401C95
:1014A0000990A00502D51399681C0860B9696D1CE4
:1014B000129888470090002ECCDC59E0002E57DDB2
:1014C0000098652801D0452852D1A00550D50320A9
:1014D00000028443B9696D1C761E129888470090FB
:1014E000002E0CDD2B2804D02D2808D1FF20013040
:1014F0000443B9696D1C12988847761E0090E00578
:1015000001D52D2100E02B21029801700298401C8A
:101510000290019025E00120400204430EA90298A8
:101520000131761E88420ED20098029930380006AA
:10153000000E087003D10299019881420AD90298DD
:10154000401C029006E0E00501D5244801E0234854
:1015500040420990B9696D1C129888470090139811
:101560000560002E04DD009810F0C0F80028D2D1EC
:10157000F969129888470F99FF200870029903AA09
:10158000087000200A900B900CA90AA8099BFFF78D
:101590006DFEA00502D40120C0431AE724200442B6
:1015A00009D0E00713D138680B9A0A99031D3B60F4
:1015B000006806C00BE00B990A98FFF77DFA014618
:1015C000E00704D13868021D3A60006801602846CF
:1015D000FFE60000000014400000F03FF1D8FFFFDC
:1015E000F7B582B0029C00272078641C154601974D
:1015F000302802D0002D15D015E020780127641C7A
:10160000782804D0582802D0002D09D00BE0002DF6
:1016100001D0102D07D1002710252078641C02E08E
:10162000082500E00A250026009610E00099012711
:1016300069430818020C294680B2714300908E1845
:101640003804864201D3012001902078641C294689
:1016500000F056F80028E9DA0398002805D0002F9A
:1016600001D0641E00E0029C04600198002806D0AE
:101670000FF06EFF02210160C81E05B0F0BD009999
:1016800030040843F9E7F0B51FB486B0002000909D
:10169000019002900698069980B204900798090C70
:1016A00002040014114307900027089D0998069131
:1016B0003E463C4603900398A9B20204000C0390F6
:1016C00004982D0C1543484300212246FFF740FAA9
:1016D000C719714110340E46402CECDB3846029A93
:1016E000FFF736FA009A019B801800905941029842
:1016F0000191103002904028CCDB00980BB0F0BD77
:101700003A2800D23038202302469A43412A01D396
:1017100010463738884201D30020C043704700008C
:101720000EB5054A02920022009213460192FFF77D
:101730005BFB03B000BD00003304000070B58C18E3
:101740000578401C6B075B0F01D10378401C2A1100
:1017500006D10278401C03E006780E70401C491C3C
:101760005B1EF9D12B0705D40023521E0DD40B703C
:10177000491CFAE70378401CCB1A921C03E01D7841
:101780000D70491C5B1C521EF9D5A142D8D3002014
:1017900070BD000010B52148016A8A0715D44A07B8
:1017A00015D4C90732D01E498A89002A15D0531E84
:1017B0008B8182688C6904C48C610A691B040DD01A
:1017C000002A22D10121016010BD022100E0042184
:1017D000C16113488021416110BD0A69012A09D104
:1017E000026801239A430260C361FF206830993088
:1017F0000C4A106001204861CA69002A05D0886936
:1018000009898B00C01A904710BD10BDFF226832B5
:10181000054806A109A30DF0FDFAC04608D0014015
:10182000A095010280E200E0402E01004144435FA8
:1018300049525148616E646C65720000556E65785E
:101840007065637465642041444320696E746572F9
:10185000727570740D0A000070B582B00023019398
:10186000444801688A6A4C6813252540132D02D12B
:10187000CB689B07DB0F4361930772D453070AD4ED
:10188000D30711D1130724D5048F838E1C1B102C72
:101890000EDD102310E0042088620220032142A202
:1018A0000EF014FB02B070BD0120886202B070BD62
:1018B000048F1B1B1C0610D0DBB20024058FC66AE8
:1018C00075192D5D0D74641CA342F7D1048FE318C4
:1018D0000387D20607D400212FE04B6A0824A343D4
:1018E0004B62D206F7D5CB68C28E448F141B5B04C3
:1018F000DB0EA34201D3438FD31ADAB2002A16D0EB
:10190000097D438F046BE1540199012A10D0012312
:101910001C46890145582D7D41184E8F9B19096B36
:10192000CD54641CE3B201999A42F2D800E0002140
:101930008B01C3185C8FA2185A878A0181184B8FBC
:10194000CC8EA3420BD301230B618058002242624C
:10195000CA6B002A03D03A31098801A8904702B027
:1019600070BD02208862044804A1084A08A30DF053
:1019700051FAC04674900102592E01004145535F4F
:1019800049525148616E646C65720000CE020000DD
:1019900041455320696E707574206F766572666C70
:1019A0006F770D0A00000000414553206F75747079
:1019B000757420756E646572666C6F770D0A000031
:1019C000F0B581B001243F2900D993E00346806837
:1019D000456B2D688E0001A7BE59B7461B1B000042
:1019E000371B0000131B0000131B0000F51A00003A
:1019F000F51A0000F51A0000F51A0000F51A0000AB
:101A0000F51A0000F51A0000F51A0000F51A00009A
:101A1000F51A0000491B0000651B0000F51A0000C4
:101A2000F51A0000F51A0000F51A0000F51A00007A
:101A3000F51A0000F51A0000F51A0000F51A00006A
:101A4000F51A0000F51A0000F51A0000F51A00005A
:101A5000F51A0000F51A0000F51A0000F51A00004A
:101A6000F51A0000F51A0000F51A0000F51A00003A
:101A7000F51A0000F51A0000F51A0000F51A00002A
:101A8000F51A0000F51A0000F51A0000F51A00001A
:101A9000F51A0000F51A0000F51A0000F51A00000A
:101AA000F51A0000F51A0000F51A0000F51A0000FA
:101AB000F51A0000DD1A0000DD1A0000DD1A000032
:101AC000DD1A0000DD1A0000DD1A0000DD1A00003A
:101AD000DD1A0000DD1A0000DD1A0000434800692D
:101AE0000024022809D001280DD0002802D103CA01
:101AF00004F0A8FF204601B0F0BD03CA04F094FF33
:101B0000204601B0F0BD03CA04F0B2FF204601B088
:101B1000F0BD022931D0022430E0344D00242C6184
:101B20006C619849354A01F061FE6869401C686142
:101B3000204601B0F0BD01F093FE284602F000F906
:101B40000024204601B0F0BD284909690C234B430D
:101B50002749CA58C918496801F048FE00242046A0
:101B600001B0F0BD0024204604F03AFF0128C1D1A5
:101B70001E483030204900241CE001241B490F6915
:101B80000C26314679431A4A51188968214208D0F7
:101B900000247D1C15490D614C61042D10D315499D
:101BA00006E012494869401C4861032812D32949BC
:101BB00000241846224602F073F8204601B0F0BD1A
:101BC0006E430B498A598919496801F00FFE204676
:101BD00001B0F0BD0E20009000240A2228462146C4
:101BE00002F04EF8204601B0F0BDC046AC990102AB
:101BF000F01E0100F0250100D0250100BE390100D2
:101C0000B0B504290FD804468068C04679440979E4
:101C100049008F44020A0E1C1700104910A201F05F
:101C2000E5FD0020B0BD0120B0BD01F019FE00208F
:101C3000B0BD00250321284604F0E2FE06492046F7
:101C40002A4602E003490022204602F029F800203B
:101C5000B0BDC046E02501006026010088130000E9
:101C6000415445300D0A0000B0B582B001240A2964
:101C700010D883687944097949008F440E290505F5
:101C80000B0B0B0B0B0B1A00194909680024224699
:101C900002F006F8204602B0B0BD50681449086052
:101CA000144915A2184601F0A1FD0024204602B0F7
:101CB000B0BD0024019403CA09A201AB02F00EF9E1
:101CC0000228E7D1019804F0EFFE204602B0B0BD33
:101CD000184601F0C5FD0024204602B0B0BDC04644
:101CE0002B4353513A2025642C252A0D0A0000006D
:101CF000C89A01028813000041542B4353510D0A26
:101D000000000000B0B582B00546002404F0C6FE15
:101D100001280DD108498C60E86B426853684B601C
:101D2000009401926A4601F0BBFF204602B0B0BDAC
:101D3000E443204602B0B0BDC8930102B0B50546E9
:101D4000881E02280AD3A868012913D0002915D1BA
:101D50000C490DA201F04AFD0020B0BD0220014651
:101D600004F04EFE064900242846224601F098FF62
:101D70002046B0BD01F074FD0020B0BD0120B0BD13
:101D8000B02501008813000041542B4346554E3DB9
:101D9000300D0A00B0B5E0B00324E1016D462846DD
:101DA0000FF0A6FB204621462A460EF08FF80020B1
:101DB00060B0B0BDF0B597B00820149064201390C7
:101DC0002548109002200E904B20C0011690234D04
:101DD00028461430129001270F97B8021190032063
:101DE0000EA906F03FF90026F443002802D0204651
:101DF00017B0F0BD0C35284601F0B0FF0028F6D131
:101E000080200C9016490B910A90164809901648AC
:101E100008901648079016480690392005901548F6
:101E20000490154803900D95144D03A9284601F020
:101E300047FD0028DBD1009501970F4C104911A2F6
:101E4000124B204601F0E0FE1149204601F010FF40
:101E50003446204617B0F0BD48C001022497010265
:101E600048C40102C8C40102452F0000952F00009C
:101E7000152F000070270100DC99010258C90102EA
:101E80005025010041495237383045007026010085
:101E9000951D000010B50348002404700EF0A2FF49
:101EA000204610BDE09E010280B501F053F90020EC
:101EB00080BD0000F0B58DB00E4600270C970B9743
:101EC0000A970997089707970697059702908068E1
:101ED0000490406B0068019004F07CFD04465BA117
:101EE00005220392FEF788F95A4D00281ED05AA108
:101EF00005222046FEF780F9002817D058A10522B8
:101F00002046FEF779F900280FD059A10522204676
:101F1000FEF772F9002809D057A105222046FEF7E6
:101F20006BF9002807D156A500E04FA505A8202190
:101F30002A4602F0A5F801203F2E00D936E0C0461F
:101F40007E4436797600B7443340474A57313131C1
:101F5000313131313131653031313131313131313E
:101F60003131313131313131313131313131313161
:101F700031313131313131313131313131311F1F75
:101F80001F1F1F1F1F1F1F1FBE48416A04290CD19E
:101F9000039A426287620C2050433D490A58081850
:101FA000416805AB049801F021FC38460DB0F0BD46
:101FB000B44C00206062A062CD49364A049801F01A
:101FC00015FCA06A401CA062EFE7049801F048FCF1
:101FD000019801F0B5FEE8E7AA48406A05E0A94982
:101FE000486A01220243032A1CD1A649421C4A62C4
:101FF0008F62062ACFD30BE0A2494A6A012013461A
:102000000343052BD2D1501C48628F62062803D3AC
:102010001E490DE09B48406A0C2141431C48425830
:102020004018BDE7886A401C8862032805D316491A
:102030000022029801F034FEB7E70E200090002144
:102040000A220198029B01F01BFEAEE734363030C5
:1020500030000000E6390100343630303200000034
:102060003436303031000000554E494E45540000A2
:102070003436303036000000343630303300000063
:1020800043544E455400000050250100A025010096
:10209000201F01006639010070B5022956D30F29AF
:1020A00007D1784C217A012905D1002222728F496B
:1020B0004AE0012070BD866801F076FE002004F041
:1020C00097FC012803D10020032104F099FC00258E
:1020D000284604F085FC012804D130346A490022E6
:1020E000204631E0304600F0EBFD00282ED030468F
:1020F000FFF708FE002829D004F08CFC012807D146
:102100005F498D60F06B4268E26252684A601AE093
:10211000022004F065FC012808D159498D61F06B5B
:102120004268E26252684A6110310CE0022004F019
:102130005FFC01280AD152498D62F06B4268E2626D
:1021400052684A6220312A4601F0AAFD002070BD83
:1021500010B582B003460120272931D87944097986
:1021600049008F442C132D2D162D2D2D2D2D2D2D69
:102170002D2D2D2C2D2D2D2D2D2D2D2D2D2D1C2DA1
:102180002D2D2D2D2D2D2D2D2D2D2D2904F0C2FF82
:1021900015E0DF490022184601F082FD0FE0002023
:1021A000019003CA08A201AB01F098FE012806D1F4
:1021B000019805F0CBF802E00248012101720020ED
:1021C00002B010BDAC9901022B51495552433A203F
:1021D00022636C6F736564222C25640D0A00000075
:1021E000B0B502294AD30F2914D18568002004F024
:1021F000FFFB012803D10020032104F001FC00248F
:10220000204604F0EDFB012806D1D94830301E49A4
:10221000002231E00120B0BD2846FFF773FD002801
:102220002CD004F0F7FB012808D115498C60E86B2D
:102230004268CF4BDA6252684A601CE0022004F028
:10224000CFFB012809D10E498C61E86B4268C84B6D
:10225000DA6252684A6110310DE0022004F0C8FBD6
:1022600001280BD106498C62E86B4268C04BDA62E8
:1022700052684A622031224601F012FD0020B0BDB2
:1022800040900102AC990102D025010080B50229DD
:1022900005D3042905D19E49002201F001FD00204B
:1022A00080BD012080BDC046B0B50546881E02280D
:1022B0000AD3A868012913D0002915D10C490DA211
:1022C00001F094FA0020B0BD0220032104F098FB35
:1022D000064900242846224601F0E2FC2046B0BD13
:1022E00001F0BEFA0020B0BD0120B0BDF025010014
:1022F0008813000041542B4346554E3D310D0A00D2
:1023000010B50F290BD001291DD000291DD1FFF7D1
:10231000C1FD0020022104F073FB002010BD044623
:10232000002004F05DFB012803D10020022104F00D
:1023300067FB002004F05CFB012804D10449002263
:10234000204601F0ADFC002010BD012010BDC046AC
:10235000E0250100F0B581B00124322928D80546D6
:102360008768786B0668C0467944097949008F44CC
:102370002F3F1919191F1F1F1F1F1F1F1F1F221F4C
:102380001F1F1F1F1F1F1F1F1F1F1F1F1F1F1F1F5D
:102390001F1F1F1F1F1F1F1F1F1F1F1F1F1F1F1F4D
:1023A0001F1F26001E4900242846224601F078FC03
:1023B000204601B0F0BD1B48017800291FD0184904
:1023C00000242846224601F06BFC204601B0F0BDF7
:1023D0000024FC623969384688470028FAD0114841
:1023E0000470FC62FFF756FD0E20009001220EE003
:1023F000304601F0A5FC0024204601B0F0BD0121CB
:102400000170FFF751FD0E20009000240522304698
:1024100021462B4601F034FC204601B0F0BDC046F9
:1024200070250100CC9A010210B586B00346012048
:102430003B2900D956E0C0467944097949008F44C8
:10244000505051513351515151515151515151519C
:10245000515151515151515151515151515151516C
:10246000515151515151515151515151515151515C
:102470005151515151391D1D1D1D1D1D002005902B
:1024800003CA02AA009218A205AB01F027FD022898
:1024900027D1039A029817A1FDF7AEFE002820D19C
:1024A000059804F053FF1CE0B5490022184601F0DE
:1024B000F7FB16E0002002900590049003CA05AADD
:1024C000019204AA00920DA202AB01F007FD0328BD
:1024D00007D1049A0599029805F004F8029804F0CF
:1024E000A3FF002006B010BD25642C2025700D0A26
:1024F00000000000434C4F53454400002B5245431D
:10250000454956452C25642C25643A0D0A2565005D
:10251000C0250100012901D8002070470120704723
:10252000B0B50546881E03280BD2104604F07AFA8F
:102530000F48C16A00242846224601F0B1FB20461C
:10254000B0BDAC6801290BD000290ED104F044FACB
:102550000346084908A2204601F048F90020B0BD12
:10256000204601F07DF90020B0BD0120B0BDC0467D
:10257000AC9901028813000025730D0A00000000C9
:1025800070B582B001240F293DD803468568686B79
:102590000668C0467944097949008F4407141E34FF
:1025A0003434342F373434343434434E66480024C2
:1025B00004708461C461012101716649664A28463C
:1025C00001F014F91FE0284601F04AF9304601F005
:1025D000B7FB0024204602B070BD5B4800240471A4
:1025E0008269042111430278002A2ED0052958D18E
:1025F000016A491C016259D2624961E0524B187864
:102600000024002831D0204602B070BD4E4B18780F
:10261000012816D103CA183351A201F05FFC002033
:1026200002B070BD48480024846101210171007826
:102630004849002812D1484A11E0434E3079002819
:102640001BD00024204602B070BD052932D10024E1
:10265000012101708461C46101713E493F4A2846ED
:1026600001F0C4F8204602B070BD03CA183340A27E
:1026700001F034FC204602B070BD002004F0B8F92F
:10268000012803D10020032104F0BAF900242046D8
:1026900004F0A6F9012816D130362D490024304621
:1026A0004BE000210162C169491CC1610E2000900C
:1026B00000241CE0C169491CC161652915D330495A
:1026C0000024184639E02846FFF71CFB00289AD062
:1026D00004F0A0F9012812D11C4900248C60E86B99
:1026E0004268F26252684A6027E00E20009002229F
:1026F0003046214601F0C4FA204602B070BD0220E7
:1027000004F06EF9012809D1104900248C61E86BAE
:102710004268F26252684A6110310EE0022004F011
:1027200067F9012800D06EE7084900248C62E86B45
:102730004268F26252684A622031224601F0B0FAE1
:10274000204602B070BDC046AC9901024090010223
:10275000D025010088130000823901008D39010065
:102760002B43475245473A20252A2C256400000078
:102770002B435245473A20252A2C256400000000AF
:10278000C025010080250100B0B584B001243B299B
:1027900000D937E0134605468068C0467944097978
:1027A00049008F444B5532322F2F2F2F2F2F2F2F91
:1027B0002F2F2F2F2F2F2F2F2F2F2F2F2F2F2F2F29
:1027C0002F2F2F2F2F2F2F2F2F2F2F2F2F2F2F2F19
:1027D0002F2F2F2F2F2F2F2F2F2F1D1D1D1D1D1D75
:1027E0000024039403CB01AA00921C4A03AB01F01E
:1027F00075FB022806D1029A019819A1FDF7FCFC8D
:1028000000280FD0204604B0B0BD1848006804F07E
:102810009DFD174900242846224601F041FA204632
:1028200004B0B0BD1148006804F090FD10490022CA
:10283000284601F035FA204604B0B0BD0B490B60C4
:102840001E210CA200F0D2FF0024204604B0B0BD2F
:1028500001F006F80024204604B0B0BDE63A0100BD
:10286000434C4F5345204F4B00000000D09A0102CB
:102870009025010041542B434950434C4F53453D53
:1028800025640D0A00000000F0B589B0044601205F
:102890003B2900D9AAE01646A7687A6B1568C0469E
:1028A0007944097949008F44536AA071A1A1A1A17B
:1028B000A1A1A1A1A1A18AA1A1A1A1A1A1A1A1A11F
:1028C000A1A1A1A1A1A1A1A1A1A1A1A1A1A1A1A1F8
:1028D000A1A1A1A1A1A1A1A1A1A1A1A1A1A11D1DF0
:1028E0001D1D1D1D0027089703CE06AA0092414A10
:1028F00008AB01F0F3FA022877D13F480568089841
:10290000854272D1079A069E3CA130460592FDF79A
:1029100073FC002847D03DA13046059AFDF76CFCBA
:10292000002840D03CA13046059AFDF765FC002800
:10293000314E5AD1284604F023FD7068401C706067
:1029400003283CD303207060306804F0A1FC36E01B
:1029500029480660304604F0EFFC059026480068E0
:1029600004F0BEFC04902448006804F0C5FC0499FF
:10297000019102900598012827D02EA026E0384624
:1029800000F06EFF284601F0DBF92EE01A4D2868B2
:1029900004F0F6FC6868401C686003280FD300222E
:1029A0006A6022490DE0144E7760284604F0FEFC70
:1029B000306804F03DFE002801D01B4900E00C49BE
:1029C0000022204601F06CF90FE019A000901A498E
:1029D0001AA23846334600F009FF0E20009000216D
:1029E000B4222846234601F04BF9002009B0F0BD7F
:1029F00090250100E63A01009C970102414C5245A6
:102A000041445920434F4E4E45435400434F4E4E90
:102A1000454354204F4B0000434F4E4E45435420F6
:102A20004641494C000000003026010050250100BD
:102A300054435000554450008813000041542B4328
:102A4000495053544152543D25642C222573222C65
:102A5000222573222C25750D0A000000B0B582B026
:102A600014468A1E022A12D38568012917D000292C
:102A70001CD1204604F026FC00901E210EA2284600
:102A8000234600F0B3FE0024204602B0B0BD094941
:102A90000024224601F004F9204602B0B0BD2846C9
:102AA00000F0DEFE0024204602B0B0BD0124204626
:102AB00002B0B0BD4026010041545E484541525429
:102AC000434F4E4649473D312C25642C25750D0A50
:102AD00000000000F0B583B014468A1E022A1CD301
:102AE0008568012921D0002926D1164F3C60204657
:102AF00004F0DAFBFDF76CFB0646386804F0D4FB03
:102B00007108009101901E210FA22846234600F073
:102B10006DFE0024204603B0F0BD09490024224682
:102B200001F0BEF8204603B0F0BD284600F098FE44
:102B30000024204603B0F0BD0124204603B0F0BDC0
:102B400090250100D49A010241545E4845415254F7
:102B5000424541544845583D25642C25752C257324
:102B60000D0A0000F0B585B0044601203B2900D9CC
:102B700085E0A5687944097949008F443F547F5B1B
:102B80008080808080808080808080806080808065
:102B90008080808080808080808080808080808035
:102BA0008080808080808080808080808080808025
:102BB00080801D1D1D1D1D1D0020049003CA02AA3A
:102BC0000092304A04AB01F089F9022856D12E4810
:102BD00085680498854251D1039E029F2BA13846F7
:102BE0003246FDF709FB00283AD02AA13846324682
:102BF000FDF702FB002841D128461DE0224CA260CF
:102C0000104604F085FB002838D001F0D0FAE060CF
:102C1000002833D0A36840680090234923A22846A7
:102C200000F0E4FD2AE018480021C160284600F0C9
:102C300017FE23E01448806804F088FB19E000F0D8
:102C40007FFE012804D11048C16803C900F080FF4D
:102C50000D48C0680CC81349284600F007FE0DE077
:102C6000284604F055FB0028074907D0C96801F041
:102C700074FA0B490022204601F012F8002005B03A
:102C8000F0BDC046E63A01009C97010253454E4410
:102C9000204F4B0053454E44204641494C00000014
:102CA00090250100204E00008813000041542B4362
:102CB000495053454E443D25642C25750D0A0000AE
:102CC000F0B583B0074601F06FF80026304604F0F7
:102CD00029FB032835460BD10421284604F098FC33
:102CE000F86B51492A4600F0DBFF304603B0F0BDD7
:102CF00002970024204604F015FB0428254609D13C
:102D00000298C06B49492A4600F0CAFF2646304661
:102D100003B0F0BD0027384604F004FB05283D460B
:102D200009D10298C06B40492A4600F0B9FF3E46DF
:102D3000304603B0F0BD01970125284604F0F2FAB1
:102D40000328029FC8D00125284604F0EBFA042886
:102D5000D6D00125284604F0E5FA0528019FE0D0E9
:102D60000225284604F0DEFA0328029FB4D002258B
:102D7000284604F0D7FA0428C2D00225284604F0D9
:102D8000D1FA0528019FCCD0254C2068401C032196
:102D9000FDF7B6F90D46084604F0C4FA0628029F6E
:102DA00008D1284604F0B4FA002803D001F0FFF956
:102DB00000282AD1681C0321FDF7A2F90D46084618
:102DC00004F0B0FA062808D1284604F0A1FA002839
:102DD00003D001F0ECF9002817D1681C0321FDF79E
:102DE0008FF90D46084604F09DFA0021CE430628CF
:102DF00000D07AE7284604F08BFA002800D174E767
:102E000001F0D5F9002800D16FE72560F86B05497E
:102E10002A4600F045FF0026304603B0F0BDC0460C
:102E2000D89A010250260100102601002026010038
:102E300080B58AB00620042108F05EFE4B20C00158
:102E400009900820079064200690B448143005903B
:102E50000648039002200190012002908002049015
:102E6000032001A905F0FEF80AB080BD48C00102A8
:102E7000B0B582B001220F293ED803468068446B6A
:102E80002468C0467944097949008F44071F2527E3
:102E9000343535353535353535350A152749002270
:102EA00004E02649CA68092A20D8521CCA6016497B
:102EB000164A00F09BFC1EE0002003F091FD012863
:102EC00019D11E4830300E49002212E000F0C8FC33
:102ED000204600F035FF0EE00D4908E00E2000907E
:102EE00000210122204600F0CBFE04E0054900222B
:102EF000184600F0D5FE0022104602B0B0BDC04614
:102F0000D0250100B0250100881300009939010087
:102F10006025010080B5032005F08CF880BD00001D
:102F20000648416B0020002905D0054A914203D094
:102F300049680029FAD1704701207047AC99010215
:102F4000A0250100B0B514460D460846114600F014
:102F5000ACFF012816D1285D002813D1002C0BD01E
:102F60006019401E00780A2806D10320084A01464D
:102F70002B460CF0ABFF05E00320054A01462B462B
:102F80000CF0A4FF03202946224605F03FF9B0BD0E
:102F90002F390100F0B585B0054604A8002404705F
:102FA000E743002D12D0EA68002A0FD0686A002893
:102FB0000CD0A86A002809D0401EE96A814200D3DB
:102FC0008EE004A928469047002803D03C462046BE
:102FD00005B0F0BD514EE86A411CE962696A049A85
:102FE0000A54E86A696A002202920A54E86A0928C7
:102FF00006D1696A09224848FDF7F1F800283ED059
:103000003078411E022908D800F0CEFEB168401A7F
:103010004349884264D8414E30780A2820D001289C
:1030200023D16E6A3A213046FDF7C8F8002847D010
:10303000019002980390E96A03AB304639A200F090
:103040004DFF02284CD10398002849D00A21334A69
:10305000117001990818696A401AC01C50602FE06D
:103060007068E96A81422BD13AE004A800780A2806
:103070000FD00D2814D101202863E86A1AE001203E
:10308000307000F091FEB0603078411E0229BBD94B
:10309000C3E7296B012904D102202863E86A03E011
:1030A000296BE86A022905D1022817D10298E86243
:1030B000286305E0012803D1686A00783E280FD014
:1030C000A86AE96A401E81420AD2EA6804A9284631
:1030D00090470028114E00D17DE777E702982863DA
:1030E000E96A686A00F0E1FE01280FD16B6AE86ABC
:1030F000002806D0C018401E00780A2801D10DA271
:1031000000E010A2032001460CF0E0FE034804702A
:10311000204605B0F0BDC04672320100249701027E
:10312000DC0500002B524543454956452C252A2CE9
:1031300025643A005B415420526563765D20257317
:10314000000000005B415420526563765D202573CA
:103150000D0A000010B5064C2078002108F088FC0C
:10316000044806F02DFD2078012108F081FC10BDF7
:10317000AE96010260E31600B0B50F2001F0DEFB51
:10318000194D6870287033282AD120243721204611
:1031900001F020FC2120032101F01CFC2220402111
:1031A00001F018FC2320082101F014FC3020AA2192
:1031B00001F010FCA24802210187322001F00AFC34
:1031C0003320012101F006FC5F21204601F002FCC2
:1031D0000F2001F0B3FB28700A2006F0F1FCB0BD0F
:1031E00097480021C187B0BD04960102F0B581B0B7
:1031F000364C212100916172354909886170354F43
:10320000FA886271BD6ABD61334B1B782370090A6D
:10321000A170110AA171B978814207D10AF052FE5A
:103220006421FCF757FF3981B978BD6A2B484843C0
:103230002B4940180A21FCF74DFF4519FD620AF0A1
:10324000D7FD40190BF030FA06460D462548007BA5
:103250000BF0B6F8244909882222A15482B2D20B7D
:10326000801802B2D0175210B2186841130E009D98
:103270006355130C202563553B6DA3761D0AE57637
:103280001D0C25771B0E637723462233090A5970DC
:10329000A277BA64F864BA65F865100AE0770AF0B4
:1032A00011FEF861FB6A2821012220460EF0A6F8E3
:1032B0000AF008FE786108F0E3FF0028FBD1042043
:1032C00008F096FB002001B0F0BDC04606D4010214
:1032D000A89801023099010284980102800A1B001B
:1032E00040C20C00B69001028E98010270477047F0
:1032F000F0B587B04F480068FDF718FB04460D464F
:103300004D48406AFDF7C4FB02460B46204629465D
:10331000FDF710FA02460B46002448492046FDF707
:1033200093F90490039106204549085EFDF7FEFAE3
:10333000019000910120069040020290414F05E06B
:103340004F4908517F1C241D642C70D03878052803
:103350003D48F5D105973D4801593D4E31613D4805
:103360000359B3603C480059B0613C4A125932627B
:1033700000275D1A35637369F1689941069B00DB8C
:103380003B46002B01D0029BC918314E7163F36993
:10339000716A101A9941069A00DB3A46002A01D058
:1033A000029A8918FDF7E4FA02460B46049803993D
:1033B000FDF758F9FDF744FB254A9062D162401BA6
:1033C000C10F4018401010601546FDF7AFFA244AAF
:1033D000244BFDF747F9A863E963234A234BFDF724
:1033E00041F93A46224BFDF73DF93A46214BFDF7AC
:1033F00087F805460E4616480564416428463A4655
:103400001D4BFDF755FA0028059F9BD10022284649
:1034100031461A4BFDF762FA002893D1284631460F
:10342000019A009BFDF76CF8FDF7E6FA88E707B014
:10343000F0BDC046F09601024C2001000000F03FB4
:1034400032A9010200980102FFFF0100949F0102CE
:1034500018960102F89F0102F4DF010258E0010210
:10346000699006699006903F52257997532ED33F75
:103470000000594000003E4000408FC0006AF84004
:1034800020D20102B0B582B0194C2068056801A9AC
:103490000020087007E090470198401C01A90870BF
:1034A000C0B2082822D2012211048140294209D049
:1034B0002268516080002018826A002AECD001A89E
:1034C0000121E8E7130283402B4201D0022104E0EE
:1034D00082402A42E0D003211346226853608000D4
:1034E00020188268002AD7D001A8D4E702B0B0BD66
:1034F000D4920102FEE7000010B509480168CA69CC
:1035000020231343CB610269032A08D101229305CA
:103510000C689C430C605102C26E0A43C26610BD27
:103520004893010281B010B581B00393002807D001
:10353000C16A002904D003AB0093C46A0021A047EC
:1035400001B010BC01BC01B00047000080B50246CC
:1035500008480068002807D091B2120C03889A42EC
:1035600003D040690028F9D180BD002200F0F4FAB0
:1035700080BDC04654C90102F0B581B05C4C2068E2
:10358000856BE80707D0E168002904D00020884750
:10359000206801218163A80707D52169002904D08B
:1035A00001208847206802218163680707D5616987
:1035B000002904D00220884720680421816328075D
:1035C00007D5A169002904D0032088472068082175
:1035D0008163E80607D5E169002904D00420884703
:1035E000206810218163A80607D5216A002904D02C
:1035F00005208847206820218163680607D5616A15
:10360000002904D0062088472068402181632806CD
:1036100007D5A16A002904D00720884720688021A7
:1036200081630126E80507D5E16A002904D0370245
:103630000820884720688763A80507D5216B0029E3
:1036400004D077020920884720688763680507D57A
:10365000616B002904D0B7020A208847206887637D
:10366000280507D5A16B002904D0F7020B20884755
:1036700020688763E80407D5E16B002904D037038D
:103680000C20884720688763A80407D5216C00298F
:1036900004D077030D20884720688763680407D526
:1036A000616C002904D0B7030E2088472068876327
:1036B000280407D5A16C002904D0F7030F20884700
:1036C00020688763E80307D5E16C002904D037043C
:1036D0001020884720688763A80307D5216D00293B
:1036E00004D07504112088472068856301B0F0BDBF
:1036F000D893010202480068411E88417047C046C5
:103700009C980102F0B58DB0002862D00446406854
:1037100000285ED0A06840285BD8E56A002D58D00C
:103720000746204640300026039003E0019E4AE011
:10373000039848E0402101220691FCF72DFDAE429E
:1037400002963ED200203146019009900398069BD4
:103750003E46002EEAD0606A0491405C07900998CA
:10376000401C05900021042708916518EA5C012A95
:1037700017D10A966268D3191B1F1B68099E9E5DAC
:103780000798864208D1059D5B5D002B0A9E22D0DA
:103790000898401C089003E0403500222A70A66873
:1037A000069B0837491CB142DFD308980028BFD0D8
:1037B0000499491CE06A8142059809900398C8D38E
:1037C00001E003983E463746E56A029E761CAE420B
:1037D000B0D30DB0F0BD616A0B91E16A0C91D15983
:1037E0000BAA204600F09CF80DB0F0BD81B0B0B53A
:1037F00083B00D460446079307AB02938069E169E5
:103800000DF076FE206265480078002803D1216A19
:10381000A06900F09FF96369A169226A2046984770
:103820000146A06B002905D069460C600021224B9F
:103830000A460CE000F084FA7D2081002846FCF75F
:1038400049FC0246A06B69460C6000211B4B00F04E
:10385000D3FA002003B0B0BC02BC01B00847C04698
:1038600080B5806B00F06CFA002080BD70B582B02E
:103870000D460446466911461A46B0470146A06BFC
:10388000002907D069460C6000210B4B0A4600F066
:10389000B3FA0EE000F054FA7D2081002846FCF7D0
:1038A00019FC0246A06B69460C600021034B00F036
:1038B000A3FA002002B070BDA5390000BB3900009A
:1038C00070B50D460446802100F0C0FA2868E06318
:1038D00068686060A868A060E868E06028692061A6
:1038E00068696061A869A061E86900262662E061F4
:1038F000286A6062686A2663E662A062A86A6063FA
:103900002046383000F02AFA002802D0F64330462C
:1039100070BD2148016821600460304670BDC0461A
:1039200070B514460D460646881E032802D8B06BB3
:1039300000F006FAF06B2946224600F00DF970BD42
:1039400016480178012048407047C04670B51248BB
:103950000468002C1FD0114E11A52169204688470C
:10396000002815D1307800280DD1E16A606A00F096
:103970009CFA0146606A012903D0E16A00F0E8F888
:10398000284600F0E3F82046FFF7BCFE0020E06286
:103990002468002CE1D170BD50C9010248C9010260
:1039A0000D0A000010B50446806B00F0C9F9E06B09
:1039B0000521002200F0D0F810BD10B50446806B40
:1039C00000F0BEF9E06B0421002200F0C5F810BD44
:1039D000F0B581B000910646C7680468A01C39465E
:1039E000FCF778FB00257068814201D1ED430BE0C4
:1039F000601C3946FCF76EFB316032695143B06898
:103A000008180099FCF7B6FB284601B0F0BDB0B528
:103A1000012400250560446008300EC0B0BD70B5BB
:103A20000E460446C1680068401CFCF753FB0025A5
:103A30006068814202D1ED43284670BD226950433F
:103A4000A16841183046FCF795FBE1686068401CAE
:103A5000FCF740FB6160284670BDB0B5002400282B
:103A60000DD0054600688842FDD3401A286068687A
:103A70004018E968FCF72EFB69602046B0BDE443BE
:103A80002046B0BDB0B5002400280ED00546006821
:103A900040182860EA689042FDD8A868401811468E
:103AA000FCF718FBA9602046B0BDE4432046B0BD3A
:103AB000F0B583B0164602460027F843002E22D008
:103AC0001C46002B1FD00D46D168136899421AD9A5
:103AD000CB1AAB4217D39268019252198A423A46E6
:103AE00007D9019A8A1A0292029A52199342029AAB
:103AF00009D3029201981018FCF7ECFA3160029891
:103B000040192060384603B0F0BD406870478068B7
:103B1000704702460020002A04D010605060906078
:103B2000D1607047C0437047002803D00168484205
:103B30004841704701207047002805D00168C068DF
:103B4000411A4842484170470120704700207047A1
:103B50000020704700207047F0B583B014460D4632
:103B600006464088012818D1306900280CD0A900E9
:103B7000405801782D2910D0F368716809686A46A9
:103B80001160506010A205E0F36870680068694633
:103B900021C115A23046FFF7C5FC7768FB683046A7
:103BA000294622469847012808D00AE0C3683046D3
:103BB0002946224698477F68012802D17868002864
:103BC000F4D103B0F0BDC04646534D3A252D3873AD
:103BD0002053544154453A252D32387320455645DB
:103BE0004E543A25730D0A0046534D3A252D38732D
:103BF0002053544154453A252D32387320455645BB
:103C00004E543A25750D0A00F0B581B0002828D031
:103C10001E460C460546079B0698009000206862E9
:103C2000A862E862104909886B8029800F4B1F68E1
:103C30006C60009BAB602B460C33C4C3A861E86189
:103C40002862481C0849088008480560002C08D0F4
:103C50006C60002128460A46FFF77EFFA468002C0E
:103C6000F6D101B0F0BDC046D8CC010254C9010262
:103C700002460020002A01D0D1627047C04370473D
:103C800010B582B004AC24881B881B041B196C4639
:103C90002360024B00F0B0F802B010BD4D350000BB
:103CA000F0B597B01646029105464268002A30D01A
:103CB00001966A6001210024284616462246FFF735
:103CC0004BFF3046029FBE4232D003A85021FCF782
:103CD0006AFA32467268002F0CD003AF029811C7FF
:103CE0004068083F824209D0394608313C460028E6
:103CF0000F46F4D1002A019EDBD10AE0019E38680C
:103D00006860002128463246FFF726FF7F68002FB3
:103D1000F5D102988468002C08D06C6000212846F8
:103D20003246FFF719FFA468002CF6D117B0F0BD9A
:103D300000212846019E3246FFF70EFFE9E700000A
:103D4000014600201F2901D9C043704718224A4369
:103D5000344901238B5089188860704710B50021C1
:103D6000CC4300280BD00A4A1368002B09D0183224
:103D7000491C2029F8D306D106A0FFF7E7FE20460C
:103D800010BD0123136001600024204610BDC04611
:103D9000D8C9010274696D65722049442069732095
:103DA00066756C6C0D0A0000264800687047C046B6
:103DB00070B520241B4D234E2868022817D1306887
:103DC000A968EA68401A904211D96969002907D0A8
:103DD0002879002807D0022028603068A86004E015
:103DE0000120286003E001202860286988471835F1
:103DF000641EE1D170BDC046F0B5044600201F2C02
:103E000001D9C043F0BD059D18266643054C022725
:103E1000A751A41921710B4909682646083626C600
:103E20006361F0BDD8C9010206480168491C016000
:103E30000548416802680023521C02604B41436000
:103E40007047C0468CAD010290AD010280B5FCF711
:103E5000AAF980BDB0B50278002A24D0441C002104
:103E6000084601E0573A08E023460001D5B2302D5C
:103E70000C4611D3392D02D8303A14460CE0412DAE
:103E80000C4609D3462D01D8373AF6E71446613C73
:103E9000E4B2062CE6D30024E2B280185C1C1A7847
:103EA000002AE1D1B0BD0020B0BD10B5024601200E
:103EB00000290DD00023D45C202C02D37F2C04D306
:103EC00007E00D2C01D00A2C05D15B1C8B42F2D3EC
:103ED00010BD002010BD002010BD000081B0F0B565
:103EE00084B0099300230393002800D1C2E0002A84
:103EF00000D1BFE009AB03931678002E00D1A8E0F3
:103F00005623DB43009300231D46002900D1A2E085
:103F1000252E3FD1971C52781446643C0023142C64
:103F200043D8C0467C4424796400A7440A99A3A3DB
:103F3000A3A3A3A3A3A3A3A34CA3A3A3A3A3A3A3A8
:103F40005F000297039A131D0393126801920122E6
:103F5000002317461E460478FF0703D02D2C01D1FD
:103F6000164607E02746303F092F09D80A275F4346
:103F70003B19303B491E401C00270029EBD1394634
:103F8000029A019C002C03D0012E00D15B422360D9
:103F90006B1C06E00378B3425BD1491E521C401CE7
:103FA0002B461678002EAFD164E02A2A62D13A78E7
:103FB0000378934204D0491E401C0029F8D1002107
:103FC0006B1C3A46EDE7039A131D03933E78126883
:103FD0000023C45CB44233D0491E5B1C0029F8D1D5
:103FE0003C46C7180021002A2ED12EE00297039AE2
:103FF000131D039312680023009E0778302F18D3F7
:104000003A2F02D2344627340BE0612F03D3672FB7
:10401000344606D30DE03C46413C052C09D83446D5
:1040200020341B011B19DB19491E401C0029E4D157
:104030000021029C002A00D013606B1C2246B0E7CE
:104040003C46C718002A00D009C26B1C22463846DD
:10405000A7E700230EE0252E0BD15178652908D162
:1040600003990A1D03920968002900D008606B1C9F
:1040700000E02B46184604B0F0BC02BC01B0084773
:1040800081B010B581B00C46039303AB00930DF0E3
:104090002FFAA04200D3601E01B010BC02BC01B0D8
:1040A000084770B504460020002A1BD0002C19D008
:1040B000002B17D014600120022B13D32578002D7C
:1040C00010D0641C01208D4205D1651E00262E7083
:1040D00085005451401C984204D2661C2578002D5E
:1040E0003446F0D170BDB0B504467821FCF766F8CF
:1040F000002805D158212046FCF760F8002828D078
:104100004278002A23D0841C00210846234600015F
:10411000D5B2302D0C4613D3392D01D8303A0EE0EC
:10412000412D0C460CD3462D01D8373A07E01446F2
:10413000613CE4B2062C01D3002401E0573A144656
:10414000E2B280185C1C1A78002ADFD1B0BD0020D2
:10415000B0BD2046FCF7F2F8B0BD70B504460026AD
:10416000F043002C0DD00D4600290AD02046103017
:104170000121FFF772FCA96820342046FFF76DFC8F
:10418000304670BD70B504460026F043002C0DD0BB
:104190000D4600290AD0204610300121FFF772FC9D
:1041A000A96820342046FFF76DFC304670BD70B51D
:1041B0000024002814D00546064610363046FFF786
:1041C000B3FC01280CD028462030FFF7ADFC0128B5
:1041D00006D02C683046FFF798FC0C214143641848
:1041E000204670BDF0B583B00025029501950028EA
:1041F0001FD00C460646074610373846FFF79CFC92
:10420000002816D13046203002AA01AB2146FFF724
:104210004FFC00280DD135683846FFF778FC0C219B
:104220004143B068029A101868506D186C6001988C
:10423000A860284603B0F0BD70B505460C20584371
:104240000024904211D2121A461829606860AE60AC
:10425000EA60284610301946FFF75BFCE968203514
:104260002846FFF756FC204670BDE443204670BD4B
:1042700004217046084204D0EFF30983EFF308826B
:1042800003E0EFF30883EFF309829BB004A8F0C0CA
:1042900044464D4656465F4608A8F0C01846F0C84A
:1042A0006846F0C018690C90202018440D90586999
:1042B0000E9098690F90D8691090EFF310801190CC
:1042C000EFF31480129009490868139008490868B0
:1042D00014900849086815900749086816901793C4
:1042E00018927046199068460AF0AEFF04ED00E09F
:1042F0000CED00E010ED00E014ED00E0F0B581B051
:10430000032600243046214607F0F6FB0425284604
:10431000214607F0F1FB0127304639463A4607F0BF
:104320007FFB30462146324607F00EFC28463946D0
:104330003A4607F075FB02212846224607F004FCA6
:1043400001B0F0BDF0B589B008900425284607F00B
:104350004FFB0A27384605F033FC284607F058FB88
:104360000324204607F04CFB07900526304605F055
:1043700027FC284607F03CFB384605F021FC284680
:1043800007F046FB204607F03BFB0690304605F061
:1043900017FC284607F02CFB384605F011FC284690
:1043A00007F036FB204607F02BFB0590304605F062
:1043B00007FC284607F01CFB384605F001FC2846A0
:1043C00007F026FB204607F01BFB0490304605F063
:1043D000F7FB284607F00CFB384605F0F1FB2846B2
:1043E00007F016FB204607F00BFB0390304605F064
:1043F000E7FB284607F0FCFA3846019705F0E0FB9A
:10440000284607F005FB204607F0FAFA02903046EE
:1044100005F0D6FB284607F0EBFA384605F0D0FB4E
:10442000284607F0F5FA204607F0EAFA0746304634
:1044300005F0C6FB284607F0DBFA019805F0C0FB43
:10444000284607F0E5FA204607F0DAFA0446304637
:1044500005F0B6FB284607F0CBFA0699481E8141C5
:104460000A460799481E8141480080188000059A35
:10447000511E8A4151004018049A511E8A418018E9
:104480008000039A511E8A4151004018029A511E21
:104490008A4180188000791E8F4179004018611E82
:1044A0008C4106190898002803D0032007F0A0FAD1
:1044B00002E0032007F0ACFA0A24204605F080FB56
:1044C0000425284607F0A4FA204605F079FB284683
:1044D00007F08EFAF0B209B0F0BD70B504460420C2
:1044E00007F086FA60B2002803D4032007F080FAB0
:1044F00002E0032007F08CFA0A25284605F060FB4D
:104500000426304607F084FA284605F059FB304669
:1045100007F06EFA284605F053FB600603D403202B
:1045200007F066FA02E0032007F072FA0A2528462F
:1045300005F046FB0426304607F06AFA284605F0E7
:104540003FFB304607F054FA284605F039FBA00639
:1045500003D4032007F04CFA02E0032007F058FAD6
:104560000A25284605F02CFB0426304607F050FAB1
:10457000284605F025FB304607F03AFA284605F0B4
:104580001FFBE00603D4032007F032FA02E0032009
:1045900007F03EFA0A25284605F012FB04263046AD
:1045A00007F036FA284605F00BFB304607F020FAF4
:1045B000284605F005FB200703D4032007F018FA6E
:1045C00002E0032007F024FA0A25284605F0F8FA4D
:1045D0000426304607F01CFA284605F0F1FA30466A
:1045E00007F006FA284605F0EBFA600703D403202B
:1045F00007F0FEF902E0032007F00AFA0A25284630
:1046000005F0DEFA0426304607F002FA284605F0E7
:10461000D7FA304607F0ECF9284605F0D1FAA007A2
:1046200003D4032007F0E4F902E0032007F0F0F9D7
:104630000A25284605F0C4FA0426304607F0E8F9B2
:10464000284605F0BDFA304607F0D2F9284605F0B5
:10465000B7FAE00703D1032007F0CAF902E003200C
:1046600007F0D6F90A24204605F0AAFA04252846C0
:1046700007F0CEF9204605F0A3FA284607F0B8F96E
:10468000204605F09DFA70BDF0B581B003260025E7
:10469000012430462946224607F0C2F9304607F089
:1046A000B7F90626304605F08BFA042007F0B0F97A
:1046B000304605F085FA032007F0A2F900281BD048
:1046C000681CFA2D0546F6D30425284607F090F914
:1046D0000326304607F08CF90A27384605F070FAB1
:1046E000284607F095F9304607F092F9384605F06C
:1046F00067FA204601B0F0BD032001210A4607F009
:104700008FF9042007F074F90024204601B0F0BDB1
:10471000B0B50446C00703D1032007F069F902E0F1
:10472000032007F075F90825284607F071F9284697
:1047300007F05EF9A00703D4032007F059F902E05F
:10474000032007F065F90825284607F061F9284697
:1047500007F04EF9600703D4032007F049F902E09F
:10476000032007F055F90825284607F051F9284697
:1047700007F03EF9200703D4032007F039F902E0DF
:10478000032007F045F90825284607F041F9284697
:1047900007F02EF9E00603D4032007F029F902E020
:1047A000032007F035F90825284607F031F9284697
:1047B00007F01EF9A00603D4032007F019F902E060
:1047C000032007F025F90825284607F021F9284697
:1047D00007F00EF9600603D4032007F009F902E0A0
:1047E000032007F015F90825284607F011F9284697
:1047F00007F0FEF860B2002803D4032007F0F8F8B1
:1048000002E0032007F004F90824204607F000F92D
:10481000204607F0EDF80724204607F0F9F8204677
:1048200007F0E6F8B0BDF0B581B0032700243846A4
:10483000214607F051F93846214607F05DF9012578
:1048400038462946224607F0EBF805263846294621
:10485000324607F079F908273846214607F04CF927
:1048600038462946224607F0DBF8384629463246C4
:1048700007F06AF907273846214607F03DF9384620
:104880002946224607F0CCF838462946324607F03A
:104890005BF901B0F0BD000080B50B2007F0B0F867
:1048A00012490A78002804D0002A12D003F0E4FA52
:1048B00080BD012AFAD1002008700F49C8830C4935
:1048C00008700C48012101700BF03CFC03F0D4FA95
:1048D00080BD0748012202700A700648002101705D
:1048E0000BF050FC03F0C8FA80BDC0461C900102DA
:1048F000189001021990010232A901020248406990
:10490000811E4842484170476896010280B5FDF714
:1049100051FA002801D00020C04380BD80B5FEF7C9
:10492000FFFA80BD10B504480F2100242246FFF78E
:1049300013F9204610BDC046DC990102F0B581B0E4
:1049400007460324204607F063F80425284607F0AD
:104950005FF8204607F04CF80A26304605F030F99B
:10496000284607F045F83220FFF7B7FDFFF78CFE29
:10497000F8B2FFF7B2FDFFF787FE204607F048F8D0
:10498000284607F045F8204607F032F8304605F093
:1049900017F9284607F02CF83320FFF79EFDFFF7A4
:1049A00073FE0020FFF7CEFC0746284607F020F8EC
:1049B000204607F01DF8304605F002F9284607F0BA
:1049C00027F8204607F024F8304605F0F9F8384675
:1049D00001B0F0BDF0B581B0009107460324204638
:1049E00007F016F80426304607F012F8204606F0C5
:1049F000FFFF0A25284605F0E3F8304606F0F8FFE9
:104A00003220FFF76AFDFFF73FFEF8B2FFF765FDC2
:104A1000FFF73AFE0098FFF760FDFFF735FE3046DE
:104A200006F0E6FF204606F0E3FF284605F0C8F84A
:104A3000304606F0EDFF204606F0EAFF284605F076
:104A4000BFF8284605F0BCF801B0F0BD80B50748B6
:104A500001210170064802680A43026005480268A5
:104A6000002A02D000200146904780BDDECC010222
:104A70001C100050E0CC0102F0B599B0F548017B64
:104A8000C67A427B0E92F44C221F1368F34A1268D6
:104A9000069242780C9202790592C76A04931F40ED
:104AA00001200F907A0200D5BCE03A0200D5BFE0A9
:104AB000FA0102D50F9802062260502508968A193D
:104AC0001826BB0102D50F984306236041230795A2
:104AD00069430A96354655431426FC0210D50F98B3
:104AE000040538463746DC4E3460DA4CA469B464B9
:104AF000D84CE4697464DA4C241D34603E460746A1
:104B000090000B90D8040D90681809900E9B734389
:104B10000F988203B902D04D22D50F984105296024
:104B2000CC480E961646024681692965C1696965B9
:104B300009990D9801430898000108180B9940182D
:104B4000C018C849098892794A4380180A301C461F
:104B500005F016FB234632460E9EC04988672A6040
:104B60000F98C404380300D52C60F80302D50F98C1
:104B7000000428600F984104B80300D52960380468
:104B800000D4E4E1039402910E9308920D980B99DE
:104B90000C180A980C9941430C910F98C0030B9084
:104BA000286008F021F9002801D005F0CBFA0C9814
:104BB000005B410B43D1099800190E9940180599E3
:104BC000090140180E90E74D287B079B4343E97A83
:104BD0000A010D9C2243D21841188B00D2180A9B5F
:104BE0004B43D1186A7B564389190E9E2A791018B7
:104BF000DF4A12884243881816903068C000800D42
:104C000010A9C882002511957079C0077ED110A81F
:104C10000F998182069C00940020E8A2049B0BF06F
:104C200055F978E00F98820522603A0200D43FE7F8
:104C30000F98C2052260FA0100D53BE73DE7072146
:104C400049030840032149038842089A00D07EE1C5
:104C5000069707F03DFD0020169009901590C14C75
:104C6000E07A217B08180A99414380000D9A10438D
:104C70004118627B0E9672438A186178A379079E69
:104C80007343D718FA683F26324063789A420C97EC
:104C90006ED105960A9A4A4380580F210A070240AE
:104CA0000398401EC04B1B68DB0903409818109006
:104CB0000F98C0020B90B868800767D42C46283C38
:104CC0000AF07AF805462068000609D5C320840159
:104CD000786A400704D40AF06FF8401BA042F7D965
:104CE00005980002B96849080140B3480368826822
:104CF000B868C40C20202040DB0700D095E00023DA
:104D000010221D461C460E9E0B9FB1E010A8858206
:104D1000B0681190069C701D924B1979E20707D17B
:104D2000491C1971D97A1A798A4202D31D7100E09F
:104D3000D9700178427812025118827812048918C9
:104D400003229143017035715878401C5870D87A0D
:104D5000197B08185978884200D85D70D879401EB0
:104D6000D871596B002901D010A888477E4DEDE01D
:104D700010A80B998182F868304063780090002079
:104D80007CA20F990BF0A2F80E9E94E0388A874A15
:104D9000024010A8C2822022BA5C9307DB0F3C6855
:104DA000C3720F9B1A4082726205D20C0D9B1A438C
:104DB0001692FA68130E0372BB69FC697C4D2D686C
:104DC0002D0C05745204920F427211931394654C8A
:104DD000A07B002809980E9E0B9F5FD07548006845
:104DE000007A0328099859D00C98007D08400928BA
:104DF000099853D1C320840109F0DEFF05460C98C1
:104E0000406A41070BD4594909680906890F06D140
:104E100009F0D2FF401BA042F1D90C98406A41032F
:104E20000898884310A9888237E0D2070E9E0B9F0E
:104E300003D108230022154619E00C9B9A68029CB6
:104E4000224211D19A68520C022494430022134644
:104E500015460DE0E4D1010228A000503CA100500D
:104E6000FC1F0000E0D10102042500221346144675
:104E70000843104318432843204310A9888238422E
:104E80000BD10C9B198A494A0A4010A9CA82196899
:104E90004905C90C0D9A11431691324C2921615CC8
:104EA000002908D03037B84205D010A90846113083
:104EB000123109F09BFAE77A2A48047BE519294860
:104EC00000790E9027484078401C2946FBF702F9EC
:104ED00088000D9A104318900799614338011043D8
:104EE00040182049497B4E4380191C2169434018D2
:104EF0000E9909191B4B1E4A12884A4380181790B5
:104F0000099A0C998A60987B002800D04A629879A7
:104F1000401C9871187B99798142069F00D39A7141
:104F20005978491C5970D97A0818597888420E4D19
:104F300000D85A70187A401E18722820185C002871
:104F400004D0996B002901D010A88847089A17420D
:104F500002D00F98000328601C480449486019B02B
:104F6000F0BDC046E4D1010228A000503CA1005091
:104F7000E0D1010248572045542069647820256417
:104F800020616E642045542069647820256420697E
:104F90006E2052582064657363206D69736D61746F
:104FA00063680D0A0000000038200040FF03000085
:104FB0009430004044940102604000404D41432041
:104FC0004556542025782025780D0A00FFFFFF0361
:104FD000F0B5A5B01E460C9208910024239422A996
:104FE0000C8016A90C8024A909250D80598C0D91DF
:104FF000FBF770F82A99012900D0DFE031890129F7
:1050000000D0DBE0318C012900D0D7E00D990029D8
:1050100000D1D3E0224607962C990B912B9906914B
:1050200080B205900F9415A8058090000E900C9901
:105030000C582E460025204629461746FBF7F2FB62
:105040000028119636D12C200A9778430899081821
:1050500017A90A4668C868C2E8C8E8C2E8C8E8C232
:10506000079F119880B280000E5822AD019523A8A9
:10507000009020463946059A069B04F0AFFD0F9834
:10508000401C0F90288800282DD03B8A239913AC10
:10509000039416A8029014A8019015AE009617A8C4
:1050A00024AA04F075FF2588308811900120149EF1
:1050B0000A9A05E013A8058014952E4628463A461C
:1050C0000E9F51000B9B119C5C52591808830D8454
:1050D000D81986600F981885521C0D9882426DD0A1
:1050E00024A805889FE7099616A800250580149531
:1050F00024A80688239812902F46109503E06D1C73
:10510000A8B2B04213D8A8B2800017A90C58204604
:105110001299FBF795FB0028F1D1002FEFD115A8CC
:10512000058016A80127078014941094E7E715A8B6
:105130000288B01A012805D115A80680099F149786
:10514000119628E010200799095E0129119221DBB0
:10515000551CA8B20C18109F0E9B099403E06D1CFF
:10516000A8B2844218DDAAB2B242F8D8800017AAC9
:1051700010581090394634461E46FBF753FB334611
:105180002646099C0028EAD115A80580109F14978F
:105190001195E4E7109F0E9B1C463E463846129937
:1051A000FBF76FF9FBF7FAFB0546052800D3052549
:1051B00013A8058001200A9A274682E725B0F0BD92
:1051C000F0B58BB00243159A149C139E2BD0054664
:1051D00001A856C0129CD869196A09900A911E4606
:1051E0009F6B0123009309A807AA0146059306F0C7
:1051F000D1FC716C3846FBF744F90746E06A616BF5
:10520000FBF73FF9002D069613D00446119801993B
:10521000012924D10921081A0421069A515E8842E5
:1052200029D16425B1E000203080207010700BB0CF
:10523000F0BDB08800226425002829D00592694974
:105240003846FBF719FB0028049C039E6FD1664982
:105250003846FBF711FB00281DD05A2567E03C2596
:10526000082800D191E05F492046FBF705FB0028A4
:1052700019D0502589E00A291DDB1D293BDC59493D
:105280003846FBF7F9FA0022002854D05A253AE0B4
:105290003346049C39E055493846FBF7EDFA0028BF
:1052A00021D0502543E050492046FBF7E5FA00287D
:1052B0002ED0462569E03C25012866D04949204684
:1052C000FBF7DAFA0028D4D147492046FBF7D4FA95
:1052D0000028EED145492046FBF7CEFA002854D1EC
:1052E000434920466EE042493846FBF7C5FA00289C
:1052F0001CD128251BE03B493846FBF7BDFA0022AC
:10530000002832D05025049C069B0299039E41E060
:1053100036492046FBF7B0FA002836D134492046FA
:10532000FBF7AAFA00282FD114252EE03725029981
:10533000059A069B2EE005922B493846FBF79CFA0E
:10534000002896D129493846FBF796FA0028B0D1B3
:1053500027493846FBF790FA0028049C069B0299DF
:10536000039E059A3BD11E2514E005921E4938463E
:10537000FBF782FA00289CD11C493846FBF77CFADF
:1053800000281DD03C2500E02325049C069B0299A3
:10539000039E059A2580327000200870307800281E
:1053A0000CD118681349FBF759FA002806D1208858
:1053B000102803D30F3820800BB0F0BD0BB0F0BD28
:1053C0000B493846FBF758FA0028049C069B0299C3
:1053D000039E059A01D11425DCE72325DAE72D2564
:1053E000D8E7C046CDCCCC3DCDCC4C3DCDCCCC3C93
:1053F0000AD7233C0000204070B588B00C46064612
:105400004088002820D0FBF78AFA059005A804A957
:1054100001252A4606F028FE3088B188081AFBF7D5
:1054200073FA0390049903A807AA2B4606F0DCFD43
:105430005249079D2846FBF71FFA002808D0BF20D5
:105440000006206008B070BD0020206008B070BD6C
:105450004B492846FBF7F4F9002804D03F2000060A
:10546000206008B070BD47492846FBF705FA0028C0
:1054700001D0002010E000212846FBF7FDF90028AC
:1054800001D0022008E040492846FBF7F5F9002842
:1054900001D0042000E0062001957F21C90502917A
:1054A00080003A49091801A806AA022306F050FD17
:1054B0000698206008B070BDF0B587B00C46054670
:1054C0004768002638463146FBF7E4F9002802D049
:1054D000266007B0F0BD049704A803A90126324650
:1054E00006F0C2FDA8682968FAF786FF02900399C2
:1054F00002A806AA334606F077FD2049069D2846F5
:10550000FBF7BAF9002804D0BF200606266007B0D2
:10551000F0BD1B492846FBF793F9002804D03F2033
:105520000606266007B0F0BD16492846FBF7A4F929
:10553000002801D0002010E000212846FBF79CF94C
:10554000002801D0022008E00F492846FBF794F913
:10555000002801D0042000E0062000957F21C90525
:105560000191800009490918684605AA022306F03E
:10557000EFFC059E266007B0F0BDC046CDCC0C3FC9
:10558000295C0FBFCDCC4C3ECDCC4CBE4C9401021F
:10559000F0B587B00C4606467F270088002801D06A
:1055A000FD0503E0B08800282ED0334DFBF7B7F996
:1055B00003907088FBF7B3F9049003A802A90126B1
:1055C000324606F051FD029904A806AA334606F0B9
:1055D0000BFD2A49069E3046FBF74EF9002802D003
:1055E0003F20010641E026493046FBF729F9002813
:1055F00002D0BF20010638E022493046FBF73CF9D3
:10560000002805D0002024E00020206007B0F0BD75
:105610001D493046FBF730F9002801D0022018E080
:105620001A493046FBF728F9002801D0042010E081
:1056300017493046FBF720F9002801D0062008E082
:1056400014493046FBF718F9002801D0082000E083
:105650000A200096F905019180000F490918684653
:1056600005AA022306F074FC05992846FAF7CCFE39
:10567000206007B0F0BDC046000080BF0000384386
:105680003333733F0000C8420000704200002042E4
:105690000000A0410000C0406C940102F0B59DB034
:1056A00015460B917F210391C9051C9102911B9115
:1056B00019A900248C80199418941794598C069178
:1056C000198C0F91DE8B998B0791997805911F8822
:1056D0002B21CA432799914201DB7F0015E040222C
:1056E000D243914211DC4922D243914202DB790834
:1056F000CF190AE05322D2439142EEDA5D22D2431F
:10570000914201DBBF0000E0FF000A971396269E3E
:10571000597E00290BD0002132460F46D17091707E
:1057200051701170121D7F1C5C7EA742F6D30C9342
:1057300011952599149122990D91159041088C424B
:1057400011D2FD4A2346A00084583454270A451C30
:105750007755250C871CF555240EC01C34545B1C52
:105760009CB2A142EFD8239810900120099000909C
:1057700030463146149A159F3B4606F019FA0D98AB
:1057800000060890400E139D00D186E0680004904A
:10579000002F3FD0002210461146144606E01C465A
:1057A0001146159F401C82B2BA420ED283B2AB4260
:1057B000F8D09200149B9A5E0FB2BA42034600DC06
:1057C0002346BA42EBDC0A46E9E7002F25D0002247
:1057D00010461146129206E012931146159F401C86
:1057E00082B2BA4214D283B2AB42F8D0A5B2AB4275
:1057F0000CD09200149B9A5E0FB2BA42034600DCB2
:10580000129BBA42139DE7DC0A46E5E7139DE6E7E3
:10581000129903E00024214600E000211291109823
:105820000183C4828582049FF057FBF76DF87921CC
:10583000C9050E91FAF7E8FD1099C8610998074368
:10584000F057FBF761F80E99FAF7DEFD109F38620A
:105850002004C40B3057FBF757F80E99FAF7D4FD24
:105860007862601C3056FBF74FF80E9C2146FAF721
:10587000CBFDB86212980004C70BF057FBF744F851
:105880002146FAF7C1FD109CE062781C3056FBF708
:105890003BF80E99FAF7B8FD2063119805800C9833
:1058A000407E410000278D4228463A46149E1ED372
:1058B0000A9880B28AB29300F45E84420BDA491CE3
:1058C0008AB2AA42F6D9002728463A4681B2691A16
:1058D000012910D01BE0F018119B198007880804DB
:1058E0000FD0500040008019001F0288084681B286
:1058F000691A01290BD1A800301811990D80078869
:1059000026E00020024681B2691A0129F3D00A99E3
:1059100089B2079B4B43BB421AD306998A4217D8D8
:105920000599002914D0401C82B2891803E0401C5C
:1059300082B291420CD983B2AB42F8D89200B35EE6
:10594000BCB2A342F3DDB218119B18801788EEE7B2
:1059500012970B980580119800882B1A002B16DDE2
:1059600002210F9A1143032942D10E93411C421E7A
:1059700010B281420EDA0E98032824DB0C98808C3A
:10598000012820D019A818A9FFF736FD1FE0002034
:1059900018902BE00026F443374608E0B8B24000E8
:1059A00019AD2B527F1C521C10B28142E3DB13B2A3
:1059B000A3423346F2DD159B98423346EEDA80006F
:1059C000149B1B5AEAE719A818A9FFF7E1FD149EDA
:1059D000139D0F9A012A13D0032A11D0022A04D151
:1059E00011980088281A02280ADA0020179034E05B
:1059F000022A01D1022BB8DA00201890012AEBD13B
:105A0000681C691E0FB2B84208DA0C98808C012815
:105A10001DD119A817A9FFF7BBFD1CE00022D34335
:105A2000144608E0A5B26D0019AF7E53641C491CF2
:105A30000FB2B842E9DB0DB29D421646F2DD159D6C
:105A4000AF421646EEDABD00149E765BEAE719A86F
:105A500017A9FFF7D1FC149E139D249F189C17993A
:105A60002046FAF7C9FC0F99012900D82046386072
:105A70000D98002800D1CBE011990888109FB886B6
:105A80000888281AB880129880B2FAF748FF79215E
:105A9000CC052146FAF7B8FC2146FAF7B5FCB86305
:105AA000119F3888002849D081008919091F098869
:105AB000129C0C191599884203D2800080198088A5
:105AC000041915984300534916AA304606F04EFAB9
:105AD000169810994864FAF77AFFA4B2A04201D14F
:105AE0004D480FE0001BFAF71AFF1C901CA81BA9D9
:105AF000012206F0B9FA2046FAF711FF01461B9879
:105B0000FAF782FC109908603988491B4A1C92B246
:105B1000032A02D20021159F17E009B20229159F1E
:105B200012DB3F210906FAF7A7FE002802990CD1E3
:105B30000998810709E0C046402100400020129CDE
:105B400015998842B9D3BCE7344910980161089887
:105B5000800E5DD0002F1CD0002211461446104646
:105B60004B1B1DB2ED135B196B40139D1BB29200D2
:105B7000B25E53431818A418491C8AB2BA42EFD334
:105B8000FAF7CDFE06462046FAF7C9FE002C03D1EF
:105B900000E000260398C0051C901CA81BA9012545
:105BA0002A4606F061FA1B9C20463146FAF72CFC87
:105BB000014610988160002F119422D000242746BE
:105BC000264613951291B8B2FAF7A9FE1299FAF780
:105BD00013FC0546A0001499085EFAF795FE0146ED
:105BE0001398C00785432846FAF70EFC0146304655
:105BF000FAF7B1FB06467F1CBCB215988442E2D38B
:105C000000E0002611983146FAF7FEFB1099C860B3
:105C10001DB0F0BD30A7010200002041000040404F
:105C2000F0B58FB00692F74A09AF70CA70C770CA54
:105C300070C70328079320D88800F3A10858F649B5
:105C4000FAF789FB0446F549FAF785FB0D90F4490C
:105C50002046FAF780FB0C90F2492046FAF77BFBCE
:105C60000B90F1492046FAF776FB0A90EF4920465F
:105C7000FAF771FB0990EE4969E0042822D0062862
:105C800020D88800EBA10858EE49FAF764FB0446D7
:105C9000ED49FAF760FB0D90EC492046FAF75BFB03
:105CA0000C90EB492046FAF756FB0B90E949204649
:105CB000FAF751FB0A90E8492046FAF74CFB0990A5
:105CC000FD4944E00838022821D88800FBA1085883
:105CD000D149FAF740FB0446FC49FAF73CFB0D902A
:105CE000FB492046FAF737FB0C90FF208105204640
:105CF000FAF731FB0B90F7492046FAF72CFB0A9094
:105D0000CA492046FAF727FB0990FE491FE08800A0
:105D1000F1A10858F449FAF71EFB0446F349FAF7D3
:105D20001AFB0D90F2492046FAF715FB0C90F14949
:105D30002046FAF710FB0B90EF492046FAF70BFBD1
:105D40000A90EE492046FAF706FB0990EC490094C8
:105D50002046FAF700FBEC4909680E90EB4804680E
:105D6000EB4801684808EB4F05463D400022002DF6
:105D700008922DD0CA01120E07D0280CE90D12D1BD
:105D80004000E649085AE6490AE0C903090E0CD06A
:105D9000280AE90B10D14000E049085A8F218900F8
:105DA0004018E4300DE0DC490AE081B27F2905D8D3
:105DB0004800DA49085A04E0D94901E08F218900F6
:105DC000401800B2FAF7A0FDD649FAF71DFB0246CB
:105DD0000292039507252606D34B1A68002A0898D5
:105DE00040D0791C8A420BD21102090E13D0110C3B
:105DF0001F46D00D1FD14800C849085AC84907E0BE
:105E00001F46110E002A13D44800C449085AC2493B
:105E10004018E4301FE011041F46090E0ED0110A8D
:105E2000D00B12D14800BD49085A8F218900EFE7F5
:105E3000BE4808180FE0B84808180CE091B27F2956
:105E400006D84800B549085A05E0B548081802E0E8
:105E50008F218900501800B2FAF756FDB149FAF7C0
:105E6000D3FA3B460590159F2C40F50E5B69B0496F
:105E70001940089810D0DA02D20E34D0C80B3E2157
:105E80000140A648405AA6494018E43000B2FAF74B
:105E90003BFDA449FAF7B8FA0490149E6800A5A146
:105EA000085EFAF731FD0146A00009AA1058FAF77A
:105EB00052FA0146B8B20128089F019102D1022C82
:105EC0000AD9A74F052C24D1189808900C2D20D85A
:105ED0000B2D16D3A44918E00027022C089718D0E0
:105EE0008120C70515E01A04120E00D1CAE0080A85
:105EF000C90B00D0CDE040008849085A8F218900A5
:105F0000C2E7092D00D2C7E096490898FAF723FAAC
:105F1000089001200021B542034600D30B46052C12
:105F200000D308461799169A1A9C199D1843069B88
:105F3000012B12D1079B402B22D1002840D038469C
:105F4000FAF709FA01460198FAF705FA01460098AE
:105F5000FAF752FA059A04998AE0079B402B1FD161
:105F6000002838D03846FAF7F6F901460198FAF7D2
:105F7000F2F901460098FAF73FFA059A049977E09A
:105F8000002833D03846FAF7E6F901460198FAF7C7
:105F9000E2F901460098FAF72FFA059A049967E0AA
:105FA00000285BD03846FAF7D6F901460198FAF78F
:105FB000D2F901460098FAF71FFA059A049957E0BA
:105FC00002981146FAF718FA0399002900D1674898
:105FD000059A04994CE002981146FAF70DFA0399D4
:105FE000002900D16148059A049941E002981146C0
:105FF000FAF702FA0399002900D15C48059A04993E
:1060000036E0C046681F0100000068C1000088C17A
:1060100066665EC1000084C1000084410000B44196
:1060200000004841000020400000F0C0000084C192
:106030000000F841333323C1000050C19A9929C1AF
:106040009A9949C19A9949413333CB416666764161
:10605000CDCCAC40333393C09A9949C102981146D4
:10606000FAF7CAF90399002900D14048059A049922
:1060700028601046FAF7C0F90899FAF7BDF92060D0
:106080000FB0F0BD99B27F2911D848002349085AB2
:10609000FCE623494018F9E6C12001060898FAF702
:1060A0005AF90890062D00D933E7002030E78F21F8
:1060B00089005818EAE6C0463333F341000058C15E
:1060C0009A9961C19A9969C1000084C10000AC41EC
:1060D00000003841000008C1CDCC80C1CDCC88C1C2
:1060E00033338FC1333397C133339741CDCC8C4198
:1060F0003333F3409A9919C0666646C1333397C16A
:10610000CDCCB4410000D4410C00004050300040E0
:1061100068400040FFFFFF007C080000742301007E
:106120005C050000919AF63C642000409C0B000046
:10613000FFFF1F00FAFFFCFFFEFF0000020004004B
:10614000060008000A000C000E00100012001400E7
:10615000160018001A001C001E0020002200240057
:10616000000080BF0000A0C0000040C00000DCC2F2
:10617000F0B5FFB0ECB017460E460D900021E99146
:10618000E891DC919991989197919691149113913E
:1061900012919AA8F49DF39CF29A002E00D1E6E1A8
:1061A0000B938030F09B1180099529602546DBAC6C
:1061B000218095AC21800C952980DA917F24E4051B
:1061C000B994B894B794B694B594B494B394B29483
:1061D000B194B094AF94AE94AD94AC94AB94AA94B3
:1061E000A994A894A794A694A594A494A394A294E3
:1061F000A194A0949F949E949D949C949B949A9413
:10620000046644668466C466046744678467C4673A
:10621000046444648464C464046544658465C4653A
:10622000046244628462C462046344638463C4633A
:10623000046044608460C460046144618461C4613A
:10624000B0090B250B2800D3AE011095012B0B9D37
:1062500000D070E12B89012B00D06CE1298C002942
:106260000E9200D18BE16B8C002B00D1FAE1AA8C4D
:106270003021695C002900D188E10892109F5F43BA
:106280001196304639460F93F9F724FF0590FAF737
:106290003BFB01462046FAF7F4F88321C905FAF7DB
:1062A000B3F8064696A8021D119887420A9200D8B4
:1062B00079E155A811909AA9069196AF15463A46EC
:1062C000059C234605F044FE15A80F9006992A4622
:1062D000234605F03DFE02230D93384631463A46EB
:1062E00005F082FE012308930093E8AA1092384635
:1062F000394605F04FFCE898DD901198069D294637
:106300003A46234605F024FE0F9829460A9A23466A
:1063100005F01EFE384631463A460D9B05F064FEF8
:10632000089B009338463946109A05F033FCE898EC
:10633000DE9011982C4629463A46059D2B4605F0DD
:1063400007FE0F9821460A9A2C462B4605F000FEC0
:10635000384631463A460D9B05F046FE089B0093B1
:1063600038463946109A05F015FCE898DF901198E8
:10637000069D29463A46234605F0EAFD0F98294630
:106380000A9A2346254605F0E3FD384631463A464B
:106390000D9B05F029FE089B009338463946109A5C
:1063A00005F0F8FBE898E0901198069C21463A46E3
:1063B0002B4605F0CDFD0F9821460A9A2C462B4618
:1063C00005F0C6FD384631463A460D9B05F00CFEF9
:1063D000089B009338463946109A05F0DBFBE89895
:1063E000E1901198069D29463A46234605F0B0FDF6
:1063F0000F9829460A9A2346254605F0A9FD3846F6
:1064000031463A460D9B05F0EFFD089B0093384658
:106410003946109A05F0BEFBE898E2901198069C68
:1064200021463A462B4605F093FD0F9821460A9ADD
:106430002B4605F08DFD384631463A460D9B05F05A
:10644000D3FD089B009338463946109A05F0A2FB0D
:10645000E898E390119821463A462B4605F078FDDE
:106460000F9821460A9A2B462C4605F071FD3846B6
:1064700031463A460D9B05F0B7FD089B0093384620
:106480003946109A05F086FBE898E4901198069D2D
:1064900029463A46234605F05BFD0F9829460A9A9D
:1064A0002546234605F054FD384631463A460D9BB5
:1064B00005F09AFD089B009338463946109A05F07E
:1064C00069FBE898E5901198069C21463A462B46D0
:1064D00005F03EFD0F9821460A9A2B4605F038FD3F
:1064E000384631463A460D9B05F07EFD089B0093E9
:1064F00038463946109A05F04DFBE898E690119819
:1065000021463A462B4605F023FD0F9821460A9A6C
:106510002B4605F01DFD384631463A460D9B05F0E9
:1065200063FD089B009338463946109A05F032FB0C
:10653000E898E7907AE010880C9A108099919891E9
:10654000DA9E08460F46099DF59CF9F755FF28602D
:10655000DC9827606060A6600C34DDA80EC80EC40D
:106560002EC82EC42EC82EC47FB06CB0F0BDFF2044
:1065700010800021296020807FB06CB0F0BD002227
:1065800001233021695C002900D076E6DDAA1ACF0C
:106590001AC23ACF3AC23ACF3AC20B213046F9F783
:1065A00099FD054642E000200690059D0796089F4C
:1065B0001190069801460D9C0F9A4A43D219109BE0
:1065C0005A43119BD218D200A35889002E4655ADCC
:1065D0006B503546121DA25815AB5A50401C01B2E3
:1065E0008E42E9DC55A89AAE96AC314622462B463F
:1065F00005F0AEFC15A831460A9A2B4605F0A8FC1A
:10660000022320460799224605F0EEFC0123009361
:10661000E8AA2046214605F0BDFA119B9800DDA9A5
:10662000E89A0A505B1C0B2B1846C1D1F19EDDA8DD
:106630009AA9DCAA0B2305F08BFC09210E980F9177
:1066400001800B98C168DC9C2046F9F7DDFE01460D
:10665000A8B2E69F0F281BD808280DD30846F9F7E3
:106660007AFE14E0FF2010800021099A11600C9935
:1066700008807FB06CB0F0BD042803D381220846A7
:10668000D10502E0412208461106F9F7BDFE014698
:106690002B20C04386420D9704DB0846F9F75BFECA
:1066A000014603E04020C043864244DD0E9A0C9C24
:1066B0000B98408A002811D00B98038A95A8039064
:1066C000DBA80290DAA801900094DDA80D4603F043
:1066D0005FFC29462488DA9E099D68E011910F9895
:1066E000208000273D46109705E00E9804887F1C07
:1066F000B8B2A04211D8B8B28000DDA90C5820462B
:106700001199FAF79DF80028EFD1002DEDD10C98E2
:10671000078001250F971094E7E7DBA805800F9A03
:1067200090B2201A012811D10C9804800D9FDA979D
:106730003E46099D3AE04920C043864200DA8BE09C
:10674000FF2208469105F9F75FFEA9E710200B9993
:106750000E5E012E00DA90E0551CABB21846A1B2D5
:10676000AAB28A4217D805E00E990C88A1B2AAB243
:106770008A4210D88000DDA90C58204610991F4687
:10678000FAF750F83B46002805D10C9805800B9885
:10679000068A0F95109430B2C1186D1CA8B28142C0
:1067A000E2DC109EDA960F9C099D0D9F11993046F0
:1067B000F9F767FEFAF7F2F8052800D3052095A946
:1067C0000880A0B20E990988814218D9401C611E28
:1067D0000CB2A04218DA12A898A9FEF76DFE0E9826
:1067E0000188481C491E0CB2A04221DA12A899A9BE
:1067F000FEF762FE99999898099D0D9FA4E60021E5
:106800009891999108469FE60022134608E09CB2B1
:10681000A40012AF3D515B1C491C0CB2A042DADB54
:106820008DB20A2D1546F2D8A400DDAD2D59EEE744
:106830000022134608E09CB2A40012AF3D515B1C3D
:10684000491C0CB2A042D1DB8DB20A2D1546F2D8FC
:10685000A400DDAD2D59EEE75320C043864200DB96
:106860001BE70E460B9881692046F9F7DBFF0028ED
:106870000C9C08D10B98808B07E01446099D0D9F56
:106880001199109E93E70B98C08BFAF748F80146D0
:106890003046F9F7B9FD119021E70000F0B58BB053
:1068A0001C4609930E46034600200A904048008883
:1068B000224F05970AA9049103940292109C019417
:1068C000012500950B21414389B230331C4A3046E3
:1068D000FFF74EFC3868079078680890B868069013
:1068E00033480088334F009501940297324E30367A
:1068F0003249334A3346FEF76BFB0698F862079835
:10690000386308987863099800882E4905912E49C4
:1069100004912E4903910297019000962C4B284632
:1069200029462A46FEF74CFC432001060A98F9F74F
:106930006BFDFAF733F80BB0F0BDC046F8A60102C4
:10694000B0DF0102F0B589B00F9F0E9C002815D072
:106950001098079016480088164E01250095019161
:1069600002960893144B30331449154AFEF730FB56
:10697000089BF76207983063746303E00D48476330
:10698000C462002518880F4905910F4904910F49E9
:10699000039108490291019007483030009001218D
:1069A0000B4B28460A46FEF70BFC09B0F0BDC0466B
:1069B0009CAD010274D401025CA00102E49E0102BC
:1069C00084D2010228A4010298AD010238AD01026F
:1069D00040AD01023048704700487047DCAD01020D
:1069E000800037490918C86B0022CA637047C04647
:1069F000800033490918886C00228A647047C046B9
:106A000080B52F4AD369002B01D0126A9847002025
:106A100080BDC0460249087800220A707047C0460F
:106A20004CC901020020704780B5182905D80346DB
:106A30008A1E03481946F9F79DFB002080BDC04619
:106A4000A0AD0102B0B502460020022901D2C04328
:106A5000B0BD8C1E0F2C07D8044D28461146224687
:106A6000F9F788FB00202855B0BDC046BCAD010237
:106A7000B0B502460020022901D2C043B0BD8C1E31
:106A80000F2C07D8044D284611462246F9F772FB11
:106A900000202855B0BDC046CCAD01020849087899
:106AA00000220A707047C046B0B50446044DAA687B
:106AB000002A02D0E968204690472C610020B0BD32
:106AC000AC970102B0B5D44DE869002819D0284828
:106AD000007800281BD0012829D127480068CD491B
:106AE0008A8A904224DA2878002804D0002028706E
:106AF000022002F03BF90020687028621D490870EE
:106B0000B0BD0020286268701A490870B0BD2878AE
:106B1000002803D10120287002F028F9154801212E
:106B20000170002028626970C04313490860B0BD3D
:106B300001246C702A6A531C2B62C98A884209DDC1
:106B4000132AF4DB287800280DD12C70204602F09F
:106B50000DF908E0132AEADB2878002803D12C700D
:106B6000204602F003F90020286202480470B0BDFC
:106B700030990102AD9601025499010280B5124884
:106B800001681F220A40026003200840022812D137
:106B90000E480268D30D02D0FF231B06D2180C4BFF
:106BA0001A600C4A12680C4B1A6080680B4A1080FD
:106BB000000C0B4A10801A488268002A02D08268B2
:106BC0000020904780BDC0467420004064400040D3
:106BD00098D20102783000409CD20102C0A001028C
:106BE0006AD4010280B50D48016889070FD50521D7
:106BF00001600B48C178002908D00021C170C1682C
:106C0000002903D0C26841680020904780BD054834
:106C100005A10B4A0BA308F0FDF8C0462C04004068
:106C200034940102D83C01005048595F54494D4505
:106C3000525F49525148616E646C657200000000F9
:106C40008D0A0000556E657870656374656420690F
:106C50006E746572727570740000000070B5044641
:106C6000401E012814D80320084011D13F204003C2
:106C70000818050B281980280AD8164E31780120EB
:106C80004840294604F0DEF8641E6D1C002CF5D146
:106C900070BDC04680B50020014603F01BFE0028F1
:106CA00000D080BD0B480121017080BD70B5164633
:106CB0000C460546FF22F9F76FFA054831180548DA
:106CC0000278012050402A46234603F063FF70BD3E
:106CD00000E0070430A901020120000370470120F1
:106CE00040037047F0B585B048484949016005F058
:106CF000CFFF484DE98A4A2247488152AA8A482351
:106D0000C252AB888362AC7A0471AC89C4810282BE
:106D10004182A98D0187049383864A1E91414900CF
:106D2000C161A88B3B2801D83C20A8830020E883C0
:106D3000288B3A490880FF20063068806C8C0F2031
:106D4000224602407D21C900260B4E43B61822057B
:106D5000170F64225743F6192406270F0A246743A6
:106D6000F6192F4F3E80AE8C374607402B46350B29
:106D70004D43ED1937053F0F5743ED193606360FD2
:106D80006643AD19274E3580DD8C2E4606402F0B0D
:106D90004F43BE192F053F0F5743F6192D062D0FF0
:106DA00065437519204F3D801D8D28402E0B4E43A5
:106DB00030182905090F514340182906090F61436E
:106DC00040181A4E3080032419A220462146049B05
:106DD00009F07CF80F484088C1B20091030A18A25C
:106DE0002046214609F072F80D4803880D480088B6
:106DF00039883288094D2D8800AE27C619A2204651
:106E0000214609F063F805B0F0BDC04600960102C6
:106E10003184000032A901028098010274960102B7
:106E20006C9601026E960102709601027296010242
:106E3000C9E8B1B849443A202578202E0D0A00004F
:106E4000B9CCBCFEB0E6B1BE3A5557422D3447B37B
:106E5000B5D4D8CAD6BBB7205625642E25642E20BB
:106E60000D0A0000B7FECEF1C6F7B5D8D6B73A2066
:106E700025642E25642E25642E25643A25642E0D66
:106E80000A000000F0B583B030480068C16B09010A
:106E9000890F01D003B0F0BDC16BC06B2C4D054014
:106EA0004800400F0826029686400227384602F026
:106EB000B7FD01907043C10B4A1B26485043F9F7B8
:106EC0001FF9044607F0E8FE032123A238461F4FAE
:106ED0000091234608F0FAFFF88A002817D001989D
:106EE00040012946F9F7F6F84643182232400120BE
:106EF0000F2A014600D8002173095B181B4CA342DE
:106F00000DD8194DED1A6D050F2A0CD80CE0386814
:106F10000021C160112002F073FD03B0F0BD5D1CC3
:106F20006D050F2A00D956422A0C029D2E400901F8
:106F30008919A34202D80098000400E04004081810
:106F400080183968086303B0F0BDC046C4940102DC
:106F5000FFFF1F0040420F0052434F33324B20705F
:106F6000706D2025640D0A00FF070000FE7F000001
:106F7000B0B582B0154908688269D2070CD00122E9
:106F8000C2610D69002D07D000686C46214607F0EC
:106F900023FC00212046A84702B0B0BDB0B582B0A6
:106FA0000A490868026C92070ED5026C012313434C
:106FB0000364CD68002D07D000686C46214607F0B9
:106FC0000BFC00212046A84702B0B0BDC4940102CA
:106FD00006480168032291430160016801220A43C7
:106FE000026000F043FB07F079FEC0462800004035
:106FF00080B50D490868002810D52248026804238E
:10700000032A01D01A4300E01A460A601E490A68A2
:10701000002A02D041680020904780BD03A00CA147
:107020009E2211A307F0F6FE2C100140696E636CDE
:107030007564652F647269766572732F6D6B5F730B
:107040006C6565705F74696D65722E630000000089
:10705000534C4545505F54494D45525F4952514844
:10706000616E646C65720000556E6578706563745E
:10707000656420736C65657020696E7465727275E5
:10708000707400000C90010270D40102B0B582B09F
:1070900004460078002811D0094D01A9087028681D
:1070A000416A0029FCD101A901220020034609F010
:1070B000CFFC611C607800280C46EED102B0B0BD58
:1070C000FC94010270B50C784D782D022C198D7846
:1070D000C97809024919090409198000094C21508D
:1070E0009178D47815785278074E3350074B069E26
:1070F0001E50120252192302591809048918044A11
:10710000115070BD949F010258E00102F4DF0102AA
:10711000F89F010210B5CE4C216806290FD8012036
:1071200002468A4058210A4209D020600020A0600F
:107130002369002B03D06269002002219847C348CD
:107140002258062A12D801210B4693405822134296
:107150000CD021502018002181600369002B05D03C
:10716000AD20C000225801200221984747482258EC
:10717000062A11D801210B469340582213420BD006
:1071800021502018002181600369002B04D003489E
:107190002258022001469847002010BDBC0A00007A
:1071A000F0B581B00024022803D9E443204601B0A1
:1071B000F0BD17460B46094E464309488519284637
:1071C00018302A2107A2FCF75BFF42202F52032030
:1071D00003498851204601B0F0BDC0465405000067
:1071E0005CAE010225730000F0B585B0E04D2C685F
:1071F000002C0CD0DD4FDE4CE659002E0CD0234F76
:10720000E659002E0DD00020C04305B0F0BD01AC02
:107210000FC400272E4608E001AE0FC6E61901276D
:1072200003E001AE0FC6E6190227D04C30462146D6
:10723000FCF70CFE022030607C432919029D4D6052
:10724000CF60039808610498486108464430CC3107
:107250000122560210233246FCF7EEFFE4480019E3
:10726000B32189004118012D05D1B83001233246E0
:10727000FCF7CDFB04E0743010233246FCF7DCFF52
:1072800001980760002005B0F0BDC046A80A0000C4
:1072900001460020022901D9C0437047E24A4A430F
:1072A000E24988507047C046022806D8E649414363
:1072B000E64840180249401870474B20800070474C
:1072C000D4040000022802D94B2080007047DE4918
:1072D0004143DE4840184D21090140587047C046DF
:1072E000032801DB03487047D7494143D74840187A
:1072F00018307047E53A0100022806DCD2494143C4
:10730000D24840184221405A704700207047C0467A
:10731000032801DB00207047CB494143CB4840188C
:1073200044307047022804DCC7494143C7484058ED
:10733000704700207047C046022805DCC24941431F
:10734000C24840184068704700207047B0B500241C
:10735000E14302280FD8BC4A4243BC4B9D58042D40
:1073600009D0991801220A600B69002B05D04A69DF
:107370000221984721460846B0BD2046B0BDC04610
:1073800010B50024022801D9E04310BDAE494143A5
:10739000AE4A0723535051180B69002B03D04A699A
:1073A000002421469847204610BDC046F0B581B064
:1073B0000024022803D9E443204601B0F0BD05466D
:1073C000A1486843A14906220A500F1838464430A4
:1073D0003946CC310122560210233246FCF72CFFED
:1073E000786801280CD1B320800039183846B830AD
:1073F00001233246FCF70BFB3B69002B0CD1DBE78A
:10740000B320800039183846743010233246FCF718
:1074100013FF3B69002BCFD07A690121284698479A
:10742000204601B0F0BDC04610B50024022801D9A5
:10743000E04310BD84494143844A51180B69002B35
:1074400002D04A6903219847204610BD5405000028
:107450005CAE0102F0B583B017460024E243022877
:107460001AD8002B18D00D46774941437748461863
:1074700070680128029312D1002F0AD0B836002478
:1074800029193046FCF7CBFA002825D1641CA74205
:10749000F6D1029807600022104603B0F0BD0192B9
:1074A00074363046FCF783FE002811D0034642684C
:1074B000BA4209D2196828461D46F8F75BFE2B46EA
:1074C000686802990860019430461946FCF745FE49
:1074D000019A104603B0F0BD0298046000221046E5
:1074E00003B0F0BDF0B581B004460020C343022CC8
:1074F00002D9184601B0F0BD15460E461B4A62433C
:107500001B498F187968012910D1002D28D01C46FD
:107510000090B83738463146FCF75AFA002821D196
:10752000761C6D1EF6D1009801B0F0BD0090743746
:1075300038462946FCF756FE00280CD00446006861
:1075400031462A46F8F716FE38462146FCF71AFE61
:10755000009801B0F0BD07A02146FCF7F7FA0098AB
:1075600001B0F0BD204601B0F0BDC046540500009A
:107570005CAE0102536F636B65745B25755D2052D1
:10758000656376204275666665722046756C6C0D83
:107590000A000000F0B583B0154607460022D0432C
:1075A000022F19D8002D17D000AB07C30F4878431E
:1075B0000F490E18443630462946FCF713FE0028C2
:1075C0000CD00446006801992A46F8F7D3FD3046EE
:1075D0002146FCF7D7FD029803B0F0BD05A039465F
:1075E000FCF7B4FA009803B0F0BDC04654050000A3
:1075F0005CAE0102736F636B65745B25645D207321
:10760000656E64206275662066756C6C0D0A0000FC
:1076100002460020022A04DC0B4B53430B4AD15094
:107620007047C0437047C046540500005CAE01027D
:10763000022801D9002070470349414303484018FC
:10764000034940587047C046540500005CAE010233
:10765000CC04000080B504480168491C0160006941
:10766000002800D0804780BDDCDF010201480249CC
:1076700001607047709001020026B80310B5C5483C
:107680000024446110300221024A2346FFF7ACFD7A
:10769000204610BD4977000070B584B0FDF73EF973
:1076A000012814D1FCF780FB204D6969022914D010
:1076B000002909D12978002921D0A969411A062970
:1076C00002D300212970A861002004B070BD1748C2
:1076D00000214161002004B070BDE969421A1449DB
:1076E000144B9B8B9A4202D20A78002AECD0E861B4
:1076F0000020087000F006F9002004B070BD0126DB
:107700006E61AB88E88829896A8900AC07C4B10238
:10771000094C0AA22046FCF7B3FC2869AA89214635
:10772000FFF73EFD2E70002004B070BD6896010288
:107730004493010232A9010248C5010225752E2594
:10774000752E25752E257500F0B58DB0032909D845
:107750007944097949008F4401070F155948416957
:1077600001290AD00DB0F0BD564841690129F9D16F
:10777000022141610DB0F0BD52480021416101700C
:107780000DB0F0BD002500954E4C20694E494F4A82
:107790006B46FFF75FFE0028E4D103204CA20146B0
:1077A00008F094FB48484DA10A22F8F718FD00287C
:1077B00012D045484CA10F22F8F711FD0028D1D175
:1077C00041482C2101AA0C23FCF76BFC0298FCF722
:1077D00041FB60870DB0F0BD3B482C2101AA0C2372
:1077E000FCF75FFC0498FCF735FB608780B2684EBD
:1077F000B1888142B6D10298FCF775FCE06203982B
:1078000001794279120251188279C3791B029A18C0
:10781000120451188278C378077840780002C019A2
:107820001B029A1812041018206261620598FCF776
:1078300011FBA0870698FCF756FCE0870798FCF739
:1078400052FC4027E0530898FCF74DFC422160545D
:10785000E16A491E062901D80122A270062926D80C
:107860007944097949008F440318111C221E150020
:10787000E08FB082E05BF082A08FB18D814216D0A4
:107880001E4902220A60B0851D4800E01A48012105
:1078900001700CE00120B08709E018480560B5854B
:1078A00005E0B58703E0C0B23C214143B18301202C
:1078B000A07000F027F807F073F925626562A570E3
:1078C0000DB0F0BD6896010248C50102FF0300003B
:1078D000CAD5B5BDCAFDBEDD0D0A000024696E73B0
:1078E00074727563742C0000246D65737361676531
:1078F0005F7265706C792C00AC9601029C98010255
:1079000038900102F0B5C7B0214CA0881490214DE9
:1079100068781390FBF7EEFE1290A08D11906878B6
:1079200010901D4800780F90A08A0E90E08A0D906C
:107930001A48C0C81A490A684968AB78194C2468C3
:107940002035089209910A950B930C941298009097
:1079500011980190109802900F9803900E9804903F
:107960000D9805A9C1C11398002801D00F4A00E065
:107970000D4A15ADC8212846149B09F09DFD02460D
:10798000044800692946FFF705FE47B0F0BDC04630
:1079900032A9010268960102889801021099010239
:1079A0000899010254990102F1310100B03101003E
:1079B00080B582B00E4908680022C2600192CA6890
:1079C000002A02D0016801A8904702B080BDC046DD
:1079D00080B582B0064908690022C2600122019286
:1079E000CA69002A02D0016801A8904702B080BD90
:1079F0001C930102F0B582B0144C2078009000284E
:107A00001DD0134B24330025019504E09B1C6D1CF5
:107A10000098854215D262196026905D471C9755E3
:107A20000928F3D80199C8B222181C88975540003C
:107A3000074A10188484054C491C0191E6E7002090
:107A400001900198207002B0F0BDC046309901024B
:107A50000C9A0102F0B589B009F052FCE94C60784B
:107A600009F0F4F9E8498A8807A882800A884988D9
:107A700009048918079105F08DF96078052804D06C
:107A80000222E249092804D104E00122DF49092841
:107A900000D0891849792078621C09F09BFA607A35
:107AA00006F0A0FCDA48DB4904F078FCDA4C2078D8
:107AB0000026002806960AD0D8491A31D84A03462B
:107AC00010CA0C80891C5B1EFAD14600D24CD54DE1
:107AD000A872D54800886871D449097829706178FE
:107AE000E970000AA871481C607028460B30CB4F23
:107AF00039464C3103913246F8F73CFB70190B3094
:107B000039461A313246F8F735FB2020687206985C
:107B10002071E0886870000AA870C3200690840174
:107B200006F0D0F90319BC48C362BB480078810055
:107B30000D3101222846059209F060FCB6498862A1
:107B4000B548C46A06F054F90019B34C06F0ACFD10
:107B500005460E46AB48007B06F032FC81B2C90BED
:107B6000401800B2C11740102818A0657141E165A6
:107B700006F0A8F9A06104F083FB0028FBD106F011
:107B8000A1F9E0617D2006010027384639463246DA
:107B900009F0E8FBA062677125460698040206F02A
:107BA00091F9297861434118A2480818421C01D173
:107BB0009F480818984C206306F084F96063216B95
:107BC000884204D39C4A8918884200D897E006F07E
:107BD00079F9606306F076F9E06104F051FB002862
:107BE000FBD106F06FF92062607902284FD001289E
:107BF0007DD100206071914D697A212971D1697917
:107C0000AA7912025118884A1288914269D187498B
:107C100009782A788A4264D16978AA7812025118C0
:107C2000A181E278002A40D02278002A0BD07B4B39
:107C30004C3300201C888C4204D09B1C401C824288
:107C4000F8D11046744CC0B2E081236EA16BA26DD6
:107C50007A4D2C46223400946F4C019102922946B1
:107C60001A311E352A46FFF72DFAE089E17888425D
:107C700008D34100694A5118A2894C23CA5221787D
:107C8000491C21700521654A11546C4824E00020EC
:107C900060710146324609F065FBA06206F012F9F8
:107CA000206206F00FF9A06121E04C205B4A1152DE
:107CB0000598207005201070236EA06BA16D2A46D8
:107CC000223200920190029129461A312A461E3230
:107CD0000020FFF7F7F928469621F8F764FA00200C
:107CE000208200200146324609F03CFBA062226B54
:107CF000606B51495118904200D365E767E7A06D6A
:107D0000E16DFBF7F5FAA770207800282FD04448E2
:107D10004C213D463C46414B05E0891C001DFAB212
:107D20006D1C95421AD25E5D002EF6D0761E5E5511
:107D3000A3000693F6B22246414CE650374B5E5AFA
:107D40005300404CE6527F1C334B9F7003683E4CFF
:107D5000069EA3511446314B541CDEE705922E4873
:107D6000C77007700497F8B2022806D228E0E778B7
:107D700005970497F8B2022822D30598441E0021E3
:107D8000069403E0491C069CA14219D02E4A1068B3
:107D90002C4B2B4F0FE0156050605D881E885E8075
:107DA0001D8060CF083F3E607D60641E121D9B1CDD
:107DB0003F1D002CE6D05568A842ECDC2846F4E7CD
:107DC00004980006059C10D062001E490398F8F73D
:107DD000D1F9A20012481C49F8F7CCF90F4A18480B
:107DE00002C81170521C641EFAD10B4883890C48DA
:107DF00000680090032015A2014608F067F809B05A
:107E0000F0BDC046C4900102801F0100C4A0010261
:107E1000050101001DEB0000B0960102009801026F
:107E200020D20102CEE90102A89801028498010241
:107E300001CF030000CF03000026B80370D3010276
:107E4000D4E801029CE9010238E90102BBF9D5BE80
:107E50004944A3BA25582CBEE0C0EB3A2025640D56
:107E60000A00000080B5002008F0AAFA80BD80B5A5
:107E7000012008F0A5FA80BDF0B581B003F040FD07
:107E8000164CE060A178002901D001B0F0BD217945
:107E90000029FAD10121217100281BD08D02281A56
:107EA000A168814216D0614E2F46A068305C2169DE
:107EB0008847A068401CA060681EA168814201DD5F
:107EC0000020A060E168A068022F03D3691A7F1E1A
:107ED0008842EAD10020207101B0F0BDF095010286
:107EE000B0B5294C2368002B07D0022B0DD0012BF5
:107EF00039D109F0D1F900F00FFC09F0ABF9236892
:107F0000022B1FD0012B18D02DE0204D28780028FF
:107F10002FD003201EA2014607F0D8FF00202870B2
:107F200009F0BAF900F06EFD1C4D287009F092F9C5
:107F300028780028E3D001202060194800214181E1
:107F4000012310E011480178002909D114494A8918
:107F5000531C4B81152A03D3012202700020488153
:107F600008F040FF2368032014A2014607F0AEFF8B
:107F7000B0BD0B48408914210B1A032009A2014609
:107F800007F0A4FFBBE7C0469C98010238900102AD
:107F9000BFAAC6F4CBD1CBF70D0A00008598010229
:107FA00030990102B5C8B4FDBDF8C8EBCBD1CBF711
:107FB000C4A3CABDA3BA25640D0A0000555742D711
:107FC000B4CCACA3BA25640D0A00000080B5054806
:107FD0000068022805D809F05FF9FFF73BFD09F0BA
:107FE00039F980BD9C98010270B50E250024284601
:107FF000214603F081FD0D20214603F07DFD012483
:10800000204608F0E5F804262846314603F074FDC2
:108010000920314603F070FD204601F047FBA20223
:108020000249034B204608F0D1FB70BDE0CD0102B0
:10803000050A010080B5032810D800290ED07C2243
:108040004243BF488018C268012A07D12030FBF79D
:10805000E6FC002801D00020C04380BD0020C043C2
:1080600080BDC046F0B589B00022D543032800D9B1
:10807000ABE00C46002900D1A7E00095216A072754
:10808000534DA9420EDC574DA9421ADD564A914282
:108090002FDC4B22D501A9423ED0120291424BD196
:1080A000042246E04B4A914217DD4B4A91422ADCBA
:1080B000E1221203914231D0494A91423CD10C2233
:1080C00037E04B252E01B14233D06A01914227D0CF
:1080D000AA01914230D102222BE0E1225502A942AD
:1080E00020D09502A9421FD0D202914224D1092268
:1080F0001FE04B225202914218D0E122120291421B
:108100001AD1062215E0E1225203914210D0334ADF
:10811000914211D10D220CE003220AE00A2208E06C
:10812000012206E0072204E0082202E0052200E026
:108130000B22D1002D4A57587C214143804A505090
:1081400056182068B0606068F060A1683161E2682C
:108150007261002505950323049303950295019709
:108160000695079501231B020893012807D00028D4
:108170000AD18818009A8018B161F06104E0304695
:1081800020300123FBF743FC206970636069B06312
:10819000E069B067A069F063706801A908F042FA6D
:1081A0002068012806D830464030234610330ECBD5
:1081B000FCF742F86068012807D1301D703600686E
:1081C00001220B4B314608F001FB284609B0F0BDF7
:1081D000FFC10100FF0F0E00FF1F1C0080841E0066
:1081E00040420F007F250000FF950000B01F0100F6
:1081F0001D0A0100B0B50C467C214843504A1518B1
:108200002846FBF723FE6C600020B0BDF0B583B0BC
:108210000024E743032800D98EE00E46002900D150
:108220008AE01546002A00D186E07C21414344487B
:1082300041188868022832D001283AD000282BD172
:10824000EFF31080C00702D1EFF3108072B60291F5
:108250000846403001902946FBF7C4FF002863D050
:10826000014601980F46FBF78DFF386831462A46D4
:10827000F7F780FF0198FBF79AFFEFF31081C9072A
:1082800003D1EFF3108172B662B602994D6806C849
:108290002C4B284608F0DCFB204603B0F0BD4868B4
:1082A000002431462A46234608F0D2FB204603B07C
:1082B000F0BDEFF31080C00702D1EFF3108072B66B
:1082C00002910846403001902946FBF78BFF0028B9
:1082D0001ED0014601980F46FBF754FF386831461F
:1082E0002A46F7F747FF0198FBF761FFEFF310818C
:1082F000C90703D1EFF3108172B662B602994D68D7
:1083000006C8104B284608F0A3FB204603B0F0BD7A
:10831000EFF31080C0070FD1EFF3108072B662B692
:108320003C46204603B0F0BDEFF31080C00703D1F8
:10833000EFF3108072B662B63C46204603B0F0BD43
:1083400058BE0102210D0100B0B582B0602833D0C3
:10835000622843D0642854D101A82F490180EFF34B
:10836000108072B600242046214602F0B3FA2B4D4D
:10837000002805D1012002030020294602F004FA5A
:10838000103501AA02232046294602F0DBFE62B620
:1083900023A0FEF77BFE64201B490C5206F000FC74
:1083A0001A4801F00DFCBFF34F8F194819490160BD
:1083B000BFF34F8F00BFFDE76020134900220A5230
:1083C00006F0EEFB114801F0FBFBBFF34F8F1048A6
:1083D00010490160BFF34F8F00BFFDE762200A49DB
:1083E00000220A520A8006F0DBFB084801F0E8FB95
:1083F000BFF34F8F064807490160BFF34F8F00BF9F
:10840000FDE702B0B0BDC04632A90102A08601005E
:108410000CED00E00400FA05AAAA000000D0020456
:10842000BDF8C8EBC9FDBCB6C4A3CABD0D0A0000A7
:10843000F0B5D1B0A74EA8490A78002A25D0F28B12
:10844000002A22D1A54FBA68082A00D990E09300EB
:1084500001A4E3589F46C0467D840000718500005A
:108460007185000081850000AB850000B5850000A6
:10847000BF8500008F850000C9850000552800D009
:10848000BBE00120B86051B0F0BD4978002900D1AF
:10849000B7E0924D6A7996498854A979A871E97133
:1084A000521C6A710A2800D0ABE00D2900D0A8E068
:1084B00003A8019037A800902C4630348C488D4991
:1084C0001DAB2246F7F7A8FEE8608BA105222046E7
:1084D000F7F785FE00282AD1F08B002805D003206D
:1084E00087A2834B014607F0F1FC1DA8002421461A
:1084F00009F0ABFCA861E961824B2246F8F7D8F994
:10850000002814D1804800F0F7FF1DA80024214660
:1085100009F09BFC2862696237A8214609F095FCA6
:10852000A862E96203A8F7F709FF286100E028695B
:1085300000266E71002806D0744806707448012128
:108540000170744806806A489621F7F72CFE1DA832
:1085500064242146F7F727FE37A82146F7F723FEC4
:1085600003A82146F7F71FFE6E71EE8051B0F0BDF3
:10857000AA2838D1012A36D10220B86051B0F0BD06
:108580000421B9600021B970787051B0F0BD39791B
:10859000534A5054481C38717978491FC0B28142FF
:1085A0002FD10820B86051B0F0BD0522BA608870A4
:1085B00051B0F0BD0621B960B87051B0F0BD0721CF
:1085C000B960387051B0F0BD7A78062A02921AD399
:1085D000531F0025424A2C46565DA419A4B26D1CB7
:1085E0009D42F9DB10E0032807D1022A05D10120C2
:1085F000F8700320B86051B0F0BD0020B870B860CA
:10860000787051B0F0BD00242018029A8218887842
:108610001118BD7849193C780919FA78002A00D058
:10862000C91C2C4EC9B2FF2935D1012809D0022816
:1086300031D11E2D36D1FFF7D7FC0120F08351B088
:10864000F0BD284A9471032010719070AA205070D8
:108650005520107068085071651DD57040003118A4
:108660001646D01D2246F7F785FD301DE11CEAB203
:10867000D21C037892B2D218401C491EF9D1A0191D
:10868000D143C171090A0172093401200023314626
:10869000224608F0DDF90020B870B86038717870B3
:1086A00051B0F0BD70190E4E31462246F7F762FD0B
:1086B0003078012802D12846FFF746FE06F070FA0E
:1086C000BFF34F8F084809490160BFF34F8F00BFC8
:1086D000FDE7C04632A9010218900102E8980102A4
:1086E0007CCD0102DC9A01020CED00E00400FA05E9
:1086F000E4CC01024D310100474E474741000000E4
:10870000257300000000F03F99AD01022C94010296
:10871000AF9601029AAD0102F0B589B008F0F0FD04
:108720009A489B4903F03AFE9A4E00243471F47043
:1087300005F0C8FBF061042003F06AF9964D6A6801
:1087400020460694214608F00DFE05F0BBFB0446CA
:10875000306327204101686848430A21F7F7BAFCD3
:1087600070630119481C00D00846B06305F0AAFBED
:10877000F063B16B894C884202D30919884233D91E
:10878000874F884D05F09EFBF06303F079FD0028CC
:108790000AD0FCF781F805F095FBF063B16B8842D5
:1087A000F3D909198842F0D2F07801280FD138782E
:1087B0002978814211D1787A20280ED17879B97937
:1087C000090208187849898D884206D133E0724839
:1087D00042680020014608F0C5FDB16BF06B88428D
:1087E000D0D309198842CDD80125284601F0E8F9EF
:1087F000284608F0E1FD3079002816D16B4806F0D4
:108800004FFA6F4C2378032077A2014607F05EFBF6
:108810002078411C2170062807D379480221016085
:108820000698207070815C480570042003F0E0F821
:10883000002009B0F0BD012030715C48623006F0C4
:108840002FFA05F03FFBB061B87AB0700246059090
:108850007879B97909020C18F48039460B31550042
:10886000534802912A46F7F785FCE919059F0B3119
:108870004F4832302A46F7F77DFC002F069872D019
:108880004948808904904B4803680025484A03936F
:1088900026E0B11860230027CF545100464A5118F2
:1088A0008C8400B2F8F742F83A46444BF7F7DAFE08
:1088B00008900791706AF8F739F83A463F4BF7F796
:1088C000D1FE02460B4608980799F7F719FEF8F70C
:1088D00093F87062059F364A039B6D1CBD4227D0FA
:1088E0006800115A8B42F8D11118488E049A8018EA
:1088F0004886317800290ED02F4B243300221F8860
:10890000A7420DD09B1C521C9142F8D10B460A463F
:10891000172908D9BDE700231A46172903D9B8E754
:10892000D3B21729B5D88B42B3D1491C3170B0E707
:10893000002F0FD01F4801680020029C2278637826
:108940001B029A18914207D0A41C401C8742F5D103
:10895000384608E0002006E0C4B22046FAF746FC9C
:10896000B078A04201D1FAF741FC1548002101700E
:10897000052030560C498B8D716A009101900320BF
:1089800010A2014607F0A2FA2EE7C046DD00010062
:1089900075EA00003099010238900102007C31250F
:1089A000D8D201028498010232A901021A3F0000C4
:1089B000649A0102A89801020C9A01020000E03FAB
:1089C000D6D20102B1EAC7A94944A3BA25582CBEA0
:1089D000E0C0EB3A20256420D0C5BAC5C7BFB6C8F1
:1089E000A3BA25642E0D0A00B2E2BEE0CAA7B0DC2D
:1089F000A3ACBCC6CAFDA3BA25640D0A00000000E2
:108A00009C980102F0B587B008F07AFC904C607831
:108A100008F01CFA8F498A8805A882800A8849884C
:108A200009048918059104F0B5F96078052804D087
:108A300002228949092804D104E001228649092833
:108A400000D0891849792078621C08F0C3FA607A4E
:108A500005F0C8FC8148824903F0A0FC814C002647
:108A6000E67005F02FFAE061042002F0D1FF7E4DA0
:108A70003046049631462A4608F074FC05F022FA86
:108A80007A49206361634118481C00D00846A063FE
:108A900005F018FAE063A16B754E884202D389197C
:108AA000884234D9734F03F0EBFB00280AD0FBF760
:108AB000F3FE05F007FAE063A16B8842F3D9891948
:108AC0008842F0D205F0FEF9A061E07801280FD1CC
:108AD00038786949097881420AD1787A202807D103
:108AE0007879B979090208186449898D88421CD0BF
:108AF00005F0E8F9E061002001462A4608F032FC62
:108B0000A16BE06B8842CED389198842CBD801256E
:108B1000284601F055F8284608F04EFC049C042035
:108B200002F066FF204607B0F0BD554806F0B8F8E1
:108B300005F0C8F9A061B87AA07002460290787971
:108B4000B97909020D18E58039460B3156004D48B8
:108B500000913246F7F70EFBF119029F0B3149489D
:108B600032303246F7F706FB002F62D046480368E2
:108B70000026444A019326E0A11860230027CF5421
:108B80005100424A51188D8400B2F7F7CFFE3A46A1
:108B90003F4BF7F767FD04900391606AF7F7C6FE55
:108BA0003A463B4BF7F75EFD02460B4604980399A5
:108BB000F7F7A6FCF7F720FF6062029F314A019B9E
:108BC000761CBE4224D07000115A8B42F8D1101886
:108BD000408E217800290ED02C4B243300221F8890
:108BE000AF420DD09B1C521C9142F8D10B460A4655
:108BF000172908D9C0E700231A46172903D9BBE76C
:108C0000D3B21729B8D88B42B6D1491C2170B3E72B
:108C1000002F0ED01C4801680020009D2A786B7838
:108C20001B029A1891420AD0AD1C401C8742F5D114
:108C300000E000273846FAF7D9FA01246FE7C5B2F9
:108C40002846FAF7D3FAA778AF42F3D0012466E7B3
:108C5000B6900102861F0100C4A00102DD000100E0
:108C600075EA00003099010280841E000098E00E31
:108C7000007C3125D8D201028498010232A9010278
:108C80005C3F0000649A0102A89801020C9A01025C
:108C90000000E03F80B582B0002001900448C26827
:108CA000002A02D001A80021904702B080BDC04632
:108CB0008C950102F0B583B000242046FDF7EAFF51
:108CC000FEF70DF8274EB060FEF706F87060264FED
:108CD0000BE001A8C1888088084319D101A8408809
:108CE00024180834B068844235D201AD08212846E2
:108CF0002246FDF7DBFF28880028EAD0B8422AD0B8
:108D000001AD0421284600F045FFA9888842E5D03E
:108D10003460B06884420CD201AD0221284622465C
:108D2000FDF7C4FF2888B84203D0A41CB068844271
:108D3000F2D370682118491E4042084030600DD0BF
:108D40000024254601202946FDF788FF03CE4D1952
:108D5000083E8542F6D3346003B0F0BD0024346091
:108D600003B0F0BD18970102FFFF000010B5054CDD
:108D70006070FEF7C7FD6078022801D100206070A6
:108D800010BDC04668960102F0B585B01F4604923A
:108D90000646C8170C1844400A2C039114D3012529
:108DA0000A212046F7F796F96D1C632C0446F7D884
:108DB00004998D4200D329460A9C002F09D00398BC
:108DC000002808D4002207E0012504998D42F2D240
:108DD000F2E7002205E00122042323409B0813430D
:108DE000FA1A0223234004980028029412D1002B7F
:108DF00010D0F468002C62D40398002825D402987F
:108E0000400734D57068B5686F1C87422FD830682A
:108E10002B2423E0E407ECD1002A0AD1E9E73768E4
:108E200020203855B560F068441CF460521E002CB8
:108E3000DFD49142DDD27768B468651CBD42EED9BB
:108E4000F468521E002CF4D5D3E7404203907068BA
:108E5000B5686F1C87420AD830682D244455B76026
:108E6000F068441CF4600025ED43A84227DB002B8A
:108E70001CD00120029B1840049B184316D1002AE5
:108E800003D113E0521E002C0ED491420CD2706814
:108E9000B3685D1C8542F5D830683024C454B56091
:108EA000F068441CF460EDE7002C08D400920298AE
:108EB00001900A2230460399049B00F003F805B0A4
:108EC000F0BD0000F0B587B01F46154602900124A2
:108ED00006919142009407D3012406982946F7F79A
:108EE000F9F8641CA842F9D20D980C9ABC42039779
:108EF00000D3039400990140002A009109D0002971
:108F0000029C25D12021800705D40846002F11D0CE
:108F100004E0029C1CE03020002F0BD0084609E042
:108F200023685854A260E168491CE1603246721E11
:108F300000290DD4039991420AD216466368A168AC
:108F40004A1C9A42ECD9E1683246721E0029F1D5DA
:108F5000E068002859D40590012401E07F1E6C438D
:108F6000022FFBD2069821461646F7F7B3F8324691
:108F7000A842F4D2029880680490069F0195069753
:108F800038462146F7F7A6F8049D691C029F7A68C7
:108F9000914206D9069F059A019D0592002A0ED599
:108FA00016E01B4A125C3B685A55B960FA68521CBD
:108FB000FA600491069F019D0592002A08D460433F
:108FC0003F1A20462946F7F785F8AC420446D6D228
:108FD00000980028029C059B049D16D0002E14D0FA
:108FE000701C01E0002B10D4401E039981420CD26A
:108FF000691C62689142F5D8226820235355A1600C
:10900000E268531CE3600D46ECE707B0F0BDC046D4
:109010008C220100F0B583B001900291002923D089
:109020000025124F2E460AE013480818410F401839
:10903000C0103872761CB0B20299884214D20198DE
:1090400000884B24210100B200F018F840006101B3
:109050004018F88201B2064881422846E9DB0548FB
:109060008142E1DD6420E4E703B0F0BD80980102B5
:10907000E40C0000041000001CF3FFFF074A9042BC
:1090800001DD054A801800B24143C817400D081899
:10909000C00A00B27047C04600F0FFFFFF070000A3
:1090A00010B50078012819D1AC480269012A04D111
:1090B000614A13680124A3431360032905D080216A
:1090C0004161C269002A05D107E001214161C269FD
:1090D000002A02D001898069904710BDFF222E32FC
:1090E000024803A107A305F095FEC046402E0100EB
:1090F0006164635F646D615F63616C6C6261636B2B
:1091000000000000556E65787065637465642064C6
:109110006D61206368616E6E656C0D0A0000000071
:10912000F0B58DB00D460124EFF31081214002D13E
:10913000EFF3108372B6894E73690F2B06DD102B87
:1091400037D0402B2FD0802B2DD005E0002B2AD0FC
:10915000012B01D110237361B5813581B061F261BA
:10916000002900D162B63179002929D00294304C0F
:1091700005A90A4604950390E8CCE8C2E8CCE8C209
:10918000029C204600F08CFD2A4800902A4D29467A
:1091900008312046039A049B00F0F2FD2C60002465
:1091A00020460DB0F0BD0029FAD162B620460DB0C0
:1091B000F0BD02240029F3D162B620460DB0F0BD07
:1091C0003178002907D01C48072181610460002400
:1091D00020460DB0F0BD3269B3891749002B15D078
:1091E000B5693089012A02D0002A03D003E09FB27A
:1091F000874200D10C604F68FF07FCD08F6880C5A4
:109200005B1E1F04EED10023B381B561012A02D198
:109210000A68A2430A607461F2690024002ABFD080
:10922000B36931898800181A904720460DB0F0BD07
:10923000CC220100A190000008D00140F0B581B01F
:10924000002856D00446424EF068800754D41325B7
:10925000284600F0DDFB284605F0B0FA2768616873
:10926000012538462840CA07920F1018227C1207A1
:10927000120E8018627C1207120D8018A27C120751
:10928000120C8018627D13071B0AC01812091206FF
:10929000801830607D2006020029304600D12D481C
:1092A000E3681A0A7D2A1A4629D22B4EB3422AD2E3
:1092B00000292BD0002A2946254E00D01146F6F76A
:1092C00009FF401E80B2706024480761E27C027092
:1092D000237D0371224F3E686902A468012C1BD0D4
:1092E0002C0226433E60002B1ED00121184A116338
:1092F00029E0012001B0F0BD022001B0F0BD3246EE
:10930000154EB342D4D333460029D3D11A46002A8E
:1093100029460F4ED2D1D2E73F242401A643761826
:10932000F0363E60002BE0D1002A0CD0FF22120262
:109330000C4B1C6894430122D203A2181A60304AD5
:109340001160304A116001214161002001B0F0BD7F
:1093500000D001400026B80380841E00A0950102C1
:109360002C06004008E400E070B5002801D0012080
:1093700070BD0C461625284600F04AFB284605F02D
:109380001DFA002C05D01B48183014222146F6F790
:10939000F1FE28211748415C002915D041680029B9
:1093A00016D403220B469343144A9C588D07ED0EA6
:1093B000FF26AE40B4439C501F220A400121914039
:1093C0000F4A11600F4A116001210161002070BD38
:1093D0008A07D20EFF2393400F220A40083A032146
:1093E0008A43054954589C4354500121016100208F
:1093F00070BDC046749001021CED00E000E400E086
:1094000080E200E000E100E080B5684800210170E2
:1094100061480078C00161490978890101436048C9
:109420000078400108435F490978090101435E481B
:109430000078C00008435E490978490001435D484F
:1094400000780843C0B2FBF763F980BD80B5574888
:10945000012101705148007880014F490978C90104
:1094600001434F480078400108434E4909780901FB
:1094700001434D480078C00008434D490978490030
:1094800001434C480078084304210143C8B2FBF76C
:109490003FF980BD5A21014A505270475CA0010239
:1094A000F0B581B013490A78002A13D0052A01D1FA
:1094B00004220A709300CD18561C00231C462F6806
:1094C0006F60F917DB194C412D1F761E012EF6DC5B
:1094D000084902E00022134614464860521C0A70F4
:1094E000C11718186141D2B20023F6F71DFE01B072
:1094F000F0BDC046C0950102F0B581B004460078C9
:1095000041424141217024480078C0012349097833
:109510008901014322480078400108432149097824
:109520000901014320480078C00008431F4F3978E3
:10953000890001431E4D2878400008431D4E3178B4
:109540000143C8B2FBF7E4F87D20C00000F038FB0F
:1095500020784142414121700F480078C0010F49F5
:109560000978890101430E480078400108430D49FC
:109570000978090101430C480078C0000843397894
:109580008900014328784000084331780143C8B27C
:10959000FBF7BEF801B0F0BDE09E0102AE960102FD
:1095A0001D90010264EA010299AD0102E19E0102EF
:1095B00024A3010225A30102B0B5094D28600224AD
:1095C000002120460A4602F02BFA012105222046FE
:1095D00002F0BAFA2A680321204602F099F9B0BDD8
:1095E000DC9E01025C219D480022425282847A2145
:1095F00041840284C2830283C28202821149416093
:109600008260C2603D21490441834182090C81830B
:10961000818270475C2191480022425282847A21E3
:1096200041840284C2830283C2820282054941606E
:109630008260C2603D21490441834182090C8183DB
:10964000818270474C37373770B585484C210160AF
:1096500001252C02601C00F05BF9322000F0B0FA0A
:1096600000F044F9284600F04BF9284600F05AF87B
:1096700000F036F90C4800F04BF900263046314630
:1096800000F056FA2846314600F052FA204600F023
:109690003FF9022000F03CF94834204605F032FB47
:1096A00005F090FB70BDC0460102000010B50446F5
:1096B000072106F069FA0148046010BD60960102B6
:1096C00070B505200424214602F016FA0620214632
:1096D00002F012FA0A20214602F00EFA0920214671
:1096E00002F00AFA00240121204602F005FA0225C0
:1096F00020462946224602F027FA0B26304621460C
:10970000224602F08DF930462946224602F01CFA24
:1097100070BD00000248016801229143016070475A
:109720005800004002490A6802408242FBD170475B
:1097300004600040B0B5494D28688107484C0ED5FB
:1097400028797F21084022688A4310182060236806
:109750000B4002200321434A06F0B8FB286880042E
:109760000ED55E20285C7F21084062688A4310186D
:10977000606063680B40022003213B4A06F0A6FBB1
:10978000172000F045F93948016802220A430121F7
:109790008A43026036483749016037480021C17169
:1097A00081791F2529408171817A427C837C1B024B
:1097B0009A18C37C1B04D218037D1B06D2182F4BAA
:1097C0009A4218D1427B837B1B029A18C37B1B04ED
:1097D000D218037C1B06D218294B9A420BD1C27AAD
:1097E000037B491E122906D819028918254A91427D
:1097F00001D1202101720178CA0602D11022114341
:1098000001701C3C20682021884320601E481F49AD
:10981000016041680029FCD503F020FA04460220CB
:1098200003211BA2234606F051FB0A20C441032C4E
:1098300005D8022003211DA206F048FBFEE71848C8
:10984000C1680F229143C1600168164A0A40026054
:1098500019200001144948600D60B0BDC4A0010288
:1098600048000040882E0100722E010004020040D2
:109870000C060040AF6B100A6B0001404D383650AB
:10988000312E32360734000000600040FE1C00809C
:10989000436869702049443A20253038780D0A0021
:1098A000C8600040FEFFC3FF0C0400404F6C642002
:1098B00063686970206D6F64656C206973206E6FDA
:1098C0007420737570706F7274656420627920748F
:1098D0006869732053444B2121210D0A00000000C8
:1098E00080B5172000F08CF8002080BD10B517243B
:1098F000204600F08DF8204604F060FF002010BDE7
:109900000121C90701430148016070470060004020
:1099100010B5C1B2000AC2B202290CD0012913D07D
:10992000002930D1911E7F4802291BD20121032A30
:109930002AD0490429E07B484168002A1FD002460A
:10994000203A1143416010BD76480168D31E022BB6
:1099500010D3012A29D0002A41D101229207914334
:10996000016010BD002A16D10121490702688A430F
:10997000026010BD0123042A1FD05A041EE00122F8
:1099800092079143416010BD0904194A7F32C36AAE
:1099900013405918C16217498A699207FCD5012101
:1099A000490702680A43026010BD0522120791436D
:1099B0000246203A0A43026010BD1A04836A0C4C26
:1099C0001C40A21882620B4A131F00241C600A4B21
:1099D0000A4C1C600D235B0214681C431460054A8A
:1099E00093695B06FCD5052212071143016010BD87
:1099F00080FFFCFF1402004004010040FF0F000044
:109A000001218140474802688A4302607047C0468E
:109A100001218140434802680A4302607047C04602
:109A200010B5052811D8C046784400794000874415
:109A3000020E192434393B490A680868C0003CD535
:109A40003A4820390A425DD03BE0002010BD35493C
:109A50000A680868C00035D534480B46203B1A42D6
:109A600037D134E02F490A680868C00036D52F483E
:109A70000B46203B1A424CD135E02A494C68012064
:109A8000C0030A680B46203B1C421AD00C68E40055
:109A90003BD5264C1A423CD03AE0224800680120CF
:109AA000C00310BD1F490A680868C0001ED51F48C2
:109AB0000B46203B1A4220D11DE01B4820390A42A8
:109AC00020D010BD18480B46203B1A4201D101207E
:109AD000C00349688900890FC84010BD12480B4671
:109AE000203B1A4215D10120C00312E00E480B465C
:109AF000203B1A4201D10120C00349680903890FA4
:109B0000C84010BD0120C00310BD074C1A4200D050
:109B100020464A689200920FD04049680901890F97
:109B2000C84010BD20000040006CDC020026B803D5
:109B300004282CD8164AC04678440079400087444F
:109B4000020A121A210003200007136883438807C2
:109B5000800818181AE003208006136883438807DA
:109B60000009181812E00320800413688343880753
:109B7000000B18180AE0FF20000213688343080254
:109B8000181803E01068FF239843401810607047CE
:109B900024000040B0B5002200290CD0074B047807
:109BA00095B22D0A65406C001C5B12026240491E92
:109BB000401C0029F3D190B2B0BDC0468C200100FA
:109BC00000280AD030B407252C02CD256419604343
:109BD00040091238001FFDD830BC7047F0B583B083
:109BE0001F4616460D460146E8680291F6F70CFC42
:109BF00004460F2E11D8082E04D320462146F6F72E
:109C0000AAFB09E0042E02D38120C10501E0412016
:109C100001062046F6F7F8FB04460999089E2B201A
:109C2000C043874205DB20460F462146F6F793FBEB
:109C30000DE03F20C04387420BDA4920C0438742F2
:109C40000CDBFF200F4681052046F6F7DDFB394689
:109C50000446688A0880346003B0F0BD0191532047
:109C6000C043874206DB20462146F6F774FB0446D4
:109C7000688A10E0A8690299F6F7F0FD002801D182
:109C8000A88B00E0E88BF6F74AFE01462046F6F77F
:109C9000BBFB0446002001990880346003B0F0BD8E
:109CA000F0B581B005460120072D66D80C46002985
:109CB00063D04A4F38680169C90736D10526304656
:109CC000FFF7A6FE304604F079FD03CF03690122B9
:109CD00013430361002918D403200B4683438E48A5
:109CE0001E588807C00EFF278740BE434027874085
:109CF000374389481F501F20084082408748026030
:109D000087480260354800680FE08A07D20EFF26B8
:109D100096400F230B40083B03218B437D495F583E
:109D2000B743402696403E435E50690140180121EA
:109D300009024218E369DB069B0CA569ED00EDB250
:109D4000EB18536062685207520B23685B075B098C
:109D50009A18A3685B079B0CD218E3685B075B0D3E
:109D6000D21823695B01DBB2D21863699B07DB0E53
:109D7000D218802313434350002001B0F0BDC046E9
:109D8000F0B581B0002A23D005460835134C26686B
:109D9000F668EE40F50702D0022001B0F0BD069D46
:109DA0008600A619B560400124682018009301239D
:109DB0001D02461977680724A7437760F160326176
:109DC0000099B160415919434151002001B0F0BDE3
:109DD00003A00AA174220DA305F01CF8D49201027D
:109DE000696E636C7564652F647269766572732F32
:109DF0006D6B5F646D612E6300000000646D615FD8
:109E00007472616E7366657200000000496E76615F
:109E10006C6964207472616E736665722064737419
:109E200020616464720000000001584908584068CD
:109E30007047C046F0B581B005460120012D4CD8D1
:109E40000C46002949D0002D03D0012D04D10F204C
:109E500000E00E20FFF7DCFDA668012E04D0002EE6
:109E60004FD1E08900284CD12901294843580020CE
:109E7000D860F507AD0F27686668B607360F761904
:109E80002569EA07920EB618022F04D0012F03D1DC
:109E90000122164300E040361D4F9E60E2681A60C2
:109EA00079188D606269CA604968002917D4032255
:109EB0000B469343184A9C588D07ED0EFF26AE4083
:109EC000B4438026AE4026439E501F220A40012103
:109ED0009140124A1160124A116001B0F0BD8A0728
:109EE000D20EFF2494400F230B40083B03218B43E9
:109EF00008495D58A543802494402C435C5001B030
:109F0000F0BD08A00FA1492212A304F083FFC046B0
:109F10001C9301021CED00E000E400E080E200E0A0
:109F200000E100E0696E636C7564652F64726976A8
:109F30006572732F6D6B5F6475616C5F74696D65BD
:109F4000722E63006475616C5F74696D65725F6F1A
:109F500070656E00636F6E66696720697320696E55
:109F600076616C69640000000001084A10580160C5
:109F7000816880220A4382607047C046000103491D
:109F80000858816880229143816070471C930102C8
:109F9000F0B58DB0019315460E460A901298002434
:109FA00008900480149F3C801398099004601598D1
:109FB00004900480FF2081053046F6F725FA0290D0
:109FC000304603963146F6F7C6F92B463D460690D5
:109FD000274607950B9311E01180188880002858B8
:109FE000099908600120079D2880052004990880B0
:109FF0007F1CBCB21888844200D9A0E028880028C1
:10A00000F6D1A0000A9D2E5830460699F6F718FCA6
:10A01000002817D030460399F6F712FC00280B9B56
:10A02000079DE5D1089A1780099D2E601888011BAD
:10A03000012934D11080198889000A9A5158296061
:10A04000059035E0089A1780099806600B9B1988DF
:10A05000081B0128C0D00C96019825187E1CB0B2B0
:10A060008542BFD389B2B2B28A420ED880000A9923
:10A070000C5820460C99F6F7D5FB0B9B002804D111
:10A0800009980460089806800C94761CB0B285424A
:10A09000A8D3198889B2B2B28A42E7D9F5E70C96FB
:10A0A000019962187D1CA9B216468A4205972CD2E6
:10A0B000059884B2A5000A9E7259002C104609D05A
:10A0C000A819001F016810460C92F6F744F90C9A83
:10A0D000062C07D80446A81941681046F6F73BF944
:10A0E0000C902046079D0299F6F7B8FB00280B9BC1
:10A0F00007D10C980299F6F7A3FB0B9B002800D020
:10A1000076E701202880032070E780B2AAB282425D
:10A110000FD888000A990C5820460C99F6F782FB54
:10A120000B9B002805D109980460089805800595C7
:10A130000C946D1CA9B28E42BAD31888E5E70DB015
:10A14000F0BD00000A490A680A4802400A60FD2181
:10A150004900094A1268515C002908D007490A6C75
:10A1600002400A64012000060A6882430A607047C0
:10A1700000040040FFFFFF7F4494010220000040E4
:10A1800000207047F0B583B00D4604467C26464358
:10A1900050488719F869396AF5F79CFFA84200D83A
:10A1A00092E0019502940121EFF31080084002D162
:10A1B000EFF3108272B63C4610343B690025062B43
:10A1C0000CD80A469A40D3065B0F06D161231A4287
:10A1D00075D00D46002803D003E00225002800D1E9
:10A1E00062B6002D02D0284603B0F0BD00943C4674
:10A1F0002034384880591021C1613E46143604F09D
:10A20000DBFD05463868C069C00605D504F0D4FDFD
:10A21000401B31888842F5D90621029D284600F06E
:10A220000BFF206801994143B869091838688160BB
:10A23000172179563C461734002909D5C1692022D7
:10A240000A43C2610121F966890502680A43026076
:10A250000521284600F0F0FE207840B200250028B5
:10A26000C1D42B4800687D24E100F5F733FF61017C
:10A270004143029800F0B2FE04F09EFD04463868A7
:10A28000C069C00705D004F097FD001B31888842E3
:10A29000F5D904F091FD04463868C169890706D5EF
:10A2A00004F08AFD001B31888842F5D93868012105
:10A2B000009A116053498161284603B0F0BD032123
:10A2C000216000288CD08CE7034804A1084A09A328
:10A2D00004F0A0FD48930102B82E0100666C617382
:10A2E000685F626C6F636B5F65726173650000002D
:10A2F0005D020000626C6F636B2069647820697393
:10A30000206F7665722072616E67650D0A0000002D
:10A31000F0DF0102F0B583B002907C214143934A03
:10A320005418E56EEAB2511E02291FD229040126F3
:10A33000090E18D001960092022100F07DFE2746FA
:10A34000143704F039FD06462068C169890606D431
:10A3500004F032FD801B39888842F5D92068007DE1
:10A36000C007019E08D0304603B0F0BD032A36D1A5
:10A3700000922804000E36D020466C302D0C0021AF
:10A38000019101602746143704F016FD0646206847
:10A39000C069C00705D004F00FFD801B39888842D2
:10A3A000F5D904F009FD06462068C169890706D57C
:10A3B00004F002FD801B39888842F5D920681149D4
:10A3C0008161E9B20120002911D003290099019E81
:10A3D00000D006202061226F002A0ED1C3E700269C
:10A3E000304603B0F0BD0126304603B0F0BD009901
:10A3F000019E2061226F002AB5D002A89047304606
:10A4000003B0F0BD000093EB70B5002801D001202F
:10A4100070BD7825CD4E705D00280ED00024092136
:10A42000204600F009FE0F20FFF7CAFB1520FFF7BA
:10A43000E7FA74553461204670BD042070BDC046F3
:10A44000F0B581B00C460078484EF16881422CD1BD
:10A45000032C54D1706EB16E884261D9002406215C
:10A46000204600F0E9FD3068F16D8160204621460C
:10A4700000F0E2FD354660352CCDF0683168B48CD3
:10A48000414F00975B1BA34200D81C46A308143120
:10A49000FFF776FCB06E0019B066306E00193066BA
:10A4A000F06D0019F06501B0F0BDB168814255D181
:10A4B000032C45D1F08CF16D0918F165316E091846
:10A4C0003166B16E0818B066716E814238D90024C9
:10A4D0000621204600F0B0FD3068F16D8160012159
:10A4E000204600F0A9FD316EB068F38C3268264C2E
:10A4F000009414329B08FFF743FC01B0F0BD3068B4
:10A500001021C16104F058FC05463068C069C006DE
:10A5100016D504F051FC401BB18A8842F5D90FE0F2
:10A5200030681021C16104F047FC05463068C069FD
:10A53000C00605D504F040FC401BB18A8842F5D91D
:10A540000120C107326813688B431360F16E220447
:10A550000A4300021043F06601B0F0BD4D20020135
:10A56000034804A1844B04F055FCC0464893010203
:10A57000B82E0100666C6173685F646D615F636132
:10A580006C6C6261636B000041A40000F0B581B0A7
:10A5900000786E4DAA68824200D0D0E001263002D9
:10A5A000032942D16A6DAA66AB6DAC6AA418EB654B
:10A5B0002C66AB6C5B1CAB646B6E934235D95E3022
:10A5C000FFF7FEFA686CA96C02293AD3814238D1B0
:10A5D000E88C696D081868650020062100F02CFDE4
:10A5E0002868E96D81602F6D04F0E6FB0446286859
:10A5F000C069C00705D004F0DFFB001BA98A8842B0
:10A60000F5D904F0D9FB04462A68D069800706D53D
:10A6100004F0D2FB001BA98A8842F5D92A6874206D
:10A62000285C012841D0F10440E0F2072B681C6847
:10A6300094431C60EA6E090411430143E96601B0CA
:10A64000F0BD0229FBD38142F9D2E88C696D09186B
:10A650006965A96D0818A8650020062100F0ECFCCA
:10A660002868E96D8160EF8C04F0A6FB0446286839
:10A67000C069C00705D004F09FFB001BA98A88426F
:10A68000F5D904F099FB04462A68D069800706D5FD
:10A6900004F092FB001BA98A8842F5D92A6874202D
:10A6A000285C012822D0F10421E03105334B3B40E6
:10A6B0005918012802D01920400601E00720C006E1
:10A6C00008182F4940185060002F0DD004F074FB7B
:10A6D00004462A68D069800706D404F06DFB001B8D
:10A6E000A98A8842F5D92A682B6D1FE03105234BD2
:10A6F0003B40C918012802D01920400601E007207C
:10A70000C00608181E4940185060002F0DD004F0F4
:10A7100053FB04462A68D069800706D404F04CFB3A
:10A72000001BA98A8842F5D92A68EB8C296EA86893
:10A73000144C00941432FFF723FB01B0F0BD044821
:10A7400004A10C4A0C4B04F065FBC046489301027F
:10A75000B82E0100666C6173685F646D615F77722B
:10A760006974655F6E62797465735F63616C6C6256
:10A7700061636B00720400009F2E0100FF3F000028
:10A78000008080008DA50000F0B587B0044601264A
:10A79000880E14D01546002A11D00F468120C0041F
:10A7A000401B88420BD37C206043F0490818059079
:10A7B000818C38460691F5F78DFC002902D0304691
:10A7C00007B0F0BD28460699F5F784FC0029F6D1BC
:10A7D000059880693E1A30460699F5F77BFC0746D6
:10A7E000039670190190069E3146F5F773FC0546F5
:10A7F000C01B04900598006A02903146F5F76AFC88
:10A80000049981420FD20026BD42D8D9204639464C
:10A8100000F018FB2046FFF77DFD0028FAD17F1CD1
:10A82000AF42F3D3CBE700900398029D2946F5F79A
:10A8300051FC0646284670430399081A019800D037
:10A84000761C2946009D7543F5F744FC0590029956
:10A8500041430198401A03900699F5F73BFC049098
:10A86000AF420BD22046394600F0ECFA2046FFF703
:10A8700051FD0028FAD17F1CAF42F3D305988642E0
:10A88000069D009F0CD220463146FFF77BFC2046F8
:10A89000FFF740FD0028FAD1761C05988642F2D3D6
:10A8A0000398A84203D20026304607B0F0BD0598B1
:10A8B00047430025E919204600F0C4FA2046FFF777
:10A8C00029FD0028FAD16D1C002604988542F1D399
:10A8D00075E7C046F0B585B0002803D001242046B6
:10A8E00005B0F0BD7822A14FB85C002803D0002449
:10A8F000204605B0F0BD0492002905D0384614303A
:10A900000CC90CC01CC91CC00020F86615242046C8
:10A91000FFF77EF8204603F051FF38681021C1612F
:10A9200004F04AFA04463868C169C90607D504F03C
:10A9300043FA001BB98A8842F5D9386800E0B98A21
:10A94000BA7D1207120B5218F97DCB07DB08D2181B
:10A950008B07DB0F5B05D218CB06DB0FDB05D218AC
:10A960004B07DB0FDB06D2188B06DB0F5B07D21819
:10A970000907C90F89071143016000240A212046F5
:10A9800000F05AFB3220FFF71BF90821204600F0A7
:10A9900053FB04F011FA05463868C169890606D4EC
:10A9A00004F00AFA401BB98A8842F5D93868017D5B
:10A9B0000A46C23A5342534174257B550904027D2D
:10A9C00012025118007D0B180220032668A231469E
:10A9D00005F07CFA785D0128039619D1F87D029084
:10A9E00000260621304600F027FB0721304600F004
:10A9F00023FB012102988143785D012847D1386803
:10AA00008901017506757521795C012938D048E006
:10AA10000020032100F010FB04F0CEF90646386850
:10AA2000C169890606D404F0C7F9801BB98A884237
:10AA3000F5D93868007D46080122F87D014631438A
:10AA40001640C90701D0304036D0029500250621B6
:10AA50002846019200F0F0FA07210095284600F000
:10AA6000EBFA019846400298385C012813D1386807
:10AA7000B1010175009901757521795C012910D129
:10AA800014307621795C4A424A41510008E0386826
:10AA90000675490003E038680099017571001430AB
:10AAA0000170374800687D21C900F5F713FB2821A4
:10AAB0004143002000F092FA7720385C012803D14E
:10AAC00002200021FFF734F804F076F906463868D2
:10AAD000C069C00705D004F06FF9801BB98A8842AD
:10AAE000F5D904F069F906463868C169890706D5C1
:10AAF00004F062F9801BB98A8842F5D93868D049D8
:10AB0000816117203856002829D57868002816D486
:10AB10000146039A91431C4A8B588507ED0EFF2688
:10AB2000AE40B3438026AE401E438E501F210140ED
:10AB30000120884015490860154908600FE0810729
:10AB4000C90EFF228A400F230340083B039883432A
:10AB50000C481D58954380228A402A431A500120F0
:10AB6000049978543861204605B0F0BD489301023D
:10AB70006A656465635F69642025780D0A000000DA
:10AB8000F0DF01021CED00E000E400E080E200E004
:10AB900000E100E0F0B593B07C270A90474393486A
:10ABA000C619980704D0F07D4024044000D017E176
:10ABB0000125880E2ED0002B2CD08120C004C01A75
:10ABC000884227D309920122EFF31084144002D166
:10ABD000EFF3108072B630461030059030690025D2
:10ABE00006280891069310D8079414468440E1067D
:10ABF000490F04D161210C4203D0154604E002251F
:10AC000002E00221059B1960079C002C00D162B66E
:10AC1000002D02D0284613B0F0BD344617347348D7
:10AC2000C05910210491C1613746143704F0C4F8AB
:10AC300005463068C069C00605D504F0BDF8401B64
:10AC400039888842F5D92078400665D40297B78CB8
:10AC5000069C20463946F5F73DFA079039464143B0
:10AC6000601A039035462435A74200D894E0039833
:10AC700000281CD006210A9C204600F0DDF9288817
:10AC80000799484308994018316888600027204692
:10AC9000039C394600F0D0F9079B099A288858434D
:10ACA000C0193168097D11547F1CA742F6D3306862
:10ACB0000499C16104F080F80446029D3068C069BF
:10ACC000C00605D504F078F8001B29888842F5D91C
:10ACD00004F072F804463068C069C00705D004F07B
:10ACE0006BF8001B29888842F5D904F065F8044602
:10ACF0003068C169890706D504F05EF8001B298811
:10AD00008842F5D930680121059A1160B249816104
:10AD10000025284613B0F0BD03200025089FF765E5
:10AD20000999316606997166B566F0660120C0071B
:10AD300031680A6802430A6006210A9C204600F036
:10AD40007BF9306887602046294600F075F93A4F54
:10AD50000BAA0A921BCF1BC21BCF1BC2B48CF0687C
:10AD60000A99FEF79DFFF0683168344A0092069A0E
:10AD7000944200D31446A3081431099AFFF700F84F
:10AD8000B06E0019B066306E00193066F06D0019B3
:10AD9000F065284613B0F0BD002404E0641C079859
:10ADA000844200D363E706210A9800F045F9288819
:10ADB0006043089940183168886000270A9839462E
:10ADC00000F03AF928880028099AE7D06043101863
:10ADD0003168097DC1557F1C28888742F6D3DDE79D
:10ADE000034804A1064A07A304F014F8489301029B
:10ADF000B82E0100666C6173685F72656164000063
:10AE0000C603000054686520444D412072656164AA
:10AE1000206C656E6774682073686F756C6420625F
:10AE20006520746865206D756C7469706C65206F41
:10AE30006620340D0A0000002C23010041A400000C
:10AE4000000093EBF0B583B00D4604467C264643E4
:10AE500051488719F869B98CF5F73CF9A84200D830
:10AE600094E0019502940121EFF31080084002D193
:10AE7000EFF3108272B63C4610343B690025062B76
:10AE80000CD80A469A40D3065B0F06D161231A42BA
:10AE900077D00D46002803D003E00225002800D11A
:10AEA00062B6002D02D0284603B0F0BD00943C46A7
:10AEB0002434394880591021C1613E46143603F0CC
:10AEC0007BFF05463868C069C00605D503F074FFEE
:10AED000401B31888842F5D90621029D284600F0A2
:10AEE000ABF8208801994143B86909183868816036
:10AEF000172179563C461734002909D5C16920220B
:10AF00000A43C2610121F966890502680A430260A9
:10AF10000421284600F090F8207840B22C46002505
:10AF20000028C0D42B4800687D21C900F5F7D2F86D
:10AF300020492D314143204600F050F803F03CFFFA
:10AF400004463868C069C00705D003F035FF001B10
:10AF500031888842F5D903F02FFF04463868C1696B
:10AF6000890706D503F028FF001B31888842F5D9F0
:10AF700038680121009A116017498161284603B0A1
:10AF8000F0BD0321216000288AD08AE7034804A18C
:10AF9000084A09A303F03EFF48930102B82E0100BE
:10AFA000666C6173685F736563746F725F6572610D
:10AFB000736500002B020000736563746F72206973
:10AFC0006478206973206F7665722072616E6765A0
:10AFD0000D0A0000F0DF0102000093EBF0B583B032
:10AFE00001917C220290424353498C182546143526
:10AFF00003F0E2FE06460221029800F01DF803F07D
:10B00000DBFE07462068C169890606D403F0D4FE3A
:10B01000C01B29888842F5D92068007DC00708D068
:10B020006420FEF7CDFD03F0C7FE801B0199884226
:10B03000E1D903B0F0BDC046F0B585B00491044637
:10B040007C2060433C490F183D46143503F0B4FEA4
:10B0500006463868C069C00705D003F0ADFE801B06
:10B0600029888842F5D903F0A7FE06463868C069EA
:10B07000800705D503F0A0FE801B29888842F5D9FA
:10B080001421049B5943DC2060432C4A1018039080
:10B0900002914018018A8268C47C7426BE5D012E2C
:10B0A0000DD10191012B02990CD0012B0DD07526E9
:10B0B000BE5D012E0ED0019E072B0ED10EE00E4676
:10B0C00002990BE00222012BF1D138247526BE5DD6
:10B0D000012EF0D10326072B00D0019E184B3340E0
:10B0E00024069207D20A1219D218039B5958C9078D
:10B0F000490C52184168CB071B0CD218837C5B07A4
:10B100005B0BD218C0684007000A10183A685060FC
:10B11000002E0ED001290CD103F04EFE04463868F3
:10B12000C069800705D403F047FE001B29888842C8
:10B13000F5D905B0F0BDC046489301027424010062
:10B14000FF3F0000F0B59DB00D460126890E2FD0BF
:10B15000002B2DD011928121C9041093C91AA94244
:10B1600026D30121EFF310840C4002D1EFF31082BB
:10B1700072B67C220F904243E748149287183846F3
:10B1800010303B690026062B0DD80A469A40D3069C
:10B190005B0F07D161231A4200D16FE30E46002CEA
:10B1A00003D003E00226002C00D162B6002E02D0AC
:10B1B00030461DB0F0BD0290BD6500211391796548
:10B1C0001098401E12904019B964B9690D916E1A19
:10B1D0001199B962FD6238637E63F98C0E91304635
:10B1E000F4F778FF0446B863129830180E9E314683
:10B1F000F4F770FF109B011B4A1CF86339647A64F2
:10B20000139A0029194608D0704359190D9BC91A81
:10B210000A1A7443581B80190119384648300E9099
:10B22000384644300D90384640300B903846263032
:10B230000590384658301390384654301290F964CF
:10B240003A651498B44908581021C1613846143041
:10B2500014903846503004903D464C3503F0ACFD18
:10B2600004463868C069C00606D503F0A5FD001B7A
:10B27000149909888842F4D9F87D40060C9500D5C8
:10B2800074E201230E9803600D98016800290F985D
:10B2900000D1CDE23A4674320A92DA0407921A05D6
:10B2A00009921922520606920722D206089216E047
:10B2B0009A4800687D21C900F4F70CFF10994143BA
:10B2C0000F9C2046FFF78AFE20460C9D0E9A1168BF
:10B2D0004B1C13600D9909688B4200D9A8E20B9AA8
:10B2E0001268012A55D0002A00D0A8E02E681299D1
:10B2F0000C6813990D6806211091FFF79DFE3868C0
:10B3000085601198051903F057FD04463868C06937
:10B31000C00706D003F050FD001B1499098888422D
:10B32000F4D903F049FD04463868C169890707D597
:10B3300003F042FD001B149909888842F4D938684B
:10B340000A990A78012A089900D00699012A099ACF
:10B3500000D0079A3346724C234013430B43714984
:10B360000B434360002EA3D003F026FD044638684B
:10B37000C069800706D403F01FFD001B14990988DB
:10B380008842F4D93868297801756D1C761EFAD187
:10B390008EE7012B00D0C7E02E6812990C68139934
:10B3A0000D6806211091FFF747FE386885601198F7
:10B3B000051903F001FD04463868C069C00706D0CE
:10B3C00003F0FAFC001B149909888842F4D903F0B1
:10B3D000F3FC04463868C169890707D503F0ECFC23
:10B3E000001B149909888842F4D938680A990A78A8
:10B3F000012A089900D00699012A099A00D0079AD3
:10B400003346474C234013430B4346490B434360A9
:10B41000002E69D003F0D0FC04463868C06980076C
:10B4200006D403F0C9FC001B149909888842F4D99A
:10B430003868297801756D1C761EFAD154E0012B0D
:10B4400000D0C9E02E6812990C6813990D68062186
:10B450001091FFF7F1FD386885601198051903F028
:10B46000ABFC04463868C069C00706D003F0A4FCF2
:10B47000001B149909888842F4D903F09DFC044606
:10B480003868C169890707D503F096FC001B149939
:10B4900009888842F4D938680A990A78012A0899F3
:10B4A00000D00699012A099A00D0079A33461C4C0D
:10B4B000234013430B431B490B434360002E13D01F
:10B4C00003F07AFC04463868C069800706D403F0AC
:10B4D00073FC001B149909888842F4D938682978CC
:10B4E00001756D1C761EFAD10C4800687D21C900DB
:10B4F000F4F7F0FD109941430F9C2046FFF76EFDD5
:10B5000020460C9D2A68139B196889181960129BA4
:10B51000196889181960D9E648930102F0DF010221
:10B52000FF3F0000008080008B4200D0CEE60499EF
:10B530000E6812990C6813990D6806211091FFF797
:10B540007BFD386885601198051903F035FC0446C9
:10B550003868C069C00706D003F02EFC001B1499A0
:10B5600009888842F4D903F027FC04463868C16989
:10B57000890707D503F020FC001B1499098888422D
:10B58000F4D938680A990A78012A089900D00699EE
:10B59000012A099A00D0079A3346D44C234013431A
:10B5A0000B43D3490B434360002E00D180E603F0E8
:10B5B00003FC04463868C069800706D403F0FCFB2E
:10B5C000001B149909888842F4D9386829780175D4
:10B5D0006D1C761EFAD16BE6129A1268119CA618A1
:10B5E000139A15688B425FD104990C680621039168
:10B5F000FFF722FD3868856003F0DEFB05463868FA
:10B60000C069C00706D003F0D7FB401B1499098816
:10B610008842F4D903F0D0FB10900C9D3868C169C2
:10B62000890708D503F0C8FB1099401A14990988B6
:10B630008842F3D938680A990A78012A089900D013
:10B6400006991091012A099A00D0079A2346A74922
:10B650000B40134310990B43A5490B434360002C47
:10B6600014D003F0A9FB10903868C069800707D494
:10B6700003F0A2FB1099401A149909888842F3D963
:10B68000386831780175761C641EFAD19A480068D2
:10B690007D21C900F4F71EFD039941430F9C20460C
:10B6A000FFF79CFC204611E605990C8806210391C2
:10B6B000FFF7C2FC3868856003F07EFB05463868FA
:10B6C000C069C00706D003F077FB401B14990988B6
:10B6D0008842F4D903F070FB10900C9D3868C16962
:10B6E000890708D503F068FB1099401A1499098856
:10B6F0008842F3D938680A990A78012A089900D053
:10B7000006991091012A099A00D0079A2346774991
:10B710000B40134310990B4375490B434360002CB6
:10B7200014D003F049FB10903868C069800707D433
:10B7300003F042FB1099401A149909888842F3D902
:10B74000386831780175761C641EFAD16A48006841
:10B750007D21C900F4F7BEFC039941430F9C2046AC
:10B76000FFF73CFC204605990A88CCE65E4815A9FF
:10B770000A4678C878C278C878C20125E8073A68CE
:10B78000136803431360B868FEF78AFA02200026A4
:10B79000139C2168BA6AF9653A6610997966BE66A3
:10B7A000F8660C980068129A1168091811600E9BCF
:10B7B00019684A1C1A60226810182060002900D0FD
:10B7C000F6E410953846603013903C465C343846B9
:10B7D0000830129006210F98FFF72EFC3868216878
:10B7E00081600C980068119003F0E6FA044638680E
:10B7F000C069C00706D003F0DFFA001B149909885E
:10B800008842F4D903F0D8FA0446109D3A68D0690A
:10B81000800707D503F0D0FA001B149909888842E5
:10B82000F4D93A687420385C01282DD0E9042CE062
:10B8300003F0C2FA04463868C069C00706D003F0B6
:10B84000BBFA001B149909888842F4D903F0B4FAB2
:10B8500004463868C169890707D503F0ADFA001BB3
:10B86000149909888842F4D938680121029A116034
:10B8700022498161002630461DB0F0BD04210160DF
:10B88000002C00D191E491E42905119C174B234031
:10B89000591801280C9D02D01920400601E007200C
:10B8A000C0060818124940185060002C0ED003F052
:10B8B00083FA04463A68D069800707D403F07CFA1B
:10B8C000001B149909888842F4D93A682B681398A8
:10B8D000016812980068074C00941432FEF750FA81
:10B8E00030461DB0F0BDC046EC220100FF3F000015
:10B8F000008080008DA50000F0DF0102000093EBC6
:10B900003920C0000149096808587047D4920102E3
:10B91000F0B5032920D8C0467944097949008F44FD
:10B9200001080F15012181404F4B1B685963D962F3
:10B9300012E0012181404C4B1B681963D9620BE076
:10B9400001218140484B1B68596304E0012181407B
:10B95000454B1B681963996283004349CB18DA6031
:10B960008A68002A29D14A68002A16D4032314467B
:10B970009C43174BE5589607F60EFF27B740BD438B
:10B980008027B7402F43E7501F23134001229A40DE
:10B99000104B1A60104B1A600FE09307DB0EFF2567
:10B9A0009D400F241440083C03229443074AA658A4
:10B9B000AE4380259D403543A55001228240086852
:10B9C0000262886810438860F0BDC0461CED00E04C
:10B9D00000E400E080E200E000E100E010B50124B6
:10B9E0002046FEF715F8204602F0E8FE002010BDC4
:10B9F000012181401C48006842688A4342607047C8
:10BA0000194909680968C140012008407047C046CB
:10BA1000012181401448006842680A43426070472F
:10BA2000012907D0002910D1012181400F48026867
:10BA30000A430FE0012181400B4800684368002A57
:10BA40000DD00B43436001617047012181400748DD
:10BA500002688A43026004480068416170478B4372
:10BA6000436001617047C046D8930102080100405D
:10BA700080B5114A1170114A10708001C90101434B
:10BA80000F480078400108430E4909780901014335
:10BA90000D480078C00008430C490978890001432B
:10BAA0000B480078400008430A4909780143C8B2AE
:10BAB000F8F72EFE80BDC046E09E0102AE96010260
:10BAC0001D90010264EA010299AD0102E19E0102AA
:10BAD00024A3010225A30102012282400548002976
:10BAE00003D0016811430160704701689143016010
:10BAF0007047C04600010040124A072809D880005C
:10BB00000F23834081401940106898430843106018
:10BB100070470F280AD8800020380F2383408140C7
:10BB2000194050689843084350607047800040387F
:10BB30000F238340814019409068984308439060E8
:10BB40007047C04634000040F0B54307DC0E0726BE
:10BB5000A640C3089D000E4BEF187D68B5433E1DFF
:10BB6000002908D035600122824001290CD11868D3
:10BB700010431860F0BD01218140186888431860A7
:10BB8000A24015433560F0BD186890431860F0BDC1
:10BB90000C01004010B582B014460A4601460498D4
:10BBA000009301900820234600F092F802B010BDE7
:10BBB000B0B584B014460A4601460898022500959F
:10BBC000019302900720234600F052F904B0B0BD63
:10BBD00070B500285BD031490A783149002A03D179
:10BBE0004A68012313434B60428803881B049A1858
:10BBF0000B46183B1A60828883891B049B180C46ED
:10BC00000C3C23600B46083B84681C60446903239A
:10BC10002340057CAD00EB188569AD072D0D5B1940
:10BC2000457C2D035B19C569AE07B60A9B19867C56
:10BC3000B6059B190E1F3360036A122B04D107242B
:10BC40000C60541EA2410AE0032C05D1012D03D83B
:10BC500007220A60012202E006220A600122114C3A
:10BC6000002525700F2464012034C57C6D02254019
:10BC70001B069B0BD218C3791B07DB0ED2188079E9
:10BC80000007C00D101840191439086070BD06482F
:10BC900006A1862209A303F0BDF8C046DCCC010250
:10BCA00018100050DECC0102953B01006C73705FF0
:10BCB000656E67696E655F72756E000050617261D6
:10BCC0006D65746572206973206E756C6C00000080
:10BCD000F0B58BB0109E34043ED00D46D64C2140BA
:10BCE000012701977F06B9423CD111462140B94254
:10BCF0003FD11C40BC4243D1119902AC0027E781DF
:10BD0000E780668027802782A774E1749908A18163
:10BD1000A908A1800A90099708970797900880B210
:10BD200004902046FFF754FFAA480078002801D06D
:10BD30000BB0F0BDAB480168C90708D10168C9075D
:10BD400005D10168C90702D10168C907F3D07F484E
:10BD5000019901700BB0F0BDB8480D49AF22C14B3D
:10BD600003F058F80095B5480949B022754B03F027
:10BD700051F80092B1480649B122724B03F04AF8DB
:10BD80000093AE480249B2226E4B03F043F8C0461E
:10BD90006B3B0100F0B58DB00392139E340446D086
:10BDA0000A46A54C2140012502956F06B94244D1AF
:10BDB00003992140B94247D11C40BC424CD114994F
:10BDC000129D04ACE174294921820027E781E780B4
:10BDD000668027809908A1819108A1800B95012D8B
:10BDE00001D16121CF43A7740C9002200A900990E1
:10BDF0000398800880B206902046FFF7E9FE754858
:10BE00000078002801D00DB0F0BD76480168C90760
:10BE100008D10168C90705D10168C90702D10168C5
:10BE2000C907F3D04948029901700DB0F0BD8348AD
:10BE30000D49FB228B4B02F0EDFF00927F480A492F
:10BE4000FC22404B02F0E6FF039800907B48064935
:10BE5000FD223C4B02F0DEFF009378480249FE22AF
:10BE6000384B02F0D7FFC046783B01008E8E0000B1
:10BE7000F0B58BB0119E340447D00D466E4C214076
:10BE8000012701977F06B94245D111462140B942A9
:10BE900048D11C40BC424CD11299109F02ACE174B5
:10BEA000294921820021E181E18066802180990871
:10BEB000A181A908A1800997012F01D0712100E07B
:10BEC0006121C943A1740A9003200890079090084B
:10BED00080B204902046FFF77BFE3E4800780028A1
:10BEE00001D00BB0F0BD3F480168C90708D1016817
:10BEF000C90705D10168C90702D10168C907F3D094
:10BF00001248019901700BB0F0BD4C480C49D52284
:10BF1000544B02F07FFF009548480949D622094B4F
:10BF200002F078FF009245480549D722054B02F000
:10BF300071FF009341480249D822024B02F06AFF88
:10BF4000873B0100B53B010086860000DECC010284
:10BF500010B582B014460A460146002000930190B5
:10BF600004202346FFF7B4FE02B010BD10B584B024
:10BF700014460A46014600200090019302900420D6
:10BF80002346FFF707FF04B010BD000070B50D4653
:10BF9000064604242046FDF73BFD204602F00EFC39
:10BFA0000B4805600B480670002E0ED00A48016849
:10BFB00080220A437F218A4302600120000307494F
:10BFC00008600749086007480460002070BDC0464B
:10BFD000E0CC0102DCCC01020CE400E080E200E0F5
:10BFE00000E100E01C100050B0B582B014460246DB
:10BFF0001148204001256D06A8420DD1180413D028
:10C000001748016000200093019006201146234646
:10C01000FFF75EFE02B0B0BD0094FF228C320748ED
:10C02000074908A302F0F6FEFF208C30421C0348AB
:10C0300003490C4B02F0EEFE0300FCFF953B0100B0
:10C040005D3B010044737420616464726573732006
:10C05000257820697320696E76616C696400000040
:10C0600008100050D33B010080B582B00B4601465A
:10C0700000200092019003200A46FFF729FE02B03B
:10C0800080BD0000002801D0042100E00221C54A43
:10C090005172411E8841800103490A6840239A4336
:10C0A000101808607047C04650A00050F0B583B02B
:10C0B00002912E49CD7A0E7B771987424FD9089984
:10C0C0000191182545434126F604BF00BE19745B53
:10C0D00034490C4057033C199B07D90C6418324B68
:10C0E0001B681B7A745375196C880326B6032640A7
:10C0F0009B079B0C9B193F2404401819029CA30624
:10C100001B0DC0186880012A184E13D8707B1422AA
:10C110004243307B5023434324011B199A18F37A7E
:10C12000C0181C234343D01880081E4A1040074300
:10C130000F432F800198686001F0C4FEA860E86892
:10C140001A4908403030E860286908402721715CAE
:10C150004018286100F044FE686103B0F0BDFF2282
:10C160008832034803A108A302F054FEE4D101027F
:10C17000243C01006D61635F63735F636F6E737472
:10C180007275637400000000435320696E64657823
:10C19000206973206F7665722072616E67650D0A83
:10C1A00000000000FF070000449401020000F0FFBF
:10C1B0002820D84900220A547047C046F0B581B003
:10C1C000009314460D46074606263046FDF720FC30
:10C1D000304602F0F3FA26211D4847540021017031
:10C1E00041708171017181704171C170C171022210
:10C1F0004272C16201634163816304734273C57219
:10C20000009A561C134A168001724120C004012175
:10C210004903F3F7C8FF502060432901081861194A
:10C220008A00801818224A438018B2B24A43801804
:10C23000094940180949884204D200F0B5F80020A5
:10C2400001B0F0BD064807A19A2209A302F0E2FD61
:10C25000E4D10102E0D10102280008020120080215
:10C26000243C01006D61635F696E69740000000029
:10C27000454D206F766572666C6F770D0A00000081
:10C28000A448C179002901D001207047007A411EDD
:10C2900088417047F0B583B002912A494B7B8342B5
:10C2A00048D9CB7A0C7BE31818245C439B00E31835
:10C2B0004124E4041A19142401900546654300261C
:10C2C000565100925519EE882E4F0B467A1C32407B
:10C2D000F54E3688497A711A2B4E0E40B618EE800C
:10C2E0003740997BEF80AA88284F17404A424A413D
:10C2F00091007918264A8918A980264F0F402D1DD4
:10C30000029801280AD124490E400921C902711856
:10C3100069800121C9037918298000E02F800198E4
:10C32000444300980019074A918C4182118C018284
:10C3300003B0F0BD3520C200034804A109A302F0F8
:10C3400069FDC046E4D10102243C01006D61635FD8
:10C350006C696E6B5F646573635F636F6E73747239
:10C36000756374004C696E6B206465736320696E3D
:10C37000646578206973206F7665722072616E67DC
:10C38000650D0A00FFFBFFFFFF03000003D0FFFF66
:10C39000E80F0000EF1F0000FF830000BE4A50635B
:10C3A00091637047E4D10102F0B581B04348CC21DC
:10C3B000016003214160B8490A7BD304404C1B193A
:10C3C000CC7AA218541E1C431823534392009A1887
:10C3D0004B7B14255D4352199201224301246306CD
:10C3E0001343436100228262C2620263426382633A
:10C3F000C26342650267334B1A605A609A60324BDF
:10C400001A601A619A61DC61304C1C62304C251D47
:10C410001D6325460C3D5D632546283D9D632D4EDD
:10C42000DE631C645C642C4D2F461C379F642746DA
:10C43000143FDF64103C1C65284C5C65284C9C65EF
:10C440000C369E67274CA5634035E563DA651A66AE
:10C450005A669A66DA661A67234DDD67022585619A
:10C46000224DC561C325AD03CD620A63D2435A6034
:10C470001F4A1368FF25AB4326254D5DAD072D0EE2
:10C48000EB1813601B4A102313601B4A136027220A
:10C4900060238B5419498160C160016121607D2155
:10C4A0000901016641661649C1641649416416498D
:10C4B000016400F085FC01B0F0BDC04604A000504E
:10C4C0000000F8FF94A0005034A10050FF185A005B
:10C4D00030040040041000401C2000405430004054
:10C4E00060400040B8A1005014001400FF3F3FFF1F
:10C4F00004E400E080E200E000E100E0DC05DC05AF
:10C500003F0270020133D007D007D0072921C64A65
:10C5100050547047E4D10102F0B58BB007920891F6
:10C520000146C14FB8780991FFF7B4FE78793A7B9C
:10C5300079790691824200D89FE0FB7A9A181823F5
:10C54000534392004124E10404915218D2187B7B9A
:10C5500014214B43D21850246043155801230A93E9
:10C56000DB022E469E4316504E4B2B4005937D7B9F
:10C5700003914D433E7B7443F97A0B011B195B1900
:10C5800071181C24029461435918A84B1B88069CFF
:10C590005C430919C904490D059BC91811501018AD
:10C5A0000799416038787979089A00920322099BAB
:10C5B000FFF77CFDF87A397B09183878814263D916
:10C5C00083000993049AD45C0894F7212140D15444
:10C5D000D1184D788E7836027619CB781B04F31873
:10C5E00007900A9886051E43330CCB70FB7A387B84
:10C5F000BC784D709F4D3540039E6643C018029B2A
:10C600004343981940029C4B03405C19200A8870F0
:10C61000200CC870F023089D2B401B1D3D7B089506
:10C62000FE7A099D5355C8700620079A5043801919
:10C63000089A801848701F22D20222400243100A32
:10C6400088707879401C7871387B7979814201D380
:10C65000002179713978491C3970F97A08183978CC
:10C66000884201D80020387028200A993954387A35
:10C67000401C3872387A0BB0F0BDA7204200D24877
:10C680000649074B02F0C6FBA72042007A32CE488B
:10C690007349744B02F0BEFBE4D10102443C01003B
:10C6A000ED3B010000F0FFFFE0D101020320000696
:10C6B00005490A6882430A600A6802430A6003481F
:10C6C000012101607047C0461C0000401CA00050C2
:10C6D00080B50120FDF752FC80BD0000F0B587B0A9
:10C6E00006930646504C607A504B1B88181A0C9DD6
:10C6F000A84200DC89E00F460592012E06D156487B
:10C700000021C1620169554A89180160A07831464B
:10C71000FFF7C0FDE078E178069A2B4600F0AEF80E
:10C720002078E1780097002206923346FFF7BEFC9E
:10C73000E07A217B0818217888426ED94120C20412
:10C7400004918800815C0391F7250D400292855485
:10C750004549455C4549465C360276194449475C83
:10C760003F04F6190127BF0537433E0C4654E67ACD
:10C77000217BA3783C4A85543E4D3D4014275F43BE
:10C7800089191C234B43D91949023B4B0B405D19B6
:10C79000290A364BC1542E0C35494654F0270399CB
:10C7A0000F400599002900D13F1D217BE37A029AB1
:10C7B00087542F4A86540622049E7243D218511879
:10C7C000294A81541F22D20215400D43290A274AC3
:10C7D0008154E078401CE070E07AE178814201D336
:10C7E0000699E1702178491C2170217B0818217875
:10C7F000884201D806982070E079401CE071A07A48
:10C80000401CA072E07907B0F0BD3920C20016329A
:10C81000074808A109A302F0FDFA3920C200044824
:10C820000F49104B02F0F6FAE4D10102E0D1010207
:10C83000243C01006D61635F747800004D4143202A
:10C840005458206C656E206973206F766572207273
:10C85000616E67650D0A00000804004090D0030077
:10C860005A3C01000B3C01000100080202000802D2
:10C8700003000802FF07C0FF00F83F00F0B589B0D1
:10C880000893019204914F4DEF7A874200D891E0CE
:10C89000297B502632464A434124E3040693D218AA
:10C8A000CC19A10051181822059254430A19697B2A
:10C8B0001423079359435318029000011958044652
:10C8C0000390504A0A40A97AC90251180898820573
:10C8D000D2088A181A514C4911402A7B00965643B7
:10C8E000384CE57A2C0106982418A719354E5419AE
:10C8F000A5007D19059844432819747B079D6C4356
:10C900000519049FD2194148048854432A19089CE8
:10C91000D204520D51181D460398195000F06AFABE
:10C920000146707A001902043E460CD080B2C00065
:10C93000002900D1801E029FA5214900F3F7CAFB00
:10C940001F21014001E00021029F3801281842798F
:10C9500083791B029A18C3791B04D2182C4B1340FD
:10C96000437109045918090CC171002C20D01548D5
:10C9700035460646007B009B4343F17A0A01069F39
:10C980003A43D21841188B00D218059B4B43D1185B
:10C99000727B079B5343C91840191C4A12884243B3
:10C9A00088180199884203D001992246F3F7E2FBE7
:10C9B00009B0F0BDFF225C32034804A109A302F0D4
:10C9C00029FAC046E4D10102243C01006D61635F95
:10C9D00074785F646573635F636F6E73747275639D
:10C9E000740000005458204445534320696E646528
:10C9F00078206973206F7665722072616E67650DAD
:10CA00000A000000FF0700E000F8FFFFE0D101028C
:10CA1000EFFFE00082B0FCF717FE05200025294655
:10CA2000FFF76AF806202946FFF766F80A2029462C
:10CA3000FFF762F809202946FFF75EF80124204637
:10CA400003F0C6FB284603F0C3FBFCF739FE204683
:10CA5000FCF72CFE01F032FE01F02AFE6D48016861
:10CA60006D480068890308D403210907084021079D
:10CA7000884202D0FCF7B6FD06E0FCF71BF9FCF794
:10CA8000C9FD0020FDF7C0FCFCF754FE0025284638
:10CA900004F0DEFC032661A23046314603F016FAAC
:10CAA00030462946FBF7A6FBF7F730FFFAF7E6FD1D
:10CAB000FEF794FF5F4F381DFCF7C0FBF7F71EFC35
:10CAC000F6F75AFBF7F7AFFE042630462946FFF784
:10CAD00013F8304621462A46FEF7A2FF05223046CB
:10CAE0002146FFF731F820462146FEF7C1FF674E89
:10CAF00030462430504A01902146FCF711FBFAF7EA
:10CB0000F1F8A2024D494E4B204603F05FFE01F0C2
:10CB1000B3FBF6F71FFB4B4A2046214602F090F884
:10CB2000494802F0BDF84948FCF746FDB8780028AE
:10CB30000DD104E0FBF7A0F9B878002807D1F7F78A
:10CB4000DDFE002803D1F079002815D13CE0FCF788
:10CB50007DFCB079002802D0B571F6F769F9F7F7D6
:10CB6000E1FEF6F7F3FEF7F723F9FAF795FDFCF788
:10CB70004BFCF079002827D0F571B078411CB170DA
:10CB80003D2806D30020B070012101982A4AFCF705
:10CB9000C7FAFAF72FFF2E480470F7F7AFFE002808
:10CBA00002D0BD70F57007E0F0781E28214600D352
:10CBB0002946B970401CF070F7F736F97F20C1059F
:10CBC000B069F3F7C8FBB0610B20FEF719FF3978A5
:10CBD000002810D00029ADD101201E4908703870FE
:10CBE00000201D49087003F0CDFAFBF745F9B8782D
:10CBF0000028ACD1A3E701299CD10020387050490E
:10CC0000C8831449087001201349087003F09AFA88
:10CC100090E7C046180000403000014055574220C0
:10CC200073696D706C65206578616D706C650D0A57
:10CC3000000000001C90010215900000E0CD0102F0
:10CC4000050A0100E9EB00007C3F000085CC0000F4
:10CC5000AE96010218900102199001020148006885
:10CC60007047C0460C00004081B080B581B003938E
:10CC700003AB009302F0A4FD01B080BC02BC01B084
:10CC80000847000001480021816170478098010237
:10CC9000F0B581B0002630463146FDF71BFE012578
:10CCA000AC022649264F30463A462346FDF772FF2E
:10CCB0003988244881423ED064217E5262217E52CE
:10CCC00060217E524422BE52FD87BD8778227A873A
:10CCD00002223A874322FA86BE83FE811A4ABA812B
:10CCE0007E810A223A81C822FA80184ABA803880A6
:10CCF000FE8306203885F984FF201230788487303F
:10CD0000B88450203E523A83EFF3108072B630461A
:10CD10003146FDF7DFFD00280CD12A0300263046FE
:10CD2000064D2946FDF730FD054A30462946234683
:10CD3000FEF708FA62B601B0F0BDC04600E002049A
:10CD400032A90102AA550000E1FF000034120000E0
:10CD50000020704710B50024002809D0002905D014
:10CD600003464A0003481946F3F704FA204610BD6B
:10CD7000E04310BD3C930102014600200A2901DA7C
:10CD8000C0437047014A11807047C046C4930102F6
:10CD90000020704780B50188064A11808178064AD4
:10CDA0001170C178054A11700079FCF773FB0020FF
:10CDB00080BDC0462E9401023094010294D201023B
:10CDC0000448054901601521090441600349816057
:10CDD0007047C0469C300040410008003400070006
:10CDE0000748006840697047FD2040000449096811
:10CDF000085C7047024800686221405C7047C0468A
:10CE00004494010210B5064804680648006864218D
:10CE1000F3F776F90221C9434143081910BDC04612
:10CE200098D201029CD201020A491A220A600A49D8
:10CE300048704878FF210902084A13688B43800331
:10CE400080B2C018106006482021016005480160CA
:10CE500000207047702000403494010204E400E098
:10CE600080E200E000E100E0F0B5A9B016460F4610
:10CE70000546C648002B024600D01A463921CC0090
:10CE80003D21C900511811918242189206D001200B
:10CE90004202BE491898F3F76DF9189A61201119EA
:10CEA00013910E21119C0A91A170002F0D9501D0B4
:10CEB0000A2100E00921592317938300E170784289
:10CEC000784113990870307810901070F17AE174FD
:10CED00071785170B7789770F178D1703579157194
:10CEE00074795471B1799171F179D171317A11728A
:10CEF000717A5172B17A91727E1EF0B200210328CC
:10CF0000169106D870B28000A1A210586A00805A0B
:10CF10001690179882001898C0181490F81E0228CE
:10CF200004D3012E084604D89D4800E09D4803190B
:10CF300018781290189DA818179028463030159030
:10CF40002C4656346D2080002950974A974B149EEA
:10CF500033627262B362F2623176F182139B59706E
:10CF600009229A70281841608160C160016110989F
:10CF700080008F490858F3F78BFD012F10900F9117
:10CF800004D0022F05D17F217E2004E07C217B206C
:10CF900001E05B215A20159DA984207003200C908C
:10CFA000A080012666701F200B90A8821820A8740C
:10CFB0000A46083A179BDA76169B129AD2184A4309
:10CFC0009100189A9163B702791E8B420E9109D98C
:10CFD000784860803420688477482882774813999D
:10CFE000088339E07F2B10DD802B18D031028B4273
:10CFF0001BD071028B4227D16E49618068846F48D3
:10D0000013990883CF20C00025E0202B17D0402B98
:10D010001AD1684860800420688469481BE065482C
:10D02000608006206884674815E0624860801020B0
:10D030006884624813990883C520C0000BE06248E9
:10D0400060800220688404E004206884812040001D
:10D050006080FF2002302882104600F0D7FE129830
:10D06000102806D0402808D108201499C876072037
:10D0700000E004201799887002E017980C998170DD
:10D080001898169A8078C11E02290CD3022811D054
:10D0900001280CD12672BA4200D900266672BA4223
:10D0A00013D8F44812E00D200002119908800120E5
:10D0B000800201E00C9800022081BA4201D8EE48BB
:10D0C00000E0FA20179988600EE0FA20179988602E
:10D0D000139800780028119901D0E8484880E84862
:10D0E000139A1083E7480880A88CF3F733FC0026D6
:10D0F000E54B3246F3F7B6FA02460B46E3493046B3
:10D10000F3F718FBE24B3246F3F7ACFAF3F774FC93
:10D110000746E080DF493046109A0F9BF3F70AFB81
:10D12000DD4B3246F3F79EFAF3F766FC7843404254
:10D13000800B608116990E98814208D90C20149FAB
:10D14000B872D648179988831220189A0EE0480AB8
:10D15000189A149F01D00D2003E0080A00D1DBE2E9
:10D160000A98B872CE48179988831220F872D0783E
:10D17000052844D878440079400087440227402C91
:10D180003339C848B881C8482FE0C046D49001025E
:10D190009C2201009C220100AC220100AC22010073
:10D1A0008C1F0100931F0100307500001027000044
:10D1B0004C20010005020000FF06000004080000EA
:10D1C0000A0400003604000003020000B748F8819A
:10D1D000B748388013E0B748F881B7483882B74875
:10D1E00038600CE0B448B881B5481799C88306E0A8
:10D1F000B4487882B448B8800B9800069064AE4872
:10D200003881A748F880B14802882A84B04800785D
:10D21000E874B0480078119F7875387D1390002825
:10D220005ED0AD490A681023DA413A600A794B7939
:10D23000CF8867801B029A186A840A7A4B7A8F7AA1
:10D24000C87A0D7B65701B029A183B04D218000641
:10D250001018179FF860487B8A7BCB7B3B771202C4
:10D2600010186081087C7877487C149A9072887CCA
:10D27000D072C87C159B1874087D5874487D119035
:10D280009874C87D0A7E120212181A84887DD87498
:10D2900018464B7EC375887ECD7E2D022818B88037
:10D2A000087F4D7F2D022818F880887FB877C87FC7
:10D2B000F8772020085C149D28732120085C68738F
:10D2C0002A20085C2A314D782D0228188D782D04EB
:10D2D0004019C9780906401818998864119801E026
:10D2E000EB7DA87C7D498B700A8080001F38C88246
:10D2F000C883139800281FD022227748825C0346F7
:10D3000022335B781B029A180A842422825C03462B
:10D3100024335B781B029A18CA842622825C034657
:10D3200026335B781B029A188A832822825C283075
:10D3300040780002801888846948032569A229463C
:10D3400002F0C4FD189F387814907B78B8780F905D
:10D35000FA78B8791390F8791190387A1090787A31
:10D36000B97A0890099100930F980190029216984B
:10D3700003901298049013980590119806901098B5
:10D380000790FAA2F8482946149B02F09FFD3D46FB
:10D39000643580212846F2F706FFB878C11E0229BD
:10D3A0000ED3012800D18FE1022800D0ABE1169105
:10D3B000149078787F225043F7494018F74907E0E6
:10D3C0001691149078785B225043F1494018F14946
:10D3D00041182846F2F7CEFE0D9D1898C6870E34E8
:10D3E000324602E0641C0F2A0ADA21780029F9D0BB
:10D3F000491C8907C90F91400E43C687521CF1E7AB
:10D400001699022907D31499491E012900D97DE1F3
:10D410004279D24901E04279CF4989180C78002D30
:10D4200000D177E1C1790E91032900D94AE142790F
:10D43000062A00D979E14921890041181191E43087
:10D4400010900E98401E129019A800190F900023FA
:10D450001392149403E01898290600D15AE1052A82
:10D460005AD8C0467A44127952009744455C728576
:10D4700098ABC04688130000E20400000C080000CE
:10D48000060A0000040F00000000104130C1BD4139
:10D49000000070400000F0400000D041120C00007D
:10D4A000140B000012120000140E00000E160000F3
:10D4B000130D0000121600000E120000140B0E0ACD
:10D4C00012080000101600000E0B00002E9401023E
:10D4D0003094010294D20102A0D201029C94010274
:10D4E000010800004361736520706172616D6574AD
:10D4F0006572733A200D0A001693DFB2002F04D034
:10D5000019A801223946F2F747FE002C00D191E01C
:10D5100019A8C019BB498AE0E8B2022867D00027E1
:10D52000022867D06BE00E98022872D1E8B2022878
:10D5300000D103461693DFB2002F04D019A80122B0
:10D540003946F2F729FE002C74D019A8C019ACA1F5
:10D550006DE0E8B2022800D104231693DFB2002F59
:10D5600004D019A801223946F2F716FE002C61D02A
:10D5700019A8C0199FA15AE0E8B2022800D10623D9
:10D580001693DFB2002F04D019A801223946F2F712
:10D5900003FE002C4ED019A8C01992A147E0E8B2B2
:10D5A000022800D10C231693DFB2002F04D019A853
:10D5B00001223946F2F7F0FD002C3BD019A8C01922
:10D5C000874934E0E8B2811E4A424A419700022866
:10D5D00004D119A801223946F2F7DEFD002C16D03D
:10D5E00019A8C0197CA12246F2F7C4FD0FE0062756
:10D5F000022804D119A801223946F2F7CDFD002CEA
:10D6000005D019A8C01980492246F2F7B3FD169734
:10D6100010E01693DFB2002F04D019A8012239467A
:10D62000F2F7BAFD002C05D019A8C019734922469B
:10D63000F2F7A0FD3C193F2C05D80F98C0194021E6
:10D64000091BF2F7B0FD12980228189801D20020A9
:10D6500002E0C078411E884115990870611E2E466F
:10D66000E8B202280CD1179A517019A9119AB8C9B9
:10D67000B8C2B8C9B8C2B8C9B8C2B8C9B8C20DE052
:10D68000179A117019A9109AB8C9B8C2B8C9B8C206
:10D69000B8C9B8C2B8C9B8C2C10709D180073546F0
:10D6A000149C139A169B00D4D5E602208543D2E63B
:10D6B000FE20354605401898149C139A169B29069F
:10D6C00028D0CCE637A231E01691149078780B99E7
:10D6D0004143334808181F386F21C9430D9D7A18FC
:10D6E0000378D427D3554378D827D3558378DC27BC
:10D6F000D355002900D170E6C378E027D355103107
:10D70000001D189FEBE70120404A10E00024002D87
:10D7100000D087E629B0F0BD80290ED30F20B87263
:10D72000104817998883102020E525A20120014682
:10D7300002F0CCFB189829B0F0BD1020402904D38A
:10D74000B8720849179B998310E5B8720448179975
:10D75000888314200AE5C046931F01008C1F010036
:10D76000150F0000140B000001080000256420259F
:10D7700064202564202564202564202564202564F8
:10D780002025642025642025642025640D0A0000DE
:10D79000E04501001DF7FFFFF83C010089FBFFFF9A
:10D7A000E84401007472785F6D6F64652070617287
:10D7B000616D65746572206572726F720D0A00008A
:10D7C0004E73666420706172616D65746572206568
:10D7D00072726F720D0A0000FFFFFFFF01FF000071
:10D7E0004C230100FFFFFFFFFF0101FFFF01FF01CD
:10D7F000FFFF01FFFFFFFF01FFFF01FF38290100CD
:10D80000FFFF01FF6C230100BC220100963C0100D8
:10D81000002800D10148064908607047D4900102F1
:10D82000F0B586B0002805D10148006802E0C04686
:10D83000449401023121C900049141188A791F23BF
:10D840001A40CD79ED06AD0DAA180D7AED066D0CD6
:10D8500052194D7AED062D0B52198D7AED06ED0910
:10D860005219CD7AED06AD0852194D7CED075219CB
:10D87000BD4C22600A7B1A404E7BF606B60DB218EC
:10D880008E7BF606760C9219CE7BF606360B921935
:10D890000E79F606F60992194E79F606B60892192F
:10D8A00062604A6AB14D2A40A2608A6A2A40E260F8
:10D8B0002D22D20087183A7E1A4003937E7EF60608
:10D8C000B60DB218BE7EF606760C9219FE7EF606EE
:10D8D000360B92193E7FF606F60992197E7FF60600
:10D8E000B60892190E7CF60792192261BA7F1A4087
:10D8F0000597FE7FF606B60DB218049BC35CDB06E7
:10D900005B0CD2184B78DB061B0BD2188B78DB062E
:10D91000DB09D218CB78DB069B08D2186261CA6992
:10D920002A40A2610A6A2A40E2618A7C01252A40D3
:10D93000CB7CDB079B0F9A180B7DDB075B0FD218A4
:10D940004B7D9B07DB0ED2188B7DDB079B0ED2181D
:10D95000CB7D1B079B0D9A180B7E1B079B0CD218C7
:10D960004B7E5B06DB0A13438A7E520612091A437A
:10D97000CB7E5B075B0813432362CA6A62620A6B51
:10D98000A2624A6BE2628A6B22633922D200835C14
:10D990001E462E4066635E425E41B304AE04744F81
:10D9A0003C68B443E3183B6083185A782A409C785B
:10D9B0002407E40EA2188C8F6401A2186D4C144049
:10D9C000C98FC905490A0919DA78D207120A8918D4
:10D9D0001A791207120989185A79D207D2088918B8
:10D9E000FB4EB1639968F163997904952940DA791E
:10D9F000D207920F51181A7B5207D20E89185A7B00
:10DA0000D206920D51189A7B5207D20C8918DA7BF4
:10DA1000D206920B89181A7CD206520A89185A7CAF
:10DA2000520792090A43997CC90649085118316482
:10DA3000D97C039A11401A7DD206920D51185A7D55
:10DA4000D206520C89189A7DD206120B8918DA7DFB
:10DA5000D206D20989187164197E0F2421405A7E9A
:10DA6000120151189A7E12038918DA7E1207120ADF
:10DA700051181A7F1207120989185A7F120789183C
:10DA8000B164997F01942140DA7F1207120E511878
:10DA90003D22D200835C5B075B0D591884186278C5
:10DAA0001207520C8918A278D206120B8918E27854
:10DAB000D206D2098918F164217907220A406179D6
:10DAC000C9008918A2795206920B5118E27992077F
:10DAD000120B8918227AD2078A18BF490A60627A23
:10DAE000A37A1B029A18E37A1B04D2184A60E289CF
:10DAF000BA4B13400394228AD2049209D2188A6046
:10DB000003463033598CB64A114002939A8CD205A1
:10DB1000D20A51185622825C12068918B14D29602A
:10DB2000014656314A788C782402A2188C88640504
:10DB30006409A218CC78240712196A60CA880C7A82
:10DB4000A407A40BA2184C7A6407E40A1219AA606D
:10DB50004989E960492189004118FF22663282180B
:10DB600000921035002207E000300040FFFFFF0068
:10DB700004040040FF3F000084186427E65D03278B
:10DB80003E406523E35C9B071B0F9B196626A65D41
:10DB9000B607B60EF3186726A65DB601F318DBB21A
:10DBA0006826A65DB607B60DF3186926A65DB6070A
:10DBB000360DF3186A26A65DB607B60CF3186B2669
:10DBC000A65DB607360CF3186C26A65DB607B60B35
:10DBD000F3186D26A65DB607360BF3186E26A65D04
:10DBE000B607B60AF3186F26A65DB607360AF3180D
:10DBF0007026A65DB607B609F3187126A65DB607AE
:10DC00003609F3187226A65DB607B608F318732610
:10DC1000A45DA407E31808C51032802AACD1019A8C
:10DC2000D243704EB4180B783B404D78AD072D0FA2
:10DC3000EB188D78AD07AD0EEB18CD78AD01EB1874
:10DC4000DBB20D79AD07AD0DEB184D79AD072D0D9C
:10DC5000EB188D79AD07AD0CEB18CD79AD072D0C18
:10DC6000EB180D7AAD07AD0BEB184D7AAD072D0B08
:10DC7000EB188D7AAD07AD0AEB18CD7AAD072D0AFA
:10DC8000EB180D7BAD07AD09EB184D7BAD072D09EA
:10DC9000EB188D7BAD07AD08EB18CD7BAD07EB180E
:10DCA000A3641031121DBDD1009B19785A78520718
:10DCB000520D51189A78D207120D8918B164059B3C
:10DCC0001968F164D97D5A68120251183165996852
:10DCD000454A0A40998A490589187165D9683D4CB9
:10DCE0002140B16519692140F165029E3178049D9A
:10DCF000294082785207120F5118C2799207920E6A
:10DD00008918427A9207920D5118827A9207120D61
:10DD10008918C27AD207920C89189A7DD207520CC0
:10DD2000891872789207D20B8918B2781207D20A32
:10DD30008918F2781207D2098A182C490A60327CB5
:10DD4000737C1B071B0D9A18B37C9B069B0BD21888
:10DD5000F37C1B079B0AD218337DDB065B09D218C4
:10DD6000737DDB071B09D2184A60B27D2A40C38F3E
:10DD70005B009A188A60826CCA60C26C22400A6199
:10DD8000F27D7F231340328C5204520AD2184A612A
:10DD900002698A614269CA6182690A62C2694A6229
:10DDA000026A8A62426ACA62826A0A63C26A4A6311
:10DDB000039A927CD201121D0A64027A3A40CA6523
:10DDC000808F074A10400866002006B0F0BDC046AC
:10DDD00000300040FFFFFF009C300040FF1F0000AC
:10DDE000FF03000000400040FFFF1F000020004034
:10DDF00004480068806B800803490968490040189E
:10DE000009307047449401021004004010B52D21E0
:10DE1000C9004118027A032A04D10079002807D0EA
:10DE2000082006E08378DA1E022A05D2032412E0D5
:10DE3000142088601C203DE0012B02D1C8228A609A
:10DE400012E00479042C01D3462404E0032C01D110
:10DE5000322400E014248C605B1E022B04D3022ABF
:10DE600010D24279154B01E04279154B9B181B7873
:10DE7000402B04D0102B06D11423442405E02A2380
:10DE80003E2402E04279342348244B800C80022A4D
:10DE900006D0062A08D0052A08D118224C2301E012
:10DEA000142250230B8000E01C224A80C0780428F2
:10DEB00003D1142048806420088010BD931F010006
:10DEC0008C1F0100134800687047C04610B5104A07
:10DED000107091700F49002813D050680861042019
:10DEE00048619078FF2212020B4B1C689443800318
:10DEF00080B20019186001204007084A1060084AE3
:10DF0000106000200860074901220A6010BDC04669
:10DF100034940102180400401CE400E080E200E0B8
:10DF200000E100E070000040F0B591B0002801D1A0
:10DF3000C04800688778F91E022913D3012F21D029
:10DF4000022F3CD11021CA4344782146193991420D
:10DF50003DD800970125B94A28462946234601F0B5
:10DF6000B5FF53E10821CA43447821462139914243
:10DF700018D800970125B14A28462946234601F0C2
:10DF8000A5FF43E10821CA4344782146093991425B
:10DF900034D800970125A94A28462946234601F08E
:10DFA00095FF33E1032F3CD0042F43D1C3780125E3
:10DFB000042B00D02DE106462A02042343E001256C
:10DFC000A6A2284629463B4601F080FF1EE1C37801
:10DFD0000125052B0AD806462A02284698401B210F
:10DFE000084230D10021052B08462ED00220009097
:10DFF000914A2846294601F069FF07E10646C378A1
:10E000000021022B1ED3032B1CD0042B08460A46EA
:10E010001BD001250095884A2846294601F056FF65
:10E02000F4E0C3780125032B00D0FAE006462A026B
:10E03000032308E0012583A2284629463B4601F038
:10E0400045FFE3E00A46012148020F91592189006A
:10E050007518FD21490071180291314662313F0562
:10E06000D219641E1F2727405C013C191443044346
:10E0700032795207D20C22432B789B065B0BD218C5
:10E08000B379DB071B0B13436D4D2B60F279032330
:10E0900010931A40737A9B079B0E9A18B37A5B070A
:10E0A000DB0D9A18F37ADB079B0DD218337BDB0765
:10E0B0005B0DD218737B1B075B0CD218AA60326908
:10E0C000EA6072692A61B2696A61F269AA61326AB8
:10E0D000EA61726A2A62B26A6A620F980870F06A2C
:10E0E000A8623F20C4432C353046E4300F903046C0
:10E0F000E5300E903046E6300D903046E7300C901B
:10E100003046E8300B903046E9300A903046EA302D
:10E1100009903046EB3008903046EC30079030469E
:10E12000ED3006903046EE3005903046EF300490EA
:10E130003046F03003903746F1373046F230F33650
:10E140000F990A194021525C109B1A400E9B1B1913
:10E150005B5C9B071B0F9A180D9B1B195B5C9B0755
:10E160009B0E9A180C9B1B195B5C9B019A18D2B2F0
:10E170000B9B1B195B5C9B079B0D9A180A9B1B1939
:10E180005B5C9B071B0D9A18099B1B195B5C9B072B
:10E190009B0C9A18089B1B195B5C9B071B0C9A181D
:10E1A000079B1B195B5C9B079B0B9A18069B1B1913
:10E1B0005B5C9B071B0B9A18059B1B195B5C9B0701
:10E1C0009B0A9A18049B1B195B5C9B071B0A9A18F5
:10E1D000039B1B195B5C9B079B099A183B195B5CB3
:10E1E0009B071B099A1803195B5C9B079B089A18ED
:10E1F0003319595C8907891802C51034A0D10298D7
:10E200000078042101430E48C1630025284611B05F
:10E21000F0BD04200090084A2846294601F056FE29
:10E22000F4E703200090044A2846294601F04EFEF8
:10E23000ECE7C046449401026B3C0100B13C010094
:10E2400000100040556E646566696E6564206D65FA
:10E25000616E205052462025640D0A00496E766199
:10E260006C6964206D65616E205052462025640DF6
:10E270000A0000007047704780B50E490E480246FC
:10E28000083A1268920000D4603142680A43426042
:10E290000A490A6808239A430A60091F01225204A6
:10E2A0000A600321890402688A430260FBF732FA9C
:10E2B00080BDC046200000802800004004020040CD
:10E2C000B0B5032000072D490A688243012568077D
:10E2D0001018086000242046FFF7CDFF2046FFF706
:10E2E000C9FFEFF31080284002D1EFF3108172B61E
:10E2F0008021C943224A53680B40536093680B4006
:10E300009360D3680B40D36013690B40136153696A
:10E310000B405361002800D162B6B0BD70B50C4609
:10E3200003210907154A13680B4313600122EFF319
:10E330001081114002D1EFF3108272B68025EA43BA
:10E340000F4B5E6816405E609E682E439E60DD68DF
:10E350001540DD601D6915401D615D6915405D61F9
:10E36000002900D162B6002802D00120FFF783FF08
:10E37000002C02D00120FFF77DFF70BD000400409B
:10E38000D89501020D4A002907D001290BD101219E
:10E39000814010688843106007E0012181401068C7
:10E3A0000843106001E001218140101F02680A4308
:10E3B0000121C907114301607047C0464400004075
:10E3C000032804D840000649085A00B270470020CC
:10E3D00000B27047032802D84000014A115270472A
:10E3E000CED201029E4908707047C04670B58AB00F
:10E3F0000C460546FF20FC30A8490E68315C5920C8
:10E400008000335CB278307808AE069609AE059687
:10E410000C4E04962126760603960B4E0296012694
:10E4200001960E2600965B1CDBB2F7F7F9FB099804
:10E43000F2F7B4FA28700898F2F7B0FA20700AB030
:10E4400070BDC0460000204100000443F0B58BB011
:10E450000446457C824800788249002822D000206A
:10E460000880814A1080814B01269E761E830A9087
:10E470007F4800787F4E36786DB205957E4D0495C5
:10E480007E4D03950AAD02957D4D01950096F7F7F7
:10E4900005F90A9D112020567A497B4A00F022FC9A
:10E4A000064626E000260E806F4A16806F4B01203C
:10E4B0009876188309966E4800786E4F3F786DB253
:10E4C00005956D4D04956D4D039509AD02956C4D07
:10E4D00001950097F7F7E2F8099D112021567F205A
:10E4E000C005009001900296664A674B3046F8F7E7
:10E4F00029FA432001062846F1F786FFF2F74EFA83
:10E50000089062480078002824D05120800060499B
:10E510004A7D42438D185F480068A8642F46403703
:10E5200050480078B87450480078F874554800781E
:10E53000387555480078787557480078F875504810
:10E540000069F2F72BFAB87552484069E8644C4804
:10E5500000686864FF20FE3050490968085C392271
:10E56000D2008918022812D303D04E48007801281F
:10E570000DD14B480660434800883A4A1080424813
:10E580000088394A108009200790089605E0444821
:10E59000089A02603548C08B07900B780022002B48
:10E5A00001D0114600E0D1430125002B01D0042306
:10E5B00000E0EB43A67AAD1BEE175B19714165686D
:10E5C000AE0F277AAD00ED195641677A3F1FF81755
:10E5D000ED1970414000EE0F80196D00EB184841B5
:10E5E0008001990E4118980127239B02C31A91417B
:10E5F0001D4805881B480088854201D00798421BAA
:10E6000010202056C001194D2D8C032D07D1E46830
:10E61000E5176D0A6419E4150519EC170FE0E468B5
:10E62000E5176D0A6519EC17ED15C6174519744104
:10E6300097B2002F00D03446002F00D00546581B5B
:10E64000A141130409D012B2D2015242D31780184B
:10E650005941089BDA17C01A91410BB0F0BDC04672
:10E66000C69301023CAD01023AAD01029C94010245
:10E67000B5900102B490010228A3010224A1010275
:10E6800040AD01028AAD010288AD0102F4A601028B
:10E690002CA401026420004038AD01024494010220
:10E6A00034AD010298AD0102C10D400280307047C7
:10E6B0000120C0071B4908607047C04610B51948C3
:10E6C0000068C10710D1810711D4410712D4010796
:10E6D00013D4C10614D4810615D4410616D4802162
:10E6E000084016D031A215E001240FA213E0022445
:10E6F00011A210E0032414A20DE0042416A20AE0E3
:10E70000052419A207E006241CA204E0072421A284
:10E7100001E0254A04090220032101F0D7FB20462D
:10E7200010BDC0465C00004052657365742062797C
:10E7300020504F520D0A00005265736574206279B3
:10E7400020424F520D0A00005265736574206279B1
:10E750002050494E0D0A000052657365742062799D
:10E76000205744540D0A0000526573657420627985
:10E77000204C4F434B55500D0A0000005265736505
:10E7800074206279205357205265626F6F740D0AAE
:10E79000000000005265736574206279205359535C
:10E7A0005245510D0A000000162F01005265736595
:10E7B0007420627920445644440D0A0001218140AE
:10E7C000044A1F2802D0106888431060106808436C
:10E7D000106070471C000040F0B583B00291044601
:10E7E0009949F1F777FC0546984901942046F1F7DD
:10E7F00071FC974946189749714300956F189649DF
:10E80000441864212046F1F765FC3818A108471A1E
:10E8100092492046F1F774FC381891494518914FF8
:10E8200005D464213046F1F755FC0C4614E0A6B23D
:10E8300064213046F1F74EFCB7204000A20701D119
:10E84000002907D1884B73430422D341874A93425E
:10E8500000D3401E0C464519009847430298068095
:10E86000192001013046F1F735FC2A461F3A2846A7
:10E8700000DB1046019BFF18B30705D1002C03D025
:10E880001F2D05DA0120C5E01F2D0BDA0120C1E0A4
:10E8900005461D3D034600DB2B461C2808DC0220F4
:10E8A0001546B7E000290CD01C21451A0CD50CE008
:10E8B00019461F39184600DB08461F2B1DDA0320B6
:10E8C000A8E01D21451A00D42846002D08D4014691
:10E8D0001F39024600DB0A461F2804DA032099E0AC
:10E8E0000220154696E015461E3D104600DB2846E0
:10E8F0001E2A0CDA04200D468CE005461E3D024619
:10E9000000DB2A461E280BDA04200D4682E0014671
:10E910001F39024600DB0A461F280ADA052079E083
:10E9200011461F39104600DB08461F2A0BDA052066
:10E9300070E015461E3D104600DB28461E2A0CDA04
:10E9400006200D4666E005461E3D024600DB2A46CF
:10E950001E280BDA06200D465CE001461F390246F0
:10E9600000DB0A461F280ADA072053E011461F3948
:10E97000104600DB08461F2A0BDA07204AE015463E
:10E980001F3D134600DB2B461F2A0CDA08200D46DC
:10E9900040E005461F3D024600DB2A461F280BDAF1
:10E9A00008200D4636E019461E39184600DB084699
:10E9B0001E2B0ADA09202DE011461E39104600DB15
:10E9C00008461E2A0BDA092024E01F28054601DB31
:10E9D00005461F3D1F280CDA0A200D461AE01F28A5
:10E9E000054601DB05461F3D1F2806DA0A200D46B5
:10E9F00010E01E2D05DB0C2004E01E2D06DB0C2094
:10EA000005E00B201E2D05DB1E3D03E00B201E2D17
:10EA100000DB1E3D029EB070681CF070E120010119
:10EA20003846F1F757FB3071C0B211494143CC1958
:10EA30003C212046F1F74EFB70713B21C943414315
:10EA40000819B07103B0F0BD805101008033E101BD
:10EA5000B207000093FEFFFFB107000070FEFFFF4A
:10EA6000A7FA0A0080AEFEFF295C8FC20BD7A30075
:10EA7000F0F1FFFFF0B581B00446FFF721FCA08A5A
:10EA800000280ED0FFF71EFA2049086120482CCC40
:10EA90002CC02CCC2CC02CCC2CC00020888101B0E8
:10EAA000F0BDE08A194FB881A169BA891948F1F718
:10EAB00061FB174D204629464CC84CC14CC84CC17F
:10EAC0004CC84CC1FFF7FEF938616E68FFF790F94A
:10EAD000301AB8622846FFF7B9FC06460D460E48C4
:10EAE000007BFFF76DFC0121F970617C7971396C55
:10EAF000491C396481B2C90B401800B2C1174010DB
:10EB0000301A38658D417D6501B0F0BD3099010244
:10EB10000C9A0102D8D20102B690010270B50446E7
:10EB2000FFF7CEFBA08A1B4E7082718A002908D0A5
:10EB3000B0820220707100203082FFF7C3F9F061CB
:10EB400070BDE08A3082A169328A1348F1F712FB66
:10EB50002046FFF77BFC05460C461048007BFFF77C
:10EB60002FFC81B2C90B401800B2C1174010281AFF
:10EB700030668C417466FFF7A5F9B061F06C401CFB
:10EB8000F064FEF73FF9F063FAF78AFC3064012085
:10EB9000707170BDB096010270D30102C490010281
:10EBA000F0B581B0EFF3108072B600200146FBF79C
:10EBB00091FE0446002803D062B6204601B0F0BDA5
:10EBC00001273A030025074E28463146FBF7DCFDB6
:10EBD000BB021A4A28463146FCF7B4FA62B6204610
:10EBE00001B0F0BD00E0020410B5F5F71CFE114CB9
:10EBF000E078002801D0F9F773F9F9F7E7F9F7F7AA
:10EC000061FF0D490120C8720A7B03469343CB7113
:10EC1000521C0A73094A928F002A08D08A7A4B78CC
:10EC2000134304D04A7A501C48720120904360700C
:10EC300010BDC0461C9001028098010232A9010259
:10EC400070B514460D4606461120FAF7E1FE22483B
:10EC5000042101600C4804601E4805608660002E97
:10EC60000DD0FF20000609490A6882430120C00731
:10EC700010180860064808210160064801601A2043
:10EC80000221FFF77FFB70BD70D4010200E400E0B9
:10EC900080E200E000E100E00C4908607047C046F7
:10ECA00010B504460948006860430949F1F728FA9D
:10ECB00000190849486008480022026002460C3AE0
:10ECC0004B6813600968016010BDC0466CD4010236
:10ECD00040420F000C9001022C10014000480047F8
:10ECE000C100000080B582B013460A460090034878
:10ECF000011D0348F7F7D2FD02B080BDACD401027C
:10ED00005CA0010210B50C498A1C90420DD2401E35
:10ED10000D4A50600D4803680B4003218C071B19F6
:10ED2000036000209060116010BD04480449E62291
:10ED3000044B00F06FF8C046FFFFFF00ED2E01000E
:10ED4000072F0100D32E010010E000E020ED00E0CD
:10ED5000B0B50120EFF31081014002D1EFF3108232
:10ED600072B6124A1368124C22686468850611480C
:10ED700000682840850E5D192923DB006B43002CB9
:10ED80001D4606D1002809D11E20684300290AD05B
:10ED9000B0BD121BD218551C0028F5D01D461E20F0
:10EDA00068430029F4D162B6B0BDC046DCDF010281
:10EDB00014E000E004ED00E080B50020FBF734F83B
:10EDC000404280BDB0B586B0104869460A4638C892
:10EDD00038C238C838C200242046FBF72BF8039904
:10EDE0002046FBF7C1F80198012803D00824002829
:10EDF00004D102E00424002800D104460220FAF7DE
:10EE00000FFEE0400249086006B0B0BD981F010047
:10EE1000F0DF010290B01C4605AB07C3EFF3108092
:10EE2000C00702D1EFF3108072B6EFF310800B90A1
:10EE300068460E907046089010AB0F93CF4F3E1D62
:10EE400001200490C50230462946224600F0B8FC55
:10EE500000213154EFF303800990EFF308800C9008
:10EE6000EFF309800D90EFF314800A9000F02CFC72
:10EE70003868012833D80028C14F00D0C14F2A205C
:10EE8000C1497A69920703D50A783A60401E491C45
:10EE90000028F6D1B948041D2046F1F799F9002859
:10EEA00007D079698907FAD521783960401E641C3A
:10EEB000F5E70220B5497A69920703D50A783A60E6
:10EEC000401E491C0028F6D12A20AF497A699207D2
:10EED00003D50A783A60401E491C0028F6D1FFF796
:10EEE00037FF0346AA4A30462946FDF7BDFE0446D1
:10EEF0003018291B089F3B1F049A9343A5A2FDF7D6
:10EF0000B3FE9E490968012966D8001900299C4C66
:10EF100000D09C4C00280AD09849091D62699207CC
:10EF200003D50A782260401E491C0028F6D10A2029
:10EF30009F496269920703D50A782260401E491CE6
:10EF40000028F6D10598F1F743F9002809D0616946
:10EF50008907FAD5059A11782160401E521C059246
:10EF6000F3E7022089496269920703D50A78226093
:10EF7000401E491C0028F6D10A208EA16269920722
:10EF800003D50A782260401E491C0028F6D1069855
:10EF9000F1F71EF9002809D061698907FAD5069AA8
:10EFA00011782160401E521C0692F3E70220774937
:10EFB0006269920703D50A782260401E491C002826
:10EFC000F6D10A207EA16269920703D50A782260F1
:10EFD000401E491C0028F6D17CA230462946079BDA
:10EFE000FDF742FE6549096801290E9B1BD80029DF
:10EFF000634900D0634900280AD0604A121D4C6959
:10F00000A40703D514780C60401E521C0028F6D1CA
:10F0100002205E4A4C69A40703D514780C60401E98
:10F02000521C0028F6D16AA230462946FDF71CFE84
:10F0300004463018291B694A3B46FDF715FE4F4927
:10F040000968012911D8001900294D4900D04D49FE
:10F0500000280AD0494A121D4B699B0703D5137833
:10F060000B60401E521C0028F6D15D4A30462946EE
:10F07000099F3B46FDF7F8FD0446F800C00FB900B4
:10F08000C90F7A00D20F0092019102903019291B0A
:10F09000FB0F544AFDF7E8FD04193019291B3F23E3
:10F0A0003B40514AFDF7E0FD34490968012911D878
:10F0B00020180029324900D0324900280AD02F4AAE
:10F0C000121D4B699B0703D513780B60401E521C21
:10F0D0000028F6D1454A304629460B9BFDF7C4FD72
:10F0E00004463018291B424A0A9BFDF7BDFD2349FF
:10F0F0000968012911D800190029214900D02149A6
:10F1000000280AD01D4A121D4B699B0703D51378AE
:10F110000B60401E521C0028F6D1364A3046294664
:10F120000C9BFDF7A1FD04463018291B324A0D9BAC
:10F13000FDF79AFD114909680129114A0DD80019F6
:10F14000002908D00F4A06E05169890703D53178B4
:10F150001160401E761C0028F6D128490E98091A25
:10F16000A94200D32946890800F03AFE24480068E5
:10F17000002800D0804700F045F8C046C0E00102FA
:10F180000090014000A00140472F0100D53C010044
:10F19000302F01000D0A232323204153534552549D
:10F1A000204020307825303858202323230D0A00B2
:10F1B0000A30010046554E4354494F4E3A20000054
:10F1C0004C494E45202020203A20000025640000B4
:10F1D0000D0A53503D253038580D0A00CF2F01003D
:10F1E000E52F0100F12F0100D92F01008E2F010022
:10F1F0009D2F0100AC2F0100B72F010000F8020283
:10F20000BCE00102F7480068012811D8002801D0AD
:10F210000B4800E0FC480C210A4A01E0002907D015
:10F2200043699B07FAD513780360491E521CF5E722
:10F230001E20FFF7C3FA00BF00BF00BF00BFFAE700
:10F2400000A001403A2F01008AB00646E448B066AB
:10F2500000F03AFAFFF77CFD0346E248041D012066
:10F260000590C502E04A20462946FDF7FDFC074609
:10F2700008942018DB4C0995E91BF36C3F22069299
:10F280001340DAA2FDF7F0FC2168012910D8C0195B
:10F290000029DD4900D0DD49002809D0221D4B6935
:10F2A0009B0703D513780B60401E521C0028F6D133
:10F2B000F36BD7A2089C2046099D2946FDF7D4FC94
:10F2C0000746291A2018336C069A134007D1D8A292
:10F2D000FDF7CAFCC34C2168012907D917E0CEA26B
:10F2E000FDF7C2FCBF4C2168012910D8C0190029C4
:10F2F000C54900D0C549002809D0221D4B699B078C
:10F3000003D513780B60401E521C0028F6D100274D
:10F31000CBA5B80030580090089809992A463B467A
:10F32000FDF7A2FC216801290FD80029B64900D0B9
:10F33000B649002809D0221D4B699B0703D51378D5
:10F340000B60401E521C0028F6D17F1C0D2FE0D10F
:10F35000736BBFA2089C2046099D2946FDF784FCDB
:10F36000074620189F4CE91BB36BBC4AFDF77CFC99
:10F370002168012910D8C0190029A34900D0A34948
:10F38000002809D0221D4B699B0703D513780B6019
:10F39000401E521C0028F6D1336CB14A089C20460E
:10F3A000099D2946FDF760FC0746326CD000C00F6E
:10F3B0009100C90F5300DB0F009301910290E019F7
:10F3C000E91BD30FA74AFDF74FFC3246C619A01917
:10F3D000A91B1546136C069A1340A34AFDF744FC7B
:10F3E00080490968012911D880190029864900D06F
:10F3F000864900280AD07B4A121D4B699B0703D51A
:10F4000013780B60401E521C0028F6D12E466B6C00
:10F41000964A089C2046099D2946FDF725FC07468B
:10F420002018E91B0796B36C914AFDF71DFC6D4A45
:10F430001168012910D8C0190029734900D07349F7
:10F44000002809D0121D4B699B0703D513780B6068
:10F45000401E521C0028F6D10798426E04236021FA
:10F460005C2004931A400B4600D003460693002A02
:10F4700000D00846079E33587E4A089C2046099DC6
:10F480002946FDF7F1FB074606983358E019E91BBA
:10F49000794AFDF7E9FBC619A019A91B079A536E13
:10F4A00076A2FDF7E1FB4F490968022911D28019C4
:10F4B0000029554900D0554900280AD0494A121D53
:10F4C0004B699B0703D513780B60401E521C002824
:10F4D000F6D10798C36C06466DA2089C2046099D8C
:10F4E0002946FDF7C1FB07462018E91B336D6B4A1F
:10F4F000FDF7BAFBC619A019A91B079F7B6D68A26F
:10F50000FDF7B2FB8619A019A91BBB6D67A2FDF719
:10F51000ABFB344909680129059C11D880190029E1
:10F52000394900D0394900280AD02E4A121D4B69AA
:10F530009B0703D513780B60401E521C0028F6D1A0
:10F540000798476B5D4A974237D2032087430026CE
:10F55000059CB00039580246049B1A43BA58082348
:10F560000343FB580C2505437D59009101920293FA
:10F5700003953B1808980999514AFDF775FB1949FD
:10F58000096801290FD800291F4900D01F49002808
:10F5900009D0089A4B699B0703D513780B60401E6E
:10F5A000521C0028F6D11B2E444A06D80798406BFF
:10F5B000361DB10040189042CBD30798406B111A0A
:10F5C000099A914201D8890800E0610200F008FC24
:10F5D0003C480068002800D08047FFF713FEC04673
:10F5E00022224B4DC0E00102302F01000D0A0D0A0E
:10F5F00023232320455843455054494F4E2025642A
:10F60000202323230D0A00000090014000A00140A8
:10F6100050433D25303858002C2045786365707480
:10F62000696F6E4E756D6265723D25640D0A00004E
:10F630002C205468726561644D6F64650D0A00008A
:10F6400052252D32643D253038580D0A0000000047
:10F6500053503D253038580D0A000000CF2F0100CF
:10F66000E52F0100F12F0100D92F01008E2F01009D
:10F670009D2F0100AC2F0100B72F01004558435FBB
:10F6800052455455524E3D253038580D0A00000061
:10F69000494353523D253038580D0A00C22F01000E
:10F6A0005343523D253038580D0A00004343523D24
:10F6B000253038580D0A0D0A0000000000F802023B
:10F6C000722F0100BCE00102F0B583B0344D2C680C
:10F6D000012C06D8601E8441204601F073FB0028EF
:10F6E000FAD10120EFF310810140019102D1EFF333
:10F6F000108072B62B48285A2B49695A814245D04E
:10F700002A68002A01D02A4E00E0284E1F23DB027F
:10F710000293284C022A27D205E01046214AA8521B
:10F7200082B2914232D087B2B9420A4600D8621CF6
:10F73000131A21482B5218040DD0E819001D9FB24E
:10F7400001E0002F07D073699B07FAD50378336077
:10F750007F1E401CF5E7A242DFD902981018DDE7B2
:10F76000304683B299420CD0024680B281420E46A6
:10F7700000D8661CA642F3D90298301883B2994289
:10F78000F2D108496852B01A0B4968520B4800215F
:10F7900029540198002800D162B603B0F0BDC046DC
:10F7A000C0E001020A0800000808000000900140C3
:10F7B00000A00140FF0700000C0800000F08000037
:10F7C000F0B58DB00793174600240C9409AA13C214
:10F7D00015E006986849F0F717FEF1F7DFF8C11752
:10F7E000401848406549F0F775FC009509A80622C5
:10F7F0003346F9F7C9FABDE0002C00D5BEE13878F0
:10F800007F1C25280DD0002800D1B7E10B9A511C90
:10F810000A9B9942F0D8099B9854641C0C940B9154
:10F82000EAE708940025397823390D2914D80120F6
:10F830007944097949008F44090F0F0F0F0F0F0FFB
:10F840000B0F060F0F0D05437F1CECE70820FAE7AE
:10F850000420F8E70220F6E7387801463039002422
:10F86000092902D9264639460BE000260A217143B0
:10F870000E18303E791C78780246303A0A2A0F4634
:10F88000F4D32E2817D14A1C48780146303909296B
:10F8900005D911464F1C2538532811D96AE0002498
:10F8A0000A2161430C18303C511C50780246303A12
:10F8B0000A2A0A46F4D34F1C2538532800D959E0A8
:10F8C0004000C0467844808840008744A000530030
:10F8D0005300530053005300530053005300530090
:10F8E0005300530053005300530053005300530080
:10F8F0005300530053005300530053005300530070
:10F900005300530053005300530053005300600052
:10F91000530053005300530053005300530053004F
:10F92000530053005300530053005300530053003F
:10F9300053009800530053005300530053005300EA
:10F940005300530053005300AD00B6005300600055
:10F950005300590053005300530059005300530003
:10F960005300DE0053005300BD005300D30053008A
:10F97000530098000C9C3FE70024744940420F005C
:10F98000791C38780F4625385328F3D898E707991B
:10F99000C91D07208143086807914968F1F78CF871
:10F9A00000210690F0F75AFF00280BD10B99481C54
:10F9B0000A9A904206D8099A2D2353540899491C53
:10F9C0000C910B900798083007900698F0F7E6FF27
:10F9D0000095C2178118514009A822463346F9F70D
:10F9E000D3F90B98411C0A9A914200D9F1E6099A81
:10F9F0002E2313540B910C98401C0C90E9E60798A9
:10FA000002C807900096019509A8102239E00B98CA
:10FA1000411C0A9A9142ADD8099A252313540B919F
:10FA20000C98401C0C90A5E70B9A511C079C201DBC
:10FA30000A9B994239D907909CE7079802C807901A
:10FA4000009509A82246D3E6079901C907910999AB
:10FA50000A9A089E02E0401C002E8BD40378002BEB
:10FA600088D00B9D6C1C9442F5D84B55761C0C9697
:10FA70000B94F0E7079802C807900096019509A833
:10FA80000A222346F9F71EFA74E7079B10CB102CC5
:10FA9000079308D300202146401C0A09FF2911467C
:10FAA000FAD806280AD8082009E02368099CA3543C
:10FAB000089A521C0C920B9107905BE7401C069031
:10FAC00009230C980B9D099905910A9E04940DE059
:10FAD000202104463046059E715506462046049C6A
:10FAE000401C15460146089100290AD45B1E069960
:10FAF000994206D26A1CB242EAD9089908910029B3
:10FB0000F4D50C900B950898002800D532E7012613
:10FB1000082501E06D1E3601022DFBD2204631463C
:10FB2000F0F7D8FA0F28F6D80C98059009980390AA
:10FB30000A9806900B9D20463146F0F7CBFA691CD7
:10FB4000069A914204D90899089100290CD511E030
:10FB50000C4A125C039B5A55089A521C0D4605929A
:10FB600011460891002905D47043241A3009102E3B
:10FB70000646E0D205980C900B95FBE620460DB0AA
:10FB8000F0BDC0468C22010070B588B00022032869
:10FB900003D9D243104608B070BD7F4CC34D2A51E3
:10FBA0000F4B104EEE5081231E010123AB552860F0
:10FBB0002C1962600128EDD8079300220692059265
:10FBC000049203230393029201920091411E884103
:10FBD000694600F027FD0246104608B070BDC046D9
:10FBE00004080000FFC0FFC0F0B583B00C4600233E
:10FBF000D943012C56DB074602910126EFF310850D
:10FC0000354002D1EFF3108072B65849584A505C23
:10FC1000002800D0A3E056545E48115A5E48105A9E
:10FC20000196F202161A814240D832465218A24278
:10FC300040DB00930295A642354600DB25464C4941
:10FC40000818001D39462A46F0F794FAA642484E95
:10FC500004DA7919621B301DF0F78CFA4E48305ADD
:10FC6000001981B24D4A914201D94D494018029D77
:10FC7000009B4949705230464A4E805D002865D14C
:10FC8000EFF310850198054002D1EFF3108072B6B2
:10FC9000374A4048115A4048105A884232D14248A7
:10FCA00013524FE00C46204603B0F0BD42425218BA
:10FCB000A242BEDA3B4A2E4EB25C002A0CD03A4A2F
:10FCC000B25A51188AB2354CA242284C029F01D92F
:10FCD000334A8918304A02E0244C2F4A029F335598
:10FCE000B152421A89B2884202D22C488018421C72
:10FCF00093B22F4801212FA200F0E8F83C46002DD6
:10FD0000D1D128E0019F9755884201D82348401C53
:10FD1000421A90B2800A01D0019882022248144F00
:10FD20003A52386801280DD8431E9841104B591893
:10FD3000091D92B21D4B00F08BFE009B002801D0E4
:10FD40000B488355002D029D00D162B60748084933
:10FD50000B54002DA7D162B6204603B0F0BD212080
:10FD60000201044804A108A3FFF754F80E0800009C
:10FD7000C0E001028630010074726163655F6F75D7
:10FD80007470757400000000545241434520425580
:10FD9000535900000A08000008080000FF0700008F
:10FDA00000F8FFFF0F0800000C080000F9FF00003A
:10FDB00002FF00000D0A5472616365206275666679
:10FDC00065722069732066756C6C2C20646973639E
:10FDD000617264732025752062797465730D0A0061
:10FDE000F0B587B00546002606960596049603965C
:10FDF0000296800701D007B0F0BD019102A814213E
:10FE000026A2FCF731FF29490968012911D80029E8
:10FE1000274900D0274900280BD002AA01E000287A
:10FE200007D04B699B07FAD513780B60401E521C14
:10FE3000F5E701990029DED0204C3746B8002B5851
:10FE4000D80724D0581EA04204D31B4818181C4AB7
:10FE500090421CD802A814211AA2FCF705FF1349EE
:10FE60000968012911D80029114900D01149002839
:10FE70000BD002AA01E0002807D04B699B07FAD5F6
:10FE800013780B60401E521CF5E7761C01997F1C0D
:10FE90008F42B0D2322ED1D3ADE7C0460D0A4261B7
:10FEA000636B74726163653A200D0A00C0E0010261
:10FEB0000090014000A00140FFFFFFFCFFFF020097
:10FEC000FEFF0100253038580D0A000081B0F0B562
:10FED000C4B00E4607464993812000012F49085CB3
:10FEE000002845D002920120050204A82946F0F717
:10FEF0005AF9FCB20021C8430C2C3AD8721E032ACE
:10FF000037D82748005DB042084632D3F80535D5CA
:10FF10000021B8050DD404A801904018691AA20068
:10FF200022A39B582E4AFCF79FFE0198F0F750F948
:10FF3000014678050ED404AF7818691AB20029A3D7
:10FF4000D218121F1368264AFCF78EFE3846F0F7C7
:10FF50003FF90146029A04AE70180C46691A49AB83
:10FF60000393FFF72DFC01193046FFF73DFE00E03B
:10FF7000002044B0F0BC02BC01B00847FEF7E8FE28
:10FF8000034604A8019007A22946FCF76DFE0198DC
:10FF9000F0F71EF90146B805BDD5CAE7C0E0010279
:10FFA000B848010025313075207C20002A3001003E
:10FFB000803001007A300100593001002430010006
:10FFC00045300100733001006C30010067300100E2
:10FFD0001D300100303001004030010015300100BB
:10FFE000393901005F3001004B300100523001000F
:10FFF0003630010000000000F0B581B00B46012052
:020000040001F9
:10000000EFF31084044002D1EFF3108172B6990F20
:1000100007D0022001212DA2FFF758FF002C3DD16F
:1000200041E02249224D00276F54224AAB5A224A0E
:10003000AE5AF3189EB2F60A01D0204E9B19AB526D
:10004000EFF31086064002D1EFF3108372B6AA5A7E
:100050001C4BEB5A934202D116482F521AE06854B7
:10006000934201D8164B5B1C9B1A99B2890A00D0A7
:10007000830210482B52286801280BD8411E884162
:10008000A918091D9AB2104B00F0E2FC002801D01B
:1000900006482F54002E03D0002C04D001B0F0BD30
:1000A00062B6002CFAD162B601B0F0BD0F080000B4
:1000B000C0E001020C0800000A08000000F8FFFF81
:1000C000FF07000008080000F9FF000055415254E6
:1000D000204572726F722025780D0A0010B5044613
:1000E000FEF7EEF8A08A002800D010BDFDF7EAFE6A
:1000F000034908620861486C401C486410BDC04652
:100100003099010210B50446FEF7DAF8A08A0028FB
:1001100000D010BD0A4CA06C401CA064FDF7D2FEBC
:100120006062606C002805D0FDF7CCFE60650020A1
:10013000606410BDA06920650120606410BDC046E8
:10014000B096010210B50A2000242146FBF7D4FC2A
:1001500009202146FBF7D0FC0124204600F038F8A6
:100160000E200421FBF7C8FC0549204600F05AFA8E
:10017000A2021549154B204600F028FB10BDC046D1
:10018000DC940102B0B50E2000242146FBF7B4FC3C
:100190000D202146FBF7B0FC0124204600F018F8A2
:1001A0000A2004252946FBF7A7FC09202946FBF76E
:1001B000A3FC2046F9F77AFAA2020349034B204632
:1001C00000F004FBB0BDC046E0CD0102050A01000D
:1001D00070B5012801D9012070BD48224243734BFC
:1001E0009C58A5691F218D43A5610625A5600F2593
:1001F00025629C18A27C002A05D1627C002A02D1CB
:10020000227C002A14D06368002B11D4251D0B40DA
:10021000012216469E400C4B1E60BFF34F8FBFF36A
:100220006F8F2B68002B03D40B409A4007490A605C
:10023000002803D0012804D1092000E00820F9F7A4
:10024000DFFB0020A06170BD80E100E080E200E003
:10025000F0B585B00D460278E348C368934219D0E3
:10026000446D944216D08368934203D0016D91424D
:1002700000D07FE09B1A591E8B41049348215943BB
:10028000032D46D14418E16900294ED01C340020CA
:1002900020606DE09B1A5A1E93410493032D1AD1DE
:1002A000039548225A438418A26B0121EFF310856D
:1002B0000D4002D1EFF3108772B6A7691026B7433D
:1002C000A761A669002E01D118342160002D00D14C
:1002D00062B6039D0CE048215943421891691832D7
:1002E000302902D0116810294CD1802111600022E0
:1002F0004821594340180021816301628162243002
:1003000000210160002A33D004A82946904705B097
:10031000F0BD421891691832302902D011682029A5
:1003200039D180211160002216E00395E26B01268D
:10033000EFF31085354002D1EFF3108172B6A16959
:100340002027B943A161A169002901D11834266091
:10035000002D00D162B6039D482159434018002169
:10036000C163C1624163303000210160002ACBD1FA
:1003700005B0F0BD00920E4A2E329C480D490E4B3E
:10038000FEF748FD10680093019098480949084A13
:100390000A4BFEF73FFD106800930190044A243297
:1003A00092480449054BFEF735FDC046FC94010216
:1003B000B102000002310100D7300100BB30010062
:1003C000F0B585B0049048210A464243864B9C58BC
:1003D000E6690F2535409A18167C002E31D04F2043
:1003E00040026169014200D185E0A069042188438F
:1003F000A06102202062012081076918D161D36BBE
:10040000EFF31084044002D1EFF3108572B69569C2
:100410002026B54395619569002D00D173E0104603
:100420003C30002C00D162B600240460D4625463D6
:10043000303200201060002B63D004A8984705B02C
:10044000F0BD0C2D5DD8C0467D442D796D00AF44C4
:1004500067586B580658A163585858580600956954
:10046000202D04D0154618352D68302D49D1156B37
:10047000566B3432AE4217D26669360714D56468BB
:1004800015686E1C166048431818C06A44550498D5
:100490000C4644431A19156B566B3432AE4203D2E4
:1004A0001C5966693607EAD41268AA4229D1414329
:1004B000585882690524A24382615A18D36B0121DE
:1004C000EFF31080084002D1EFF3108472B6946904
:1004D0002025AC4394619469002C02D11446183451
:1004E000216014463C34002800D162B6002121600E
:1004F000D16251639CE70C2D00D176E7012D00D12C
:1005000073E705B0F0BD15461835286010463C303D
:10051000002C00D187E787E70420206205B0F0BDFA
:100520000120206205B0F0BD082525621646183668
:100530009569102D02D03568302D4BD10396566A3F
:1005400015462835976AB74228D1A0690221884309
:10055000A061936B0121EFF31080084002D1EFF30B
:10056000108472B6039E34681027BC43346034682C
:10057000002C00D1316014463834002800D162B616
:100580000021216029601162243200201060002BBC
:10059000B7D052E70220206205B0F0BD2A68B2420F
:1005A000AFD262699207ACD52A68561C2E604843C8
:1005B0001818006A805C206004980A4642439D181F
:1005C000AC6A6E6AB4429CD228359C586269920724
:1005D000EAD496E7316800900191044804A1094AE1
:1005E00009A3FEF717FCC046FC940102A1300100EC
:1005F000756172745F6972715F68616E646C657257
:10060000000000003D030000556172742025642045
:10061000737461746520676F65732077726F6E679E
:1006200020256400F0B585B00E460546022804D3A7
:10063000002E02D1012005B0F0BD002D03D0012D08
:1006400008D1092400E008242046F9F7E1F9204602
:10065000FEF7B4F848216943E74A505883691F24DC
:100660000294A3438361062383600F2301930362F3
:1006700057180023BB62BB63FB633B627B62FB6278
:100680003B63317F3974727F7A74B27FBA7404939A
:100690007B637368B268F468920022435B1E032B8D
:1006A0000ED8C0467B441B795B009F4401050307BD
:1006B000082304E0282302E0182300E038231A432B
:1006C000C260C907090F72699201D2B28918B26972
:1006D0009207920E8918491C81607961316901295C
:1006E00001D122210161012D5CD831680E2959D236
:1006F0003846123003900324002D01D0204600E03C
:1007000004204C432D490E19B178F9F711FA3968D4
:10071000CA68802510462843C8602848005D737861
:100720001B021818C862AA43CA60F9F749FA03986D
:100730000078002809D1384611300078002804D10B
:10074000384610300078002827D07868002815D463
:10075000032102468A431B4953588407E40EFF26AF
:10076000A640B343A5401D435550029901400120C6
:100770008840A2490860144908600EE08107C90E4C
:10078000FF228A40019C0440083C032084430C481B
:10079000235893438D401D4325500120B861049890
:1007A00005B0F0BD02480349DA22034BFEF732FBE5
:1007B000A130010014310100F130010020200100BE
:1007C0001CED00E000E400E000E100E0F0B58FB0D7
:1007D0000E900125002900D14BE00393049105926E
:1007E000002A00D145E00121EFF3108201910A4077
:1007F00002D1EFF3108172B64827029747437E4932
:10080000CE19B5690023302D23D831461831C046A2
:100810007D442D796D00AF442024262626262626E9
:1008200026262626262626265E2626262626262630
:100830002626262626262626182626262626262666
:10084000262626262626262618000223002A0CD035
:100850000CE0402D01D0802D05D10123002A04D0C9
:1008600004E020240C60002A00D162B61D46002B53
:1008700002D028460FB0F0BD002575630399F163DF
:100880000499F162059931635B4CE359596913226C
:10089000D202114205D0062199600F2119627169B7
:1008A0009960317C00290CD0F56109950895079570
:1008B00006950D950B9502210A91012810D017205D
:1008C0000FE0717C9A6900292CD0952002439A612F
:1008D00028460FB0F0BD30240C60002AC5D0C5E713
:1008E0001920049F0C907068002805D41F2108402F
:1008F000019981404148016014209861B06806A9BF
:10090000F9F7CEF90E980299414360188068615852
:100910003B4A0092091D3A46059BF9F731FA2846F1
:100920000FB0F0BD3436110602D580218A439A619A
:1009300031680025059A91422DD205955D694F21B8
:100940004A0215421BD1E90502D4029CF24F0AE08B
:10095000596833685C1C3460029C6043EE4F381861
:10096000C06AC1540E98214641437E18736B346BA4
:10097000A34238D234367B585D691542E3D0022158
:100980001962019EB10729433546E34CEFF310820B
:10099000324006D008E02946019EEFF31082324033
:1009A00002D1EFF3108372B6029B4343E0188369D0
:1009B0002024A34383618369002B05D0002A08D03B
:1009C000C26B002A0AD154E7034618331E60002A7E
:1009D000F6D162B6C26B002A00D14AE70EA8904752
:1009E00028460FB0F0BD2946059D019E3C46EFF319
:1009F00010823240D5D0D7E7FC94010280E200E0BB
:100A00005102010080B5012082020249024BFFF72A
:100A1000DDFE80BDE0CD0102050A0100B0B582B067
:100A200079208400E54D285D01A9087065208000CB
:100A30002818F2F7CDFF2F20C000285829190122CD
:100A4000024BFFF7C3FE02B0B0BDC0461D0A010055
:100A5000F0B591B010900126002900D19BE00393DE
:100A60000591002A00D196E007900121EFF3108054
:100A70000291084002D1EFF3108172B6049248232C
:100A8000069307994B43D649C9188D690026302D26
:100A90006ED80C461834AD00374602A675593E464E
:100AA000AF46C046790B0100810B0100850B0100A8
:100AB000850B0100850B0100850B0100850B0100F2
:100AC000850B0100850B0100850B0100850B0100E2
:100AD000850B0100850B0100850B0100850B0100D2
:100AE000850B0100690B0100850B0100850B0100DE
:100AF000850B0100850B0100850B0100850B0100B2
:100B0000850B0100850B0100850B0100850B0100A1
:100B1000850B0100850B0100850B0100850B010091
:100B2000850B0100170C0100850B0100850B0100EE
:100B3000850B0100850B0100850B0100850B010071
:100B4000850B0100850B0100850B0100850B010061
:100B5000850B0100850B0100850B0100850B010051
:100B6000850B0100690B0100022600280CD00CE067
:100B7000402D01D0802D05D10126002804D004E0AD
:100B800010252560002800D162B6002E069D944FE6
:100B9000049C079802D0304611B0F0BD00268E624A
:100BA000039A8A63059A0A624C620A7C002A0BD077
:100BB0000C960B960A96099608960E9602220D92AE
:100BC00001282DD018202CE08A7C2831002A3BD027
:100BD0000A68A24216D22B464343FA585469A40726
:100BE00010D50868441C0C60F918096A085C10608C
:100BF0001098294641437A1811462831936A526A5F
:100C00009342E8D345437859816982220A4382613D
:100C1000304611B0F0BD302525600028B4D0B4E7CF
:100C20001A200F90C86808A9F9F73AF810984543B8
:100C30007A597819C0683949009105992346F9F71E
:100C40009FF8304611B0F0BDFB589A69140602D5E2
:100C50008024A2439A610A680026049882422ED218
:100C60005D694F225202154207980AD0022119628B
:100C7000029EB10729431FE028315D6915423E46B7
:100C8000F4D137465C69A40702D40699544E0AE0B1
:100C90000C68661C0E6006994843514E3018006A75
:100CA000005D186010984143735871188C6A4E6A41
:100CB000B442E1D329463E46069D494F01E0314604
:100CC00007985A6A002AFCD1EFF31082029B1A405F
:100CD00002D1EFF3108372B645437819836910246B
:100CE000A34383618369002B05D0002A09D0826B5E
:100CF000002A0BD14FE703461833029C1C60002AE0
:100D0000F5D162B6826B002A00D144E710A8904763
:100D1000304611B0F0BDC046FC9401025102010002
:100D2000B0B5264900684A68824202D10D1D0020F4
:100D300016E080228A58824203D10D468035012078
:100D40000EE0FC228A58824203D10D46FC35022077
:100D500006E02F22D2008B5883422ED18D1803201B
:100D60007C2242438C18A068012814D0002824D18A
:100D700040342046F3F71BFA01462046F3F7EDF91D
:100D80002046F3F714FA002817D006C828680C4B41
:100D9000FFF75EFEB0BD40342046F3F708FA014687
:100DA0002046F3F7DAF92046F3F701FA002804D0D9
:100DB00006C82868024BFFF74BFEB0BD58BE0102C3
:100DC000210D010048214143054842189269D2068D
:100DD00001D4002070474058416901200840704705
:100DE000FC94010280B511480078C00110490978CF
:100DF000890101430F480078400108430E490978F2
:100E0000090101430D480078C00008430C490978E6
:100E1000890001430B480078400008430A490978DB
:100E20000143C8B2F3F774FC80BDC046E09E0102E6
:100E3000AE9601021D90010264EA010299AD010221
:100E4000E19E010224A3010225A30102F0B587B0AF
:100E500001460127022505283A4600D02A460020EF
:100E60000929014600D01146C900374A54180E21FD
:100E70000591615EFDF7AEFA1026A15F3846FDF7D9
:100E8000A9FA1227E15F2846FDF7A4FA0695142572
:100E9000615F03200490FDF79DFA0598235EA05F33
:100EA000E15F625F00AD07C528A2069F3846049D3A
:100EB0002946FFF70BF82046263004263146FBF77B
:100EC00049FF2620235E2820205E2A21615E2C22F5
:100ED000A25E00900191029224A238462946FEF7B4
:100EE000F5FF27463E3738463146FBF751FF3E2097
:100EF000235E06983C5EB95F0622BA5E00940191BB
:100F0000029221A207462E462946FEF7DFFF56240D
:100F10000D4D285FFBF730FF2B5F2C4621A2384692
:100F200031463546FEF7D2FF264658363046FBF7A7
:100F30000FFF5820235EF05F00901FA2384629461D
:100F4000FEF7C4FF07B0F0BDC4A00102546F4620F5
:100F5000616E742064656C6179732025642025645A
:100F60002025642025640D0A0000000050446F41D4
:100F70002064656C617973202564202564202564D4
:100F80002025640D0A00000050446F41206761690C
:100F90006E732025642025642025642025640D0AB5
:100FA0000000000050446F4120616E742073706136
:100FB00063652025640D0A0050446F4120616E670F
:100FC0006C65206F666673657473202564202564E4
:100FD0000D0A0000F0B587B015467A4B1A680F2449
:100FE000A2432F783A431A60774C23462C3B774A2A
:100FF0001A60049003462246283A12681207FAD56E
:10100000734E092F029306D9754A326072600C2F15
:1010100009D175480FE0042F07D9704A3260704A31
:101020007260092F06D3714805E06A48306070602D
:10103000694800E06B486E4A1060EB7AFF2B039121
:1010400002D10020B0620AE003210B406948C05C75
:1010500040220243B2620220674AFEF737FF029F36
:101060000021384605952A460B46FBF7FDFE06464D
:101070000225032161A2284601913346FEF726FF8F
:1010800006963046FCF7C4FB012104980091084005
:101090002CD13D4033D1604900283AD1002D1ED0DB
:1010A0006548A062E06220636063644860626448EF
:1010B0000860152085046E1C8E608D6064242046B7
:1010C0000F46F8F77DFD3E603D602046F8F778FD5D
:1010D000281D386003215BA24E48FEF7F7FE0598F5
:1010E000007BFAF7CFFF069807B0F0BD2E46054605
:1010F0000698FCF719FF284635463D40CBD02E46D2
:1011000005460698FCF78CFB2846354642490028E0
:10111000C4D042480861424848614248886115206D
:10112000C8614148016840220A4302600721080360
:10113000274B5A69824300984003101858610522D2
:10114000039842432A4803689818334E766B4778D1
:101150000F40995C0907490EC919CA03334B334044
:101160009A18C9015118324A89182B4A51632A49E1
:10117000896B3822914382785207920E8918042293
:101180000A4325498A63124B19690279019E32404C
:10119000C0784007C00E80181F22914308181861BC
:1011A00055204003411C216020606420F8F708FDB1
:1011B000204A18483146039BFEF788FE1649002D49
:1011C0008DD06DE7040400402C60004000040080D6
:1011D000000600400F040F04A92A010003040304C1
:1011E00000040004DA2B0100782901000B2D010016
:1011F000489401023C2E0100403101005048592022
:10120000706172616D732073657473202530387856
:101210000D0A0000020800009060004012A83E0085
:101220009DD79B5AD579BD49340200403F0080FFCD
:1012300040400000223101002008820002D50F004A
:10124000020255007577625F72785F696E69740D8E
:101250000A00000080B52248002101702248007871
:10126000C0012049097889010143204800784001E4
:1012700008431F490978C90001431E4800788000CF
:1012800008431D490978490001431C480078084378
:10129000C0B2F3F73DFA80BD80B51148012101705D
:1012A00010480078800110490978C90101430F48AE
:1012B0000078400108430E490978C90001430D48F0
:1012C0000078800008430C490978490001430B4825
:1012D0000078084310210143C8B2F3F719FA80BD22
:1012E00064EA0102AE960102E09E01021D90010235
:1012F00099AD0102E19E010224A3010225A301028E
:10130000F0B581B01820FDF759FA1920FDF756FA0B
:10131000002420462146F8F727F820462146FAF710
:1013200035FE012603257F23304629462A46FAF753
:1013300045FF3046FBF7EAF802273846FBF774FD15
:1013400030463146FCF7C2FD03A238462946FEF777
:10135000BDFD204601B0F0BD7577625F6F70656EB0
:101360000D0A0000F0B581B0164600910446002039
:1013700001273946FCF7D2FFEFF310853D4002D13B
:10138000EFF3108072B62720400170430A21EEF778
:10139000A1FE0246002C02D00020009901E00220AC
:1013A0000021FBF7B9F80446FBF780F9002D00D1C6
:1013B00062B6204601B0F0BD70B504460E4D2968F6
:1013C0000F2001400629FAD029680140072912D1CF
:1013D0000120EFF31086064002D1EFF3108072B6C1
:1013E000FCF770FDFA30A860002C01D0FAF7E0FE9F
:1013F000002E00D162B670BD00040040F0B581B08F
:101400001D460E460446022A09D1012738463946B0
:10141000FCF784FF00960022384629460FE0174665
:1014200001200021FCF77AFF012F04D10096002053
:101430002946024603E00096022000210A46234680
:10144000FBF74CF90446FBF731F9204601B0F0BD3B
:1014500070B5002801D0012070BD0325A9020F48F6
:1014600002680F4B535000249460012253030D4E29
:101470003360BFF34F8FBFF36F8F0B4E3360036842
:101480005A50847204811020F8F7BAFA022007A299
:101490002946FEF71BFD204670BDC0468C95010213
:1014A00051E5CC1A80E100E080E200E0574454208E
:1014B000636C6F73650D0A000FB47CB50C0009AD49
:1014C00001D0611E00E0002101910090074B6A46A7
:1014D0002946089800F012F9002C02D0009A002149
:1014E00011707CBC08BC04B018470000351E010018
:1014F0007CB51D4616460C0001D0611E00E000219F
:1015000001910090054B6A462946304600F0F6F8F6
:10151000002C02D0009A002111707CBD351E010004
:101520002021020C01D010211046020A01D01046E1
:101530000839020901D01046091F820801D010465F
:10154000891E420801D0881E7047081A70470000A3
:10155000004870470890010202E008C8121F08C145
:10156000002AFAD170477047002001E001C1121F24
:10157000002AFBD170470000F0B51FB486B009986F
:10158000089A030D0021024314D05148514A1818FB
:10159000504305141198012810981AD0281A401C9D
:1015A00000264D4F4D49009601910490002812DA13
:1015B000444211E01198012449A3012801D1109857
:1015C000C1430698119A84600360C26041600BB009
:1015D000F0BD4042E4E70446210500203F4A001CDC
:1015E00051410391029012E0E00707D032463B469A
:1015F00001990098EFF736F80191009032463B468A
:1016000010461946EFF72EF806460F466410002CD8
:10161000EAD10498039B0028029A0999089806DAEF
:10162000EFF720F8019B009AEFF71CF805E0EFF7C1
:1016300081F8019B009AEFF77DF804460E460022E0
:10164000284BEFF743FC03D80020C043014607E0D6
:101650000022254B20463146EEF752FFEFF716FCED
:10166000102409E0002C0ADB0A220023EFF740FADD
:10167000079B30321A55641E02460A43F2D11122EA
:10168000641C079B121B1C19119B012B03D0012307
:1016900008430ED10AE0084304D011201090002026
:1016A000119077E71098151A6D1E0BE01098824282
:1016B00002DD00236D1C03E0824201DA00236D1E6F
:1016C000002BEED0069811998260C16030C07EE791
:1016D00001FCFFFF104D0000000014400000F03F2F
:1016E000300000000000F0430000E03F30380A28DE
:1016F00001D201207047002070470000FFB597B06D
:101700000646002518E2252877D100242746FD4902
:10171000049400E00443761C32780120203A904083
:101720000842F7D130782A280ED0022230780146BC
:101730003039092916D804990A23594330394018F9
:101740001443761C0490F1E7189802C8049118908D
:10175000002904DA01204003044348420490022097
:101760000443761C30782E2814D10420044370786A
:10177000761C2A2809D11898761C80C8189009E090
:101780000A214F43303FC719761C30780146303963
:101790000929F5D930786C2810D006DC4C281AD0ED
:1017A00068280ED06A2817D104E0742813D07A284C
:1017B00012D110E00120400504430CE0012109058D
:1017C00001E0032109050C437178814203D1012016
:1017D00000052418761C761C3078119066280BD0F2
:1017E00013DC58287DD009DC00287BD04528F6D0B2
:1017F0004628F4D047281AD1A5E118E0632835D04F
:10180000642870D0652812D19DE170286CD008DC66
:101810006728F1D069287BD06E280DD06F2806D1BB
:10182000BAE073282ED0752871D0782859D01A9A2A
:10183000199990476D1C7EE16002400F022809D083
:1018400003280DD00428189801680DD00D60001DE4
:10185000189070E11898EA1701680D604A60F6E781
:10186000189801680D80F2E70D70F0E718986A4645
:1018700001781172001D18900020507202A800908B
:10188000012005E0189802C8189000200091C0437C
:1018900061070DD5002101E00199491C0191B94270
:1018A00012DA8142F8DB009A515C0029F4D10BE096
:1018B000002101E00199491C01918142FADB019A62
:1018C0000099895C0029F5D1019904981A9B471A5F
:1018D00021463846199A00F097FA0199401945189F
:1018E0000BE04FE02CE113E04EE000980099007807
:1018F000491C00911A9A199990470198401E01902D
:10190000401CF2D1214638461A9B199A10E137E063
:101910000A200021009001916002410F022907D0A6
:10192000189A01CA1892C2179446032908D00AE0EF
:101930001898C01DC108C90005C91891944607E050
:1019400000B2C2179446042902D140B2C1178C4696
:1019500000226146944506DA0A4600214042914140
:101960008C462D2102E0210504D52B216A461173F6
:10197000012103E0E10701D02021F7E7029155E0C2
:101980000A200AE0102008E0102000900021042026
:1019900004430191082703E00820002101910090F1
:1019A0006002410F022907D0189A01CA189200223A
:1019B0009446032908D008E01898C01DC108C90042
:1019C00005C91891944603E080B2042900D1C0B241
:1019D00000210291210729D51199702906D0009A7A
:1019E0001021019B4A401A4305D00EE040216A466F
:1019F0001173012108E06146014306D030216A4697
:101A000011731199517302210291009A0821019BCF
:101A10004A401A430AD16146014301D1610705D505
:101A200030216A46117301217F1E029111995829B4
:101A300004D035A10E910DA90D910DE037A1F9E764
:101A40006146019B009AEFF753F80E9B8C469B5C16
:101A50000D9A521E0D92137061460143F0D10D98FC
:101A600005A9081A20300190600703D50120000461
:101A7000844300E001270198874201DD381A00E025
:101A80000020019900904118029809180498401A02
:101A90000490E00306D421461A9B199A049800F09A
:101AA000B3F94519002706E003A81A9AC05D1999F1
:101AB00090476D1C7F1C02988742F5DBE0030CD534
:101AC00021461A9B199A049800F09EF9451904E0E2
:101AD0001A9A3020199990476D1C0099481E009061
:101AE0000029F5DC08E00D980D990078491C0D914E
:101AF0001A9A199990476D1C0199481E0190002966
:101B0000F1DC63E1092801003031323334353637F6
:101B10003839616263646566000000003031323339
:101B200034353637383941424344454600000000D9
:101B300000F05AF94519761C3078002800D0E2E50B
:101B400028461BB0F0BD600700D406271898C01DBA
:101B5000C108C90048680A680831C30FDB0718913B
:101B6000190001D09CA108E0210501D59BA104E04A
:101B7000E10701D09AA100E09AA1430011985B0807
:101B8000109165280CD006DC452809D046281DD0C8
:101B9000472841D141E0662818D067283CD13CE075
:101BA0000021112F01DB112000E0781C0191009031
:101BB00008A911A8FFF7E0FC139905910021119ADB
:101BC00015927F1C12980197009150E00120C007E8
:101BD00003900120019008A9009711A8FFF7CCFC01
:101BE000139A149905920022119B00921298159352
:101BF000059A0192002901D0104602E0791C401894
